:1000000000000120C18E0000E98E0000EB8E000090
:10001000ED8E0000EF8E0000F18E00000000000069
:10002000000000000000000000000000F38E00004F
:10003000F58E000000000000F78E0000F98E000031
:10004000FB8E0000FB8E000095930000FB8E0000ED
:10005000A1480000FB8E0000FB8E0000FB8E00001C
:10006000FB8E0000FB8E0000FB8E0000FB8E00006C
:10007000FB8E0000FB8E0000FB8E0000FB8E00005C
:10008000FB8E0000E1950000FB8E0000FB8E00005F
:10009000FB8E0000FB8E0000FB8E0000FB8E00003C
:1000A000FB8E0000FB8E0000FB8E0000FB8E00002C
:1000B000FB8E0000FB8E000000000000000000002E
:1000C000FB8E0000FB8E0000FB8E0000FB8E00000C
:1000D000FB8E0000FB8E0000FB8E00000000000085
:1000E0000000000000000000000000000000000010
:1000F0000000000000000000000000000000000000
:1001000000000000000000000000000000000000EF
:1001100000000000000000000000000000000000DF
:1004000010B5054C237833B9044B13B10448AFF34E
:1004100000800123237010BD5C020020000000005A
:100420004004010008B5034B1BB103490348AFF377
:10043000008008BD000000006002002040040100B0
:10044000154B002B08BF134B9D46A3F5803A0021A6
:100450008B460F461348144A121A0BF074FB0F4BCD
:10046000002B00D098470E4B002B00D0984700205F
:10047000002104000D000D48002802D00C48AFF305
:1004800000800BF0CDFA2000290009F0BFF80BF036
:1004900015F900BF00000800000001200000000066
:1004A000000000005C020020440700200000000063
:1004B0000000000007B5002300931A4619460348C0
:1004C00008F034FB03B05DF804FB00BF78020020A5
:1004D00007B5002300931A461946034808F026FB87
:1004E00003B05DF804FB00BF8002002007B50023C5
:1004F00000931A461946034808F018FB03B05DF84C
:1005000004FB00BF88020020437923B180680030DB
:1005100018BF01207047184670470000016838B5C1
:10052000002304468360838000293DD00B7C062B8A
:100530003AD11E4B1B68002B36D01D4A1D4807F0D0
:1005400040FB08B143692371236818680BF0ACF8CD
:10055000194A60712168174807F033FB054608BB4C
:100560001649174808F022FB0A226179144808F05E
:100570009FFB1449124808F019FB0A222179104800
:1005800008F096FB0E4808F021FB2B460A4A21682A
:10059000084807F065FB084A2168064807F011FB88
:1005A000054608B11435A56038BD00BFE80300203A
:1005B000B6FE00004C05002013F90000E6EF000035
:1005C000A00500200BF6000010B504460160FFF7FF
:1005D000A5FF204610BD704741790C4A002352F810
:1005E0002300884203D10A4A52F82300704752F888
:1005F000230028B942F82310054A42F82300704727
:100600000133052BEBD10020704700BF980200207A
:10061000AC02002010B50A4A4079002352F823406A
:10062000844203D1074A42F8231010BD52F82340F8
:1006300014B952F82320F5E70133052BEED1F4E786
:1006400098020020AC02002070B52DED028B9AB00C
:100650000446FFF7C1FF054608F09AFF854200F205
:10066000B98006231622617905A808F033F83721EE
:1006700005A808F03FF80022114605A808F054F933
:10068000002108EE100A05A808F0E6F9564A21688C
:1006900008EE900A554807F094FA554A2168054635
:1006A000524807F08EFA20B118EE101A406903F094
:1006B00053F85049504808F079FA0A2261794E48B7
:1006C00008F0F6FA4D494C4808F070FA18EE100A96
:1006D0000AF02CFC022602460B460096464808F01B
:1006E000ADFB4749444808F061FA18EE900A0AF059
:1006F0001DFC009602460B463F4808F09FFB41490F
:100700003D4808F053FA3C4808F060FA002D65D0E7
:10071000B5EE408AF1EE10FA60D0F5EE408AF1EEC7
:1007200010FA5BD0B4EE488AF1EE10FA56D1F4EE2E
:10073000688AF1EE10FA51D100213C220BA80A91EF
:100740000BF001FA696940220AA80CF0BCF92F21CC
:100750000AA80CF04FF928B96B69032240210AA8B6
:1007600003F022FE28490AA80CF035F918EE100A09
:1007700002A903F0CDFD254807F004FD40B1244B4C
:1007800093F9003023B902AA0AA9204807F001FF13
:100790000AA80CF06AF91AAB1844482300F8413C47
:1007A00002A918EE900A03F0B3FD184807F0EAFC1E
:1007B00040B1174B93F9003023B902AA0AA9134894
:1007C00007F0E7FE08F0E4FE00F56A511831204614
:1007D000FFF720FF1AB0BDEC028B70BD08F0D8FE09
:1007E00000F59C510831F2E7EBEF00004C050020CA
:1007F000F0EF0000F5EF0000A0050020F9EF000089
:1008000009F0000010F00000B6FE00001003002008
:10081000F802002007B5002300931A461946034842
:1008200008F084F903B05DF804FB00BF90020020DB
:10083000F0B52DED028B064699B008EE101A3C4833
:100840003C4908F0B3F90A227179394808F030FAC6
:100850003949374808F0AAF918EE100A0AF066FB81
:1008600002230246009304460B4631480D4608F029
:10087000E5FA2F4808F0AAF93168304A304807F005
:10088000A0F931682F4A07462D4807F09AF9064625
:1008900010B34169402208A80CF015F92F2108A8CF
:1008A0000CF0A8F828B973690322402108A803F0C6
:1008B0007BFD18EE100A04A903F02AFD224807F078
:1008C00061FC48B1214B93F900302BB9012304AAF4
:1008D00008A91D4807F06EFE17B3B5EEC08AF1EE09
:1008E00010FA4FF000021A4B204629461CDB0AF092
:1008F000BFF90AF023FE7969049008A800F0FCFC17
:1009000008A800F0ADFC40B100210122CDE90111A1
:10091000009204AB08A800F025FF08A800F0B6FB81
:1009200019B0BDEC028BF0BD0AF0A0F9E1E700BF01
:10093000A0050020F5EF00000EF00000F0EF000031
:100940004C050020EBEF000010030020F80200200F
:100950000000E03F2DE9F041064694B00F464848BC
:10096000484908F023F90A227179454808F0A0F9AE
:100970004549434808F01AF90A223946404808F028
:100980007EF93F4808F022F93168404A404807F0B4
:1009900018F931683F4A80463D4807F012F931683E
:1009A0003D4A05463A4807F00CF931683B4A04468F
:1009B000374807F006F90646F8B14169402204A815
:1009C0000CF081F8364807F0DDFBB0B1354B93F9F8
:1009D000003093B92F2104A80CF00CF828B97369E2
:1009E0000322402104A803F0DFFC4FB315BB2E4ABD
:1009F000012304A92A4807F0DDFDB8F1000F16D045
:100A0000D8F8141004A800F077FC04A800F028FC23
:100A100050B12FB3D5B9CDE90155012100912B4635
:100A20002A4604A800F09EFE04A800F02FFB14B094
:100A3000BDE8F0816A691378002BDED00123D8E786
:100A400014B90123194AD4E76269F4E769690B789C
:100A5000002BE9D00023012204A800F08BFAE3E781
:100A60003CB901230093CDE90144234622460221EB
:100A7000D7E761690B78002BD6D03B46EBE700BF88
:100A8000A0050020F5EF00000EF00000F0EF0000E0
:100A90004C050020DCEF0000E1EF0000EBEF000070
:100AA00010030020F802002095F2000090F20000F0
:100AB00038B5037903F00203002B04460CBF022172
:100AC0000021407914BF0125002508F00DFF607951
:100AD00008F044FFA368A0EB050CDCF10001B3F9BA
:100AE000022041EB0C0191421AD093F9012012B17E
:100AF000013A5A7038BD2279D2070ED5A842F9D1F1
:100B000093F90010B1FA81F14909012219705A8054
:100B10002046BDE83840FFF71DBF19705980F7E740
:100B20000322E6E72DE9F347064601685F4A60487D
:100B300007F047F8337913F0020F0CBF02210021B0
:100B40000546707908F0D0FE707908F0D7FD07B23D
:100B5000002D67D02B7C052B64D12946544807F023
:100B600020F8032853D900222946514807F021F8DC
:100B7000012244694E48294607F01BF80222D0F8AA
:100B800014A04B48294607F014F8436948484FF031
:100B90000A080322294608FB03F907F00AF843690B
:100BA00008FB03F82146CDF800804B4652463846F4
:100BB00008F01BFC044629463D4806F0F2FF0528D4
:100BC0002DD1042229463A4806F0F3FFB0F914A0CB
:100BD00037484445A8BF44464C452946B8BF4C4613
:100BE00006F0DFFF022826D100222946304806F011
:100BF000E0FF4369BB4249DC012229462C4806F04C
:100C0000D8FF4369BB424EDB02B0BDE8F08707EB7B
:100C1000870464004FF000094FF42058CBE74FF0F1
:100C2000010AD5E707EB870464004FF000094FF491
:100C300020584FF0010AB368B3F902107A1A002A5B
:100C4000B8BF5242524505DC93F90120052A03DC66
:100C5000013200E000225A7093F90130042B03DDC9
:100C60004C4501D04445CFD1B942CDD020460AF001
:100C70004BF9104B00220AF0DBFA0AF0A7FC014600
:100C80003046FFF7D5FDB3685F80BDE70024B36849
:100C9000B3F90230A342B7D021463046FFF75AFEDF
:100CA000B3685C80B0E70124F1E700BFD8EF000033
:100CB0004C0500200000244008B50246FFF724FC44
:100CC000E0B1012903D0022911D0002018E01379E6
:100CD000402B08D005D8032BF7D81046FFF7E8FEC5
:100CE000F3E7422BF1D11046FFF71CFFEDE7137934
:100CF000042BEAD11046FFF7A7FCE6E74FF0FF30E0
:100D000008BD000038B505782D2D044600F0998007
:100D1000A5F13003092B40F2948060490BF077FE77
:100D2000002800F0A4805E4920460BF070FE0028E9
:100D300000F09F805B4920460BF069FE002800F020
:100D40008280594920460BF062FE00287DD0574929
:100D500020460BF05CFE002879D0554920460BF068
:100D600056FE002875D0534920460BF050FE00284F
:100D700071D0514920460BF04AFE00286DD04F49F2
:100D800020460BF044FE002869D04D4920460BF068
:100D90003EFE002865D04B4920460BF038FE002867
:100DA00061D0494920460BF032FE00285DD047490A
:100DB00020460BF02CFE002859D0454920460BF068
:100DC00026FE002855D0434920460BF020FE00287F
:100DD0004DD0414920460BF01AFE002849D03F492A
:100DE00020460BF014FE002845D03D4920460BF06C
:100DF0000EFE002841D03B4920460BF008FE00289B
:100E00003DD0394920460BF002FED0B33749204689
:100E10000BF0FDFDB8B37B2D37D0232D38D0032246
:100E2000334920460BF03DFEA8B30322314920464A
:100E30000BF037FE002814BF4FF0FF306FF00200B8
:100E400038BD0020FCE70320FAE70420F8E705207E
:100E5000F6E70620F4E70720F2E70A20F0E70B2088
:100E6000EEE70C20ECE70D20EAE70E20E8E7012092
:100E7000E6E70220E4E70820E2E70920E0E71020A7
:100E8000DEE71120DCE71220DAE76FF00100D7E798
:100E90006FF00200D4E76FF00300D1E736F00000F6
:100EA00054F0000082F00000A0F000006EF000009E
:100EB00060F000008CF0000073F0000069F00000AA
:100EC00064F0000024F000003DF0000087F0000016
:100ED0009AF00000A7F000001BF000002DF00000C9
:100EE00012F0000078F000004DF0000049F0000022
:100EF00045F0000058F0000010B5044608B3037830
:100F000003B316490BF083FDF0B1154920460BF0F1
:100F10007EFDD8B1134920460BF079FDC0B11249CE
:100F200020460BF074FDA8B1104920460BF06FFD70
:100F300090B10F4920460BF06AFD002814BF002035
:100F4000052010BD1846FCE70220FAE70120F8E76B
:100F50000620F6E70320F4E70420F2E75CF0000047
:100F600039F000007DF0000045F0000058F000006E
:100F700041F000002DE9F0478AB080460591914686
:100F80001C4600296AD013B31D781DB32F211846C3
:100F90000BF0AEFD90B1002300F8013BFFF7ACFF72
:100FA0000F2506460027DDF814A01AF8070098B1AF
:100FB0000BF03EFF0AF807000137F4E72046FFF781
:100FC0009BFF0F250646002818BF0024EAE71D46B0
:100FD0001E46E7E72E46E5E75046FFF793FE204919
:100FE0000746204807F0E2FD0A2239461D4807F06F
:100FF00046FE1C4807F0EAFD3B1D042B23D8DFE822
:1010000003F003221F1F0400032600270DF11C0A12
:1010100005993AB249B1032F06D005A803F050F95B
:101020004AF827000137F3E73A46CDE90164D8F8DA
:101030000030CDF800901C68294653464046A04732
:101040000AB0BDE8F087CDE90164D8F80030CDF8EA
:1010500000901C6800231A4639B2EFE70846EFE714
:10106000E0F00000A005002010B50446406960B122
:1010700003689B69984718B1606903685B69984782
:1010800060690368DB689847012010BD054B10B507
:1010900004460360406910B103685B6898472046C6
:1010A00010BD00BF38F2000008B5416804480322B3
:1010B00006F07FFD08B1007D08BDFF20FCE700BF02
:1010C0004C05002010B503220C4641680B4806F081
:1010D00070FD90B143690A4903F47063234343618F
:1010E000084807F063FD21460A22064807F0E0FDA4
:1010F0000448BDE8104007F069BD10BD4C05002054
:10110000CEF10000A005002010B503220C46416876
:10111000044806F04EFD18B1406904F470642040A4
:1011200010BD00BF4C05002010B503220C464168DD
:101130000B4806F03EFD90B143690A4904F4706221
:1011400013434361084807F031FD21460A2206484F
:1011500007F095FD0448BDE8104007F037BD10BD0D
:101160004C050020E4F10000A005002010B503228A
:101170000C4641680C4806F01CFD98B1E34363F44B
:1011800070624369094913404361094807F00EFD45
:1011900021460A22064807F072FD0548BDE81040C6
:1011A00007F014BD10BD00BF4C05002025F2000063
:1011B000A005002038B50C468168054609B9002015
:1011C00038BD0B7C022B03D1002CF8D14869F7E71E
:1011D000052BF4D1054806F0E4FC8442EFDAE2B2D4
:1011E000A968024806F0E5FC4069E9E74C050020E3
:1011F000C16808B509B9002008BD0B7C022B01D1DC
:101200004869F9E7052BF6D10022034806F0D1FC26
:101210000028F0D04069EFE74C05002038B5C368DE
:1012200005460C46A3B11B7C022B11D109490A4883
:1012300007F0BCFC0949084807F0B8FC0A2221461F
:10124000054807F0FAFC044807F0C0FCEB685C6155
:1012500038BD00BFD6F10000A0050020DEF100007F
:10126000406818B1007C431F584258417047000045
:101270002DE9F0410446FFF7F3FF48B361681548D4
:10128000DFF85480134F06F08CFC0546032D66688A
:101290000BDC38F91510384606F0C2FC3146024620
:1012A000384606F09BFC0135F0E70022314609483C
:1012B00006F07FFC4369237401226168054806F04B
:1012C00078FC0222A0606168024806F072FCE060CF
:1012D000BDE8F0814C05002092F0000010B5054BF0
:1012E000C0E90031002304464361FFF7C1FF2046F7
:1012F00010BD00BF38F200000B4B10B50360002397
:10130000044643610A4659B1084B196841B108487F
:1013100006F057FC60602046FFF7AAFF204610BD8C
:1013200000236360F7E700BF38F2000000030020ED
:101330004C05002030B5436887B005461968414820
:1013400007F03DFC2846FFF78BFF50B93E493D486A
:1013500007F02CFC3B4807F039FC4FF0FF3007B09A
:1013600030BD2846FFF7A0FE2B7C072B12D00130A2
:101370000D280FD8012404FA00F010F0490F46D1CF
:1013800043F68403184205D030492E4807F00EFC7E
:101390000120E4E7686918B10368DB6A9847DEE773
:1013A0002846FFF725FF2A7C092A044646D8012350
:1013B000934040F21932134230D113F006022CD17F
:1013C0001B063BD5AB681B7C052B39D120491D483A
:1013D00007F0ECFBAB68DC68CCB161696846FFF7ED
:1013E0008BFF6846FFF73CFF60B16846FFF7A2FF3E
:1013F000002807DD1549134807F0D8FB6846FFF7BA
:1014000045FEC5E768466468FFF740FEE4E711491A
:101410000C4807F0CBFB0020A1E7C4B20E490948F5
:1014200007F0C4FB0A222146064807F028FC0548BD
:1014300007F0CCFB201C18BF012090E70749E7E725
:101440001446EBE7A0050020EDF10000F6F10000E6
:101450000AF20000FFF100001AF2000010F2000092
:101460002DE9F04395B00C460546FFF71DFE14F438
:10147000006607460ED004F440712846FFF754FE7C
:10148000A749A84807F092FB4FF0FF36304615B049
:10149000BDE8F0834FF440712846FFF735FE044362
:1014A000A005CDE90466CDE90666CDE9026620D542
:1014B0002846FFF79DFE2B7C08901BB1022B09D913
:1014C000072B29D003461021974A0DEB01000BF0A2
:1014D000C1F90EE0BDF82230C2B2C0F3072001927C
:1014E0000090C3F30E031021904A0DEB01000BF0A6
:1014F000B1F9E10520D50F2F66D80123BB4041F695
:101500004242134214D148F20102134260D113F057
:10151000240F59D086490CE00028C3B2D3DABDF8B5
:1015200022200193C0F307200090C2F30E03DAE7F4
:10153000804902A80BF075FA00230322302108A885
:1015400002F032FF6B683022196808A80BF095FA98
:10155000794806F017FE002800F08880774B93F951
:1015600000209846002A40F0818014F4007932D19E
:10157000E20518D5012302AA08A96F4807F01AF856
:101580006F49684807F012FB08A9664807F017FB87
:101590006C49644807F00AFB02A9624807F00FFB98
:1015A000604807F013FBB9F1000F31D1E30540F1BA
:1015B000AD80013F0B2F6ED8DFE807F0AC6D6D6D8D
:1015C0006DAC6D6D6DAFAA695F49564807F0EEFAD4
:1015D00024F48074B0E7022FCAD0052FC8D00123AD
:1015E00004AA08A9544806F0E5FF55494D4807F0FC
:1015F000DDFA08A94B4807F0E2FA5249494807F0DA
:10160000D5FA04A9474807F0DAFA464807F0DEFAA7
:1016100000230322302108A802F0C6FE6B683022A6
:10162000196808A80BF029FA484908A80BF0D3F963
:10163000474908A80BF0CFF941493A4807F0B6FAF4
:1016400008A9384807F0BBFA3E49364807F0AEFA19
:1016500004A9344807F0B3FA324807F0B7FA36481D
:1016600006F090FD10B198F9003023B121B2284660
:10167000FFF75AFD0AE708A9012304AA2E4806F03D
:1016800099FF4FF400712846FFF770FD8EE731494E
:1016900002A80BF0C6F900230322302108A802F0AB
:1016A00083FE6B683022196808A80BF0E6F9274919
:1016B00008A80BF090F9284908A80BF08CF92049EC
:1016C000184807F073FA08A9164807F078FA1D4978
:1016D000144807F06BFA02A9124807F070FA114893
:1016E00007F074FA144806F04DFD0028BED098F9B2
:1016F0000030002BBAD108A9012302AA0E4806F037
:1017000059FF4FF480712846FFF730FD0126BDE6F2
:101710001249BDE72B7C052BBDD11149B8E700BFAD
:10172000AFF00000A0050020C6F00000C0F00000EF
:1017300054F0000036F0000010030020F8020020F2
:10174000D7F00000DDF00000C9F000000BF600004B
:101750005CF0000064F0000039F0000069F0000067
:1017600073F000002DE9F04F91B004460D46A548F6
:10177000A5499DF868609946174607F017FA02F0E8
:10178000C0FD0A2201469F4807F085FA9F499D48FF
:1017900007F00CFA63689B48196807F010FA9C4937
:1017A000984807F003FA1C99964807F008FA9949F7
:1017B000944807F0FBF90A221B99924807F05FFA58
:1017C0009549904807F0F2F90A2229468D4807F01A
:1017D00056FA92498B4807F0E9F96368002B3CD030
:1017E0000023CDE907330993B9F1000F23D09846C0
:1017F000DFF810A28A4B0FFA88F297421BDDB8F18E
:10180000030F18D00DF11C0B59F828204BF8282095
:1018100019465046059307F0C9F95BF828100A22CB
:10182000504607F02CFA7F49504607F0BFF908F1FF
:101830000108059BDFE77C49724807F0B7F971485A
:1018400007F0C4F9237C072B0AD14EB977496D48BC
:1018500007F0ACF96B4807F0B9F94FF0FF3676E0C6
:1018600000212046FFF7A6FC80462046FFF762FDD8
:10187000042D82461AD0072D33D0032D1AD1237C94
:10188000072B17D02046FFF70FFC052805464BD144
:1018900067495C4807F08AF929460A22594807F047
:1018A000EEF9584807F092F9012503E00028D4BF6B
:1018B000012502256069002800F08E80052D68D082
:1018C00035DC022D75D01C9A036802921B9ACDE973
:1018D000006229469E6A3A464B46B047E9B2064640
:1018E0004EE0237C072BE5D02046FFF7DDFB0628E2
:1018F00005460DD14F49434807F058F929460A22B9
:10190000404807F0BCF93F4807F060F90225D1E7ED
:1019100049493C4807F04AF90A222946394807F064
:10192000AEF9384807F052F96FF002060FE0062DC5
:1019300011D00F2DC7D11C9A036802921B9ACDE9D2
:10194000006229469C6A3A464B46A0470646304606
:1019500011B0BDE8F08FBAF1000F15D13749294811
:1019600007F024F960691C9A036802921B9ACDE97A
:10197000006201219E6A3A464B46B0472946064618
:101980002046FFF79FFBE2E72D491E4807F00EF9BE
:10199000CAE7BAF1000F0ADD1C9A036802921B9A8B
:1019A000CDE9006202219E6A3A464B46E5E72549A9
:1019B000EBE72046FFF778FB05280BD060691C9AFF
:1019C000036802921B9ACDE9006229469E6A3A4654
:1019D0004B46D2E71C49D8E70F2D00F2D780DFE84D
:1019E00015F047002B012A02D500D5003E02200148
:1019F000D500D500D500570157015701D500D500B6
:101A0000350000BFA0050020E9F00000EEF0000066
:101A1000F5F00000FBF0000002F1000008F100000A
:101A20000FF10000DEF0000011F1000013F10000E2
:101A30001CF100002BF100003CF1000054F100000B
:101A400061F1000071F1000083F10000BAF1000FB4
:101A5000D4BF4FF000094FF00109237C092B00F29D
:101A60009280DFE803F06D080E6D6D86900E866D36
:101A70004FF00109F1E7089B1BB9032F04BF7F2337
:101A800023742046FFF7B4FB022F06902AD0032FC1
:101A90003BD0012F0FD1079B8DF8183000280ADAB0
:101AA000BDF81A20C0F30720C2F30E02DBB2079282
:101AB00008900993032706992046FFF7AFFBB9F179
:101AC000000F4CD0BAF1000F33DD9DF818301BB970
:101AD00002212046FFF7F6FA4FF430612046FFF767
:101AE000BFFC53E0BDF81A30079A62F30E03ADF85D
:101AF0001A30C3F30723089A8DF81920C0B243F0B7
:101B0000800309908DF81B30D4E7BDF81A30079A8E
:101B100062F30E03ADF81A30089A8DF81920C3F35A
:101B20000723099A8DF8182043F080038DF81B30A5
:101B3000C1E7D1D19DF81830002BCDD00121C8E7E5
:101B400007992046FFF76AFBB9F1000F07D0BAF1F9
:101B5000000F01DD079BBAE7BED1079BECE74FF40E
:101B600020612046FFF77CFC237C072B0ED001264A
:101B7000EDE607992046FFF751FB26B14FF42061AF
:101B80002046FFF76DFCB9F1000FEDD000234FF0B8
:101B9000FF0919466422CDF80090089807F025FC4B
:101BA00000231946CDF800906422099807F01DFC27
:101BB000237C062B00F09F81072B00F07F81032BF5
:101BC0007FF4C5AEB8F1000F3FF4C1AEB8BFC8F1A5
:101BD00000084FF001014046B4BF0124002407F083
:101BE00083FEFF230093002C00F0BA8100231A46E5
:101BF0006421079807F0F9FB01460446404607F0C8
:101C000021FEA549A54806F0D1FF0A224146A34876
:101C100007F035F8A249A14806F0C8FF0A2221467C
:101C20008FE1BAF1000F2ED09E499C4806F0BEFF0E
:101C3000237C072B7FF478AE237C012B28D1204610
:101C4000FFF732FA012823D116B39749934806F0DB
:101C5000ADFF7F23237400226423CDE90823079975
:101C6000BDF81A20ADF8183061F30E02ADF81A2055
:101C700006992046FFF7D2FAE9B22046FFF722FA8A
:101C80004FF440712AE78949844806F08FFFD3E773
:101C9000E9B22046FFF716FABAF1000F06DD2EB1C1
:101CA0004FF480712046FFF7DBFB60E72046FFF72B
:101CB0009FFA237C0690042B0CD8DFE803F003186E
:101CC000180B0300182801DC3223069306992046DE
:101CD000FFF7A4FA0699002975D0237C092B6FD849
:101CE000DFE803F05E25255E5E696E0E5E5E00280D
:101CF000ECD0C0B218289CBF32238DF81830E5E72D
:101D0000002E3FF443AF2046FFF714FB20B94FF4F9
:101D100080712046FFF7A4FB237C012B7FF436AFB4
:101D2000089B002B7FF432AF7F2323742EE7BDF88E
:101D30001A30C3F30E0307939DF8193008939DF8EA
:101D40001830099336BB4FF0030B594BDFF84CA109
:101D50004FF000090FFA89F29345DDDD1946504630
:101D6000059306F023FF0A224946504606F087FFF6
:101D70004B49504606F01AFF07A90A2251F82910CC
:101D8000504606F07CFF504606F020FF09F101099D
:101D9000059BDFE74FF440712046FFF761FBD2E778
:101DA000079116B94FF0010BCFE74FF44071204671
:101DB000FFF756FBF6E70791002E3FF4E7AEA6E7E4
:101DC000002EA9D0A3E70A22344806F036FF39498D
:101DD000324806F0EBFE237C013B072B29D8DFE8D5
:101DE00003F00A0A2828041E28041421204607911B
:101DF000FFF714FAD5E7BDF81A106423002263F345
:101E00000E01ADF81A108DF819208DF818300699CA
:101E100009932046CDE90732FFF700FA92E76421E3
:101E200020460791FFF7FAF9002EBBD04FF48071DE
:101E3000BDE76421DAE72046FFF736F905283FF4CD
:101E4000A5AE002302212046CDE907330993FFF711
:101E500039F9002E3FF49AAE4FF480713EE6BAF1A4
:101E6000000F7FF793AE00232046CDE90733099397
:101E7000FFF71AF906280CBF022105212046FFF7BB
:101E800021F94FF480712046FFF7EAFA0A49034826
:101E900006F08CFE7AE600BFC9F10000A005002024
:101EA0000EF0000061F1000093F1000054F1000019
:101EB000BEF10000A0F100008AF10000A3681A7CC6
:101EC000052A7FF444ADDC68002C3FF440AD616925
:101ED0000AA8FFF711FA1C9B02931B9B3A46CDE917
:101EE0000063294607AB0AA8FFF73CFC0AA8646810
:101EF000FFF7CCF8E8E7B8F1000F3FF428ADBABF20
:101F0000C8F10008012400240121404607F0ECFC40
:101F100004B3012D1CD0063D18BF012529464046BB
:101F200007F00AFD1049114806F040FE0A2241461A
:101F30000E4806F0A4FE0E490C4806F037FE0A22B1
:101F400029460A4806F09BFE084806F03FFEFEE4DC
:101F50000025E3E7012DE1D0AB1F5D425D41DDE7E8
:101F600023466422214644E6C9F10000A005002072
:101F70000EF0000007B5002300931A4619460348E7
:101F800006F0D4FD03B05DF804FB00BFC0020020E2
:101F900001F0FABE01F0D2BE07B5002300931A4645
:101FA0001946034806F0C2FD03B05DF804FB00BF0C
:101FB000C80200207047000038B5084D01244FF4D6
:101FC0007A7007F0FFFA214601340A222846E4B26B
:101FD00006F06EFE142CF2D138BD00BFA005002023
:101FE00008B50449044806F0E1FDBDE8084002F0E8
:101FF00067BA00BF3DF50000A005002010B586B00F
:102000000F4C10494FF0FF3203920F4A0092002309
:1020100048222046CDE90423CDE9013306F0C6FD70
:102020000A4B0B4819686A4605F094FD684605F0AE
:10203000BDF90849204606F0B9FD06B010BD00BF45
:10204000A0050020A0F4000054FF0000E8030020D9
:102050004C050020BAF4000038B5084D0024214694
:1020600000222846013405F014F9B4F5007FF6D1BA
:1020700003490448BDE8384006F098BDD00200206E
:10208000CDF70000A005002010B5174C236853B30E
:102090001649174806F08AFD02F033F90A22014674
:1020A000134806F0F8FD2168124805F08FF9124A2E
:1020B00012490F4800231360114A23601360114A2C
:1020C0001360114A1360114A136006F06FFD02F0AD
:1020D00018F90A220146064806F0DDFD0448BDE86D
:1020E000104006F073BD10BDE803002045FA000063
:1020F000A00500204C050020FC02002020F200007A
:1021000000030020EC0300200C030020DC0300206F
:102110002DE9F04116491748174E184F154D06F096
:1021200045FD002406F1010816F8013F0F2B03D8E6
:102130003946284606F043FD052C4FF010020DD01D
:102140003178284606F079FD0D49284606F02EFD27
:102150000134E4B2062CE7D1BDE8F08198F805100F
:10216000284606F06AFD284606F030FDF0E700BF7D
:10217000CAF40000A00500200403002038FF00007E
:10218000F9F600007FB5184C0394631E0293A31E5A
:1021900001930D46E31E0093621F231F13496868D5
:1021A0000AF08CFB05280ADC1149124806F0FEFCF7
:1021B0006968104804B0BDE8704006F000BDFFF744
:1021C000A7FF0D4E0025053C625D294630460135CE
:1021D00005F05FF8062DF7D10849064804B0BDE8C0
:1021E000704006F0E3BC00BF0A0300204FF500007A
:1021F00063F50000A0050020D002002075F5000066
:102200002DE9F0410024C8B03C22214609A80894D9
:1022100009F099FC7C22214629A8289409F093FC16
:1022200023460122402108A802F0BEF87849794FE0
:1022300008A80AF0D0FB8022774928A80AF043FCBE
:10224000012328AA08A9754806F0B4F923460122FB
:10225000402108A802F0A8F8714908A80AF0BBFBC1
:102260008022704928A80AF02EFC6F4928A80AF09D
:10227000B2FB012328AA08A9684806F09BF9234667
:102280000122402108A802F08FF8684908A80AF046
:10229000A2FB8022664928A80AF015FC012328AA7F
:1022A00008A95E4806F086F923460122402108A8C5
:1022B00002F07AF85F4908A80AF08DFB80225E4997
:1022C00028A80AF000FC012328AA08A9534806F010
:1022D00071F93D68002D00F09880584BDFF88C8133
:1022E0001E88ADF8006021461E220DF1020009F0A3
:1022F0002AFC21463E220DF16200ADF8606009F033
:1023000022FC4F4EEC684F4D3A68002A73D0002CE7
:1023100071D0237C052BF8D12146284605F041FCDD
:102320000028F1D000222146284605F042FC4369EE
:10233000092B0ED8DFE803F0574F4F575705444499
:1023400057572022404968460AF0BDFB00238DF80C
:10235000603000230122402108A802F025F8402225
:10236000216808A80AF089FB384908A80AF033FB5D
:10237000374908A80AF02FFB01236A4608A9274815
:1023800006F018F99DF86030C3B100230122402106
:1023900008A802F009F84022216808A80AF06DFB9D
:1023A0002A4908A80AF017FB2A4908A80AF013FBD3
:1023B000012318AA08A9194806F0FCF86468A3E7E5
:1023C0002022254968460AF07EFB2449402218A8AD
:1023D0000AF079FBBDE72022214968460AF073FB29
:1023E00040222049F3E72022314668460AF06BFB81
:1023F00040224146EBE740210023012208A801F0DA
:10240000D3FF194908A80AF0E6FA48B0BDE8F08100
:1024100022FB0000000300201CFB00001003002032
:10242000FCFA000052FB00003FFB000029FB00000B
:102430009BFA00000EFB000095FA000040F200003D
:10244000EFFA00004C05002008FB00000BF600002E
:1024500082FA000030FB0000F7FA0000BDFA00002D
:1024600002FB0000EBFA000015FB0000ABFA0000D5
:1024700010B5114C1149204606F098FB1049204632
:1024800006F09DFB4FF4FA7007F09CF8012115202F
:1024900007F02AFA0021152007F04EFA4FF4FA70DF
:1024A00007F090F81520012107F046FA4FF4FA7072
:1024B000BDE8104007F086B8A00500205FFA0000D4
:1024C0007FFA000013B50E4C0E490F4806F06EFB64
:1024D0002146684602F05BFF684601F03FFF214657
:1024E000684602F06CFF684601F038FF21466846F6
:1024F00002F059FF684601F031FF02B010BD00BF85
:10250000DC040020D5F60000A005002070B51A4CB0
:102510001A4D88B02F231522002102A8019309F03B
:1025200012FB1749204606F041FB0DF1050206217A
:10253000144801F07DFE002613498DF8116001A8B2
:102540000AF049FA01A9204606F039FB01A92846FC
:1025500006F076F80D498DF8116001A80AF03BFAF3
:1025600001A9204606F02BFB094A01A9284606F0DE
:1025700010F8012008B070BDA00500201003002055
:102580007EF500000503002093F500009BF5000098
:102590008FFE0000FFF7BABF18B10349034806F0E9
:1025A00005BB0349FAE700BF5DFA0000A005002063
:1025B0003B04010010B5224C2249204606F0F6FAF1
:1025C0002149204606F0F2FA204B1868003018BF67
:1025D0000120FFF7E1FF1E49204606F0E7FA1D4BF8
:1025E0001868003018BF0120FFF7D6FF1A492046AF
:1025F00006F0DCFA194B1868003018BF0120FFF70D
:10260000CBFF1749204606F0D1FA164B1868003068
:1026100018BF0120FFF7C0FF204606F0D7FA124985
:10262000204606F0C3FA01F06CFE0A22014620465D
:1026300006F031FB2046BDE8104006F0C7BA00BFE7
:10264000A005002068F6000075F6000000030020D9
:102650007DF60000FC02002086F600000C0300203E
:102660008DF60000DC030020E9F000002DE9F843BE
:10267000074608460E460AF0F8F904B21F2CDFF8A8
:102680003080A8BF1F243546A7EB0609AB1B9C4230
:1026900007DD09EB0501404615F8012B04F0F9FDB3
:1026A000F4E7E11900220248BDE8F84304F0F1BD67
:1026B000D002002007B500238DF8043050B14968DE
:1026C0003620FFF7D3FF0449044806F06FFA03B041
:1026D0005DF804FB01A9F3E70DF30000A00500205D
:1026E0002DE9F04780460F4601461148164604F092
:1026F000CEFD0138C0B2FD2818D8DFF834A0002480
:10270000013E25B208EB0401B54209B207EB050909
:1027100006DA504604F0BBFD013478550028F0D1AC
:10272000002389F800300120BDE8F0870020FBE796
:10273000D00200202DE9F043944CA7B02168002579
:102740008DF81750CDE90655CDE90855B1B190483F
:1027500005F027FA90B12A4621688D488D4D05F085
:1027600028FA8D4943698D482B6006F01FFA2968C5
:102770008A4806F024FA894806F028FA884805F0C5
:1027800001FD002840F0DB802168002900F0D7809F
:102790007F4805F006FA06B2012E40F3D0800122F0
:1027A00021687B4805F005FA022ED0F8149000F05D
:1027B000C98002222168764805F0FBF9032ED0F883
:1027C000148000F0C18003222168714805F0F1F9FE
:1027D0004569102206A93620FFF782FF002840F045
:1027E000B680042E40F3B38021686948042205F0C6
:1027F000E0F96C494469694806F0D8F91FFA88F293
:102800004946674805F04DFF0AAE6749644805F040
:102810004DFF0EAF1022654930460AF054F90023EF
:1028200001222021384601F0BFFD614938460AF0F7
:10283000D2F86049594806F0B9F94946574806F0B8
:10284000BEF95D49554806F0B1F90A2241465348A0
:1028500006F015FA5949514806F0A8F929464F489B
:1028600006F0ADF956494D4806F0A0F92B780BB9A2
:102870001C461D4603964FF002080126CDE901864D
:10288000DFF8109100972A462346D9F800104448F3
:102890004C4D4D4F05F082FD00285AD04B4B4C4912
:1028A0003E4800241C6006F081F9D9F800103B482E
:1028B00006F085F9394806F089F9464B03221E7067
:1028C0004021234616A801F06FFD434916A80AF0DF
:1028D00082F816A9324805F0B3FE2346424640214D
:1028E00016A801F061FD3D4916A80AF074F816A972
:1028F0002A4806F07BF916A9294805F0A1FE2346CF
:102900003246402116A801F04FFD344916A80AF0BE
:1029100062F816A9214806F069F916A9204805F0C1
:102920008FFEFFF76DFC04232B7006F031FE00F5DF
:102930009C50083038602A49184806F037F927B00B
:10294000BDE8F08340F25B780DF1170541E706AC76
:1029500054E72449114806F029F9114805F0A9FE69
:102960000A2201460D4806F08AF91F490B4806F075
:102970001DF90A4806F02AF906F00AFE00F59C50F7
:1029800008300C2338602B70D9E700BF0C030020FF
:102990004C050020E002002015F90000A0050020F1
:1029A0001003002022F90000C5390000DEFA000003
:1029B00022FB000042F90000F9F6000062F9000075
:1029C00069F9000004030020D0030020C8030020A0
:1029D0006EF90000DC0200207CF9000080F90000A4
:1029E00082F900009FF90000ABF90000F8B5074E2E
:1029F00007460D1D0024E11915F8012B09B23046D8
:102A0000013404F046FC042CF5D1F8BDD0020020BE
:102A100030B587B00023044600931A460D4602A83D
:102A2000194606F083F804A806F078F8042C12DDA5
:102A300004A9286901F06DFC68B104A91220FFF710
:102A4000D5FF04A9E86801F064FC50B104A90E2088
:102A5000FFF7CCFF0BE002A91220FFF7C7FF032C02
:102A6000EFDC02A90E20FFF7C1FF022C17DD04A93D
:102A7000A86801F04EFC90B104A90A20FFF7B6FF48
:102A800004A9686801F045FC78B104A90620FFF7A5
:102A9000ADFF0D490D4806F089F807B030BD02A919
:102AA0000A20FFF7A3FF012CEADC02A90620FFF7AA
:102AB0009DFF012CEDD102A90620FFF797FF0449E5
:102AC000024806F073F8E4E706F30000A0050020D2
:102AD000F6F200002DE9F041104F80460C460E1D25
:102AE000002508EB050109B2384604F0D0FB01359A
:102AF000042D06F8010BF4D1207958B1FF280BD131
:102B00006379FF2B08D1A379FF2B05D1E079FF383A
:102B100018BF0120BDE8F0810120FBE7D0020020B2
:102B2000F0B593B002A805F0F9FF04A805F0F6FF90
:102B300006A805F0F3FF08A805F0F0FF5C495D4822
:102B40005D4E06F033F85B4806F040F802A9062017
:102B5000FFF7C0FF00287CD058495648584C10ADAC
:102B600006F02DF8039B10942846119301F0F6FB14
:102B700004A90A20FFF7AEFF002861D051494D4853
:102B800006F01DF8059B11932846109401F0E6FB12
:102B900006A90E20FFF79EFF0EAF002843D04A493A
:102BA000444806F00CF8079B10942846119301F056
:102BB000D5FB08A91220FFF78DFF18B343493D4804
:102BC00005F0FDFF099B11932846109401F0C6FB08
:102BD000039B3F493F480A94CDE90B34059BCDE95F
:102BE0000D34079BCDE90F34099B1193CDE9007596
:102BF0000CAB0AAA02F01AFB2E4805F0E7FF0123EE
:102C0000337046E0039B0095CDE90D34059B3049B8
:102C100030480C94CDE90F34079B11930CAA3B4626
:102C200002F020FBE8E7039B29492A480E94CDE9EE
:102C30000F34059B11933A462B4602F03DFBDBE730
:102C4000039B2349234810942A46119302F04EFB1C
:102C5000D2E72149174805F0B2FF4FF47A6342F6F4
:102C6000E0621B491B4802F07FFAA0B91B491148DA
:102C700005F09CFF1A490F4805F098FFF6233370C2
:102C800006F086FC174B00F56A4060301860FFF7CD
:102C9000EFFB13B0F0BD1449064805F087FF10A8FC
:102CA0000C4902F074FB10A801F058FBA7E700BF25
:102CB000FBF60000A00500200403002008F7000038
:102CC0002C0001001EF7000024F7000029F7000087
:102CD00005030020DC04002030F700004CF7000062
:102CE0008EF70000D0030020BDF7000010B52C4C7B
:102CF0002C49204605F05AFF2B49204605F056FF87
:102D00002A49204605F052FF2949204605F04EFF8A
:102D1000204605F05BFF2749204605F047FF26497E
:102D2000204605F043FF2549204605F03FFF244992
:102D3000204605F03BFF2349204605F037FF224996
:102D4000204605F033FF2149204605F02FFF20499A
:102D5000204605F02BFF1F49204605F027FF1E499E
:102D6000204605F023FF1D49204605F01FFF1C49A2
:102D7000204605F01BFF1B49204605F017FF1A49A6
:102D8000204605F013FF1949204605F018FF20469C
:102D9000174905F00BFF2046BDE8104005F016BFAF
:102DA000A0050020DDF70000FFF7000012F800008A
:102DB00020F8000028F8000035F8000045F8000071
:102DC00051F8000068F800007CF8000091F800005D
:102DD000A0F80000AFF80000B7F80000C2F800004B
:102DE000CCF80000D4F80000E0F800007FFA000002
:102DF000F6F8000008B5FFF779FFFFF763FB03491A
:102E00000348BDE8084005F0D1BE00BF1FF3000035
:102E1000A005002030B595B001F073FA054606F024
:102E2000B7FB0446204805F0ADF900283AD000234E
:102E30000122402104A801F0B7FA1C4904A809F0B6
:102E4000CAFD1B4904A809F0C6FD1A4904A809F0E7
:102E5000C2FD2946684601F017FB01236A4604A912
:102E6000114805F0A7FB00230122402104A801F02E
:102E70009BFA0E4904A809F0AEFD0D4904A809F01B
:102E8000AAFD0D4904A809F0A6FD68464FF47A7121
:102E9000B4FBF1F101F0F8FA01236A4604A90248F3
:102EA00005F088FB15B030BD1003002029FB0000A1
:102EB0000BF600008CFA000038FB00002DE9F04111
:102EC000144FDFF85C8000252E463C4629464046DC
:102ED00004F0DDF9E8550138C0B2FD2805F101051F
:102EE00098BF0126062DF1D17EB90B490B4805F09C
:102EF0005DFEDE232370AD236370BE23A370EF233A
:102F0000E370FE232371FF236371BDE8F041FFF7F7
:102F1000FFB800BF0503002007F50000A005002052
:102F2000D002002008B54FF4E13004F0B1FF194998
:102F3000194805F03BFE1949194804F043FF1949A7
:102F4000194804F03FFF1949194804F03BFF19499B
:102F5000194804F037FF1949194804F033FF19499B
:102F6000194804F02FFF1949194804F02BFF19499B
:102F7000194804F027FF1949194804F023FF19499B
:102F8000194804F01FFF19491948BDE8084004F02A
:102F900019BF00BFCFF40000A0050020F52D0000F0
:102FA000D3F40000FD1F0000D8F40000853D0000B0
:102FB000DDF40000D13D0000E2F4000085210000B6
:102FC000E6F40000B91F0000EAF4000095250000B7
:102FD000EFF40000112A0000F3F40000B526000011
:102FE000F6F4000059200000FAF40000E11F000090
:102FF00000F500007FB51E4C2368002B35D01D4E18
:1030000006F0C6FA3268904213D92368DD6865B1CC
:103010002B7C062B07D1294601A8FDF7D5FA012103
:1030200001A8FDF749FE6D68F1E706F0B1FA32300C
:103030003060114D06F0ACFA2A68904215D9236829
:10304000DC6864B1237C062B07D1214601A8FDF77B
:10305000BBFA022101A8FDF72FFE6468F1E706F034
:1030600097FA00F59C500830286004B070BD00BF8E
:10307000FC020020CC030020D403002010B5054C36
:10308000237801332370FFF7B5FF2378013B2370CA
:1030900010BD00BFF80200201FB5094B1B686BB1C3
:1030A000DC685CB1237C062B06D1214601A8FDF724
:1030B0008BFA01A8FDF78FFA6468F2E704B010BD3F
:1030C000FC0200202DE9F04F704F396889B00029CB
:1030D00000F0D6806E4A6F4804F073FD6E4B1860A6
:1030E00010B36E4D2B78FBB9C4686D4800F056FFE5
:1030F000002814BF012300232B7003D069496A48BC
:1031000005F054FD694B00221A606CB12B785BB15D
:10311000237C062B06D1206802A901F0BAF802A888
:1031200001F008F86468F0E7614A39685948614C71
:1031300004F047FD604A20603968564804F041FDBC
:103140005E4B5F4A1860002313602368A1469246D5
:10315000002B00F08380D3F80C80DFF888B1524C4C
:10316000D9F80030002B00F08E80B8F1000F72D03B
:1031700098F81020052AF5D14146464804F011FD83
:103180000128EDD9414602A8FEF7A8F802A8FEF7EB
:1031900067F8A8B102A8FDF767FF064680B90146A7
:1031A00002A8FEF707F8051E02A8BCBF6D42012663
:1031B000FDF77AFF9DF81820052A07D0062A24D0AB
:1031C00002A8D8F80480FDF761FFC9E718B9022109
:1031D00002A8FDF777FF0121284606F085FB0021B4
:1031E000284606F0A9FB5946204605F0DFFC294693
:1031F0000A22204605F043FD3249204605F0D6FC60
:103200003149204605F0D2FCDAE701900121284639
:1032100006F06AFB019BD6B113F1FF3618BF0126F9
:103220003146284606F088FB2849204605F0BEFCBA
:103230000A222946204605F022FD2549204605F0B0
:10324000B5FC0A223146204605F019FDD8E7013BBE
:103250005E425E41E4E7DB68CAF800301D4A396827
:103260000C4804F0AEFC1C4B1C4A18603968094835
:1032700004F0A7FC1A4B1860FFF70EFFFFF79AF94E
:1032800009B0BDE8F08FDB68FFDE00BFE803002077
:10329000A7F200004C050020DC030020E003002022
:1032A00029380000AAF20000A00500200C0400202C
:1032B000BAF200000003002098F90000EC0300209F
:1032C000E4030020C8F20000CDF20000C9F10000C4
:1032D0000EF00000CFF20000FC020020D2F200004D
:1032E0000C030020C0F2000030B5BFB005460C460C
:1032F0001C22002112A8119108F025FC012D40F399
:1033000082801F22616811A809F0DDFB11A9162037
:10331000FFF7ACF911A9574805F051FC564955483B
:1033200005F044FC534805F051FC544A5179137898
:10333000049111790391D178029191780191527899
:10334000009240214E4A19A809F084FA4D49494893
:1033500005F02CFC11A9474805F031FC19A9454896
:1033600005F02DFC434805F031FC0CA802F0F4F800
:10337000454906A806F097F811AA0CA9502329A8D8
:1033800003F0AAFC4FF47A6329A8399303F0D3FC25
:1033900019A929A803F0F6FD044629A803F0EFFDBA
:1033A000002C64D129A803F0FBFD29A9044609A833
:1033B00003F00CFF09A906A806F0BDF809A806F05D
:1033C0002DF829A803F0ACFC30492A4805F0EEFBA3
:1033D0000A222146274805F052FC2D49254805F0D0
:1033E000EEFBC82C41D1FEF74FFE0699294804F0A8
:1033F000F7FA294B1860D8B928491E4805F0D6FBC2
:103400006FF00A0426E0202211A91620FFF768F9C0
:1034100000288AD12022224911A809F054FB214911
:10342000144805F0C3FB11A9124805F0C8FB79E761
:1034300006A909A806F075F809A90E4805F0BAFB17
:1034400009A805F0EBFFFFF73DFE1749094805F015
:10345000ADFB0224154B29933BA805F0DFFF06A81E
:1034600005F0DCFF20463FB030BD1149C5E71149EA
:10347000C3E700BFA0050020A5F50000050300205C
:10348000CAF50000F9F500009AFF00000DF60000F3
:1034900085FE00004C050020E803002020F6000017
:1034A000B1FA0000ACF5000037F60000C0FE0000E5
:1034B0003EF6000058F6000038B5037C052B0546A3
:1034C0000C4601D0002038BD01460022074804F018
:1034D00070FB4369052BF5D12946044804F061FBD4
:1034E0008442CCBF00200120EDE700BF4C05002046
:1034F00010B501220C460146074804F05AFB436907
:10350000012043B10C2C06D8A04041F2424318429E
:103510000CBF0120002010BD4C0500202DE9F04F0C
:103520002DED048B87B006F033F87B4B05931A68BA
:103530009042C0F0EB80794B1B68002B00F0E680D6
:10354000DC68774E9FED779A002C00F0D180052142
:103550002046FFF7B1FF002800F0BD80042221467D
:10356000304604F026FB0746002800F0B4800146F0
:10357000304604F016FB012840F2AD8001222146BE
:10358000304604F016FB022245692146304604F01D
:1035900010FB032290ED058A2146304604F009FB1A
:1035A0000022D0F814903946304604F002FB012284
:1035B000D0ED058A3946304604F0FBFA4369B8EE8F
:1035C000C88A002B5ED12168574805F0F8FA5749A0
:1035D000554805F0EBFAF4EEC98AF1EE10FA04DD75
:1035E00022685349534804F0D4FF4F4805F0EEFADF
:1035F00021684D4805F0E3FA4F494B4805F0D6FAEB
:1036000018EE100A07F092FC4FF0020802460B4633
:10361000CDE90201CDF80080434805F00FFC474991
:10362000414805F0C3FA18EE900A07F07FFCCDF888
:1036300000800B46024682463B488B4605F0FEFB67
:103640003F49394805F0B2FA0A224946364805F0A2
:1036500016FB002DB4BF68422846012106F044F94C
:1036600038464946FFF744FF0746D8B1002D03DA34
:103670000021684206F060F90021284606F05CF956
:10368000304925E001223946304604F092FA436978
:10369000013B4361002B9ED122682B49254804F051
:1036A00078FF98E70022294BDDE9020107F0DEFAF6
:1036B00052465B4607F022FF78B1002D03DA394607
:1036C000684206F039F90121284606F035F920490B
:1036D000154805F06BFA646836E7B4EEE88AF1EE57
:1036E00010FA03D8002DC7DA0121C2E71949EFE724
:1036F00005F04EFF059B00F5EA403030186007B03A
:10370000BDEC048BBDE8F04FFFF784BB07B0BDEC08
:10371000048BBDE8F08F00BFD80300200003002019
:103720004C05002000001842A005002060F20000B7
:1037300076F200001003002083F2000089F20000FE
:103740004EF100008FF200006AF200000000F03F2E
:1037500094F2000098F20000F8B502460F4608B94E
:103760000020F8BD0378002BFAD02B4B19680029F4
:10377000F6D02A4804F025FA04460028F0D00421A7
:10378000FFF79AFE08B90120EBE72146234804F031
:1037900008FA042821D1214804F05BFA054638468E
:1037A00007F0C4FB0B4602461C4804F042FAC8214D
:1037B00007461A4804F034FA3A460646294617489E
:1037C00004F00CFA32462946144804F007FA2A4657
:1037D0002146124804F002FAD5E7042221460F4898
:1037E00004F0E7F905460028CDD0014601220B4838
:1037F00004F0DFF9002206462946084804F0D9F90A
:103800004761736923B922680549064804F0C1FE7F
:10381000C8237361B7E700BF000300204C050020F8
:103820002EF500001003002070B52DED028B8CB03A
:10383000474C04940D4608EE102A00211C2205A8CE
:1038400008F081F9009404AA002408212846CDE953
:103850000144039400F0ECFC3E4B8DF821401B68C2
:10386000002B64D0694618EE100A00F051FD3A486A
:1038700005F0ACF93949384805F098F969463648F9
:1038800005F09DF93649344805F090F9354B364836
:10389000196804AA04F095F9054600284BD0334A6C
:1038A0000146314804F08DF946692B48314605F050
:1038B00086F92F49284805F079F9274805F086F957
:1038C000DFED2C7AB4EE678AF1EE10FA2FD0DFED3F
:1038D0002A7AB4EE678AF1EE10FA28D0B5EE408A63
:1038E000F1EE10FA23D0BEB123460322202104A812
:1038F00000F05AFD2022314604A809F0BEF81F4806
:1039000004F040FC40B11E4B93F9003023B96A46E5
:1039100004A91A4804F03DFE1A4A1348294604F047
:1039200050F9406918B118EE101AFFF715FF0CB0E6
:10393000BDEC028B70BD04A9074805F040F90C49A5
:10394000054805F033F9044805F040F9EFE700BFFA
:103950004E494C00E8030020A0050020C3F90000F8
:103960000FF10000DC0300204C050020EBEF00000D
:10397000DEF000000000FEC20000AA42100300209A
:10398000F8020020F0EF000013B500231946009361
:103990001A46084C084805F0C9F8084803F074FCBA
:1039A000204601F0D9FD0648214602B0BDE810408E
:1039B00004F09CBAE4020020D4020020D0020020CF
:1039C000100300202DE9F041044692B00D46454811
:1039D0004549164605F0EAF82146424805F0EFF859
:1039E0004249404805F0E2F8ADB10023AB5500F084
:1039F00088FCF9280BDDDFF8EC802F462E44BE4210
:103A00000CD017F8011B404605F0DDF8F7E7384900
:103A1000344805F0CBF812B0BDE8F081354F31489D
:103A200005F0D4F897F90020042A4FF0000311D1D3
:103A30000322412101A800F0B7FC01A809F015F804
:103A400006B2324601A9204609F02BF800B2A0B117
:103A50002949DDE70222412101A800F0A5FC01A8C7
:103A600009F003F806B2324601A9204609F019F818
:103A700000B210B100230122DBE734441F49204685
:103A800008F0C5FF40B9284608F0EFFF012803D928
:103A9000284604F055F9BEE72F21204608F0AAFF7A
:103AA000064628B1002303704378242BB3D0013697
:103AB0002378242BAFD0214601A8FDF71DFC01A8D7
:103AC000FDF7CEFB48B197F90020043A334618BF02
:103AD0000122294601A8FDF74DFA01A8FDF7D6FA03
:103AE00099E700BFA0050020D7F20000DAF200003D
:103AF000DDF2000004030020E2F20000EDF200001D
:103B000010B51E491E4886B005F050F81C4805F057
:103B10005DF848211B4803F0BAFB7B282BD14FF0FE
:103B2000FF320392184A009200234822CDE9013364
:103B3000CDE90423FEF7A8FA6946144803F04CFFC8
:103B4000134B186040B913490D4805F02FF80C4885
:103B500005F03CF800200CE00F49094805F026F874
:103B6000074805F033F8FFF7ADFA0C4801F0DAFD2D
:103B7000012006B010BD0A49E6E700BF96F6000036
:103B8000A0050020D002002054FF00004C050020BA
:103B9000E8030020B1F60000BDF60000E4020020BA
:103BA000C4F6000010B5584C94F900300B3390B0B7
:103BB000172B15D8DFE803F06051141414141414F3
:103BC0001414140C232B492E141414141414145903
:103BD00005F0DEFC4D4B1B68984201D9FEF7A0FFB3
:103BE00094F90030002B6BDD494801F095FB01385A
:103BF000042865D8DFE800F0687884864D00454BDE
:103C0000197839BB0846FFF76FFB2070E8E7FEF72D
:103C100091FDE5E705F0BCFC3C4B1B68984214D9CC
:103C2000002303224021684600F0BEFB3A49684663
:103C300008F0D1FE6946394804F005FD03233849F0
:103C40003848237004F0B2FFCAE7344804F09AFA07
:103C50000028C5D102232370C2E705F099FC2B4B45
:103C60001B689842BCD90023F5E705F091FC274B6F
:103C70001B689842EED8B3E7FFF742FF0028E9D16E
:103C800005F086FC214B00F59C5008301860F623A7
:103C9000E1E72549234804F089FF224804F096FF14
:103CA0001E4804F06FFA10B11C4804F03AFA05F00F
:103CB0006FFC00F5EA403030144B1860F623237097
:103CC00094F9000010B010BD1849164804F06EFFBA
:103CD000124804F057FA10B1104804F022FA05F027
:103CE00057FC00F57A70E7E711490E4804F05EFFD3
:103CF0006846074901F04BFB684600F02FFBDFE701
:103D00000C49E2E70C49F0E704030020D00300204F
:103D1000DC040020DC0200207CF9000010030020FD
:103D2000C6F90000A0050020DDF90000E5F900005B
:103D3000F9F9000016FA000029FA000008B504F0AD
:103D40009BF8FFF72FFF012802DD0A4804F038FB3B
:103D5000094B1B7823B1094B1B680BB100F0D8F954
:103D6000074B1B680BB1FFF7D9FBBDE80840FFF715
:103D700041B900BF10030020E0030020DC03002055
:103D800000030020FFF7BCBE08B5FFF7CBF8FEF735
:103D9000ADFFFFF793F8FFF7B3FE142005F012FC18
:103DA000074B186810B1074900F0A8FD06490748FD
:103DB00004F07CFC4FF4FA70BDE8084005F002BC4A
:103DC000F8030020B51F0000C539000010030020D3
:103DD00008B5FFF789FA034B18700348BDE808409F
:103DE00001F0A0BC04030020E40200202DE9F04F04
:103DF00085B005F0CDFB5D4900F59C595C4804F0A9
:103E0000EBFE5C4B0293186809F1080908B100F059
:103E1000A9FD594C594E2568306800210BB2AB42C0
:103E200001F10101C0F28C80554DDFF86CA1029BBD
:103E30001868002800F08B8021682B6803EBC10113
:103E400000F018FF002840F382802368132B7EDCEB
:103E500005F09EFB48457AD22B682068072103EBCA
:103E6000C00000F06FFD2B680193019A236802EBFC
:103E7000C30B9BF807208242D9D14FF000080FFAFC
:103E800088F7BB42039325DD019B082203EBC700A3
:103E9000594607F025FE08F10108039B0028EED1E2
:103EA0003168019031F81730314843F0010321F8AF
:103EB0001730344904F07AFE2B682068019A03EB2E
:103EC000C000082100F094F92F49294804F084FE2D
:103ED000002FACDADAF80030002BA8D03368226863
:103EE0002348012123F81210284904F05FFE0A221A
:103EF00021681F4804F0C3FE25491D4804F056FE02
:103F00002B682068002203EBC000082100F070F944
:103F1000174804F05BFE22682B6803EBC20113F81C
:103F20003230282B08D10C22DAF8000000F0D5FF3F
:103F3000029B186800F0F0FD23680133236076E7E8
:103F400030F8132022F0010220F8132066E711490F
:103F5000074804F02BFE0A222168054804F08FFE72
:103F6000034805B0BDE8F04F04F030BECAFB0000C6
:103F7000A0050020F80300200C04002014040020F9
:103F800010040020E3FB0000EAFB0000F1FB00004E
:103F9000F6FB0000D4FB000004040020F8B52A4C16
:103FA00023680746002B47D128492948294E04F0A9
:103FB000FDFD274804F00AFE142005F03BFB0546F2
:103FC00000F08CFC1C20256005F034FB21680546C0
:103FD00000F0E6FEA020356005F02EFB1E4B1860B9
:103FE000282005F029FB1D4B18601D4800F0E8FA59
:103FF000206800F08BFC054600B31A49144804F011
:10400000EBFD206800F0C6FD206800F08BFC16492F
:104010000F4804F0E1FD206800F000FE18B11349DC
:104020000B4804F0D9FD306800F09AFF104B30685F
:104030001F60002100F0E8FF012004E00D49044862
:1040400004F0CAFD2846F8BDF80300205CFB000020
:10405000A005002004040020100400201404002007
:10406000200400207DFB000090FB0000B0FB00005E
:10407000FC030020BCFB0000F8B5204F3868002886
:1040800039D01F4D1F4AB5F90030126893422E46B1
:1040900006DBFFF7ABFE00232B804FF4FA50F8BD90
:1040A000194CD4F800C00CEBC3011CF833C0BCF1B0
:1040B000280F19D101F038F8144B1B6802462BB1B8
:1040C000B5F90000216801EBC00198472368B6F9F3
:1040D0000010386803EBC10100F0CCFF33880133D6
:1040E000338040F6C410DAE701334FF4FA602B80D6
:1040F00090FBF2F0D3E74FF0FF30D0E7040400204C
:10410000080400200C04002010040020FC03002000
:1041100038B5074D05F03CFA2B68984206D305F0F8
:1041200037FA0446FFF7A8FF2044286038BD00BFD7
:104130000004002070B51F4C2368132B39DC1E4A85
:104140001E4D1268012122F813102968026841F8F7
:10415000332001EBC306426872601949194804F024
:1041600025FD0A222168174804F089FD16491548E3
:1041700004F01CFD2B682068002203EBC00008211E
:1041800000F036F80F4804F021FD22682B6803EB9D
:10419000C20113F83230282B08D10C4B0C221868BE
:1041A00000F09BFE0A4B186800F0B6FC2368013350
:1041B000236070BD0C0400201404002010040020B3
:1041C000F1FB0000A0050020F6FB00000404002025
:1041D000F803002007B5002300931A461946034848
:1041E00004F0A4FC03B05DF804FB00BFF003002062
:1041F000F8B5441E0D4D16466718BC420ED014F893
:10420000011F10220909284604F039FD21781022E7
:1042100001F00F01284604F032FDEEE726B1034815
:10422000BDE8F84004F0D2BCF8BD00BFA0050020F6
:1042300070B501380C4D13464618B04203F1020325
:104240000CD010F8014F24112C5D03F8024C0478B7
:1042500004F00F042C5D03F8014CEEE709B20023D3
:1042600002F8113070BD00BF1AFC0000A0F161031C
:10427000052B02D85738C0B27047A0F14103052B77
:1042800001D83738F7E73038C0B20A2828BF0020F5
:10429000704738B50139841C00F1120514F8020C7E
:1042A000FFF7E4FF0001C2B201F8012F14F8010C7E
:1042B000FFF7DCFF02341043AC420870EED138BD8A
:1042C00038B50546D8B10468ACB124789CB12868EB
:1042D00003783BB12D2B05D0303B092B02D901309F
:1042E0002860F4E707F0E0F92C210446286808F07C
:1042F00081FB10B92860204638BD0130FAE704463A
:10430000F9E708B5002008F08BFDADEB000008BD13
:10431000704730B5441E224612F8013F002BFBD1F6
:104320001A460A2514F8010F70B1032A14DC2E284E
:1043300006D1FF2B10DC8818013203710023F1E74E
:10434000303805FB0303EDE7FF2B04DC032A02DC16
:10435000114401200B7130BD0020FCE72DE9F04134
:104360000E4D0F4FDFF83C8006460024032C0ED084
:1043700033190A221979284604F05FFC4146284681
:10438000013404F013FC042CF0D1BDE8F081F17984
:104390000A22284604F051FC3946F0E7A005002027
:1043A000FDFB00006CF900002DE9F047DFF8D48038
:1043B000D8F8006004460D4617469946002E3CD0BA
:1043C000337C062B38D1264A2648314603F0F9FBC8
:1043D000022F82462CD0032F2CD1234AD8F800106C
:1043E000204803F0EEFB0646BAF1000F25D0DAF8BC
:1043F00014102A46204608F066FB2A461B49204630
:1044000008F03BFBE6B171692A46204608F035FB0F
:104410002A461649204608F030FBB9F1000F04D0B7
:104420002A464946204608F028FB2046BDE8F0878A
:104430000F4AD3E70026D7E700262A460D49D9E7D9
:10444000022F0AD0032F05D0012FE1D10A4B2A46B3
:104450001968DAE72A460949D7E72A460849D4E71E
:1044600010FC00004C05002063FD00000BF600006E
:1044700015FC000034FC0000E00200202EFC0000CF
:104480002BFC0000EC03002030B585B0002301AA0E
:104490000A2541B1B1FBF5F405FB14113031D154BB
:1044A00021460133F5E71A44411EC41812F8015D94
:1044B00001F8015FA142F9D10022C25405B030BD1C
:1044C00010B5054C0549204604F079FB2046BDE8AF
:1044D000104004F07BBB00BFA005002000FC0000E2
:1044E00007B5002300931A461946034804F01EFB43
:1044F00003B05DF804FB00BF180400202DE9F84369
:1045000080460D46174601EB02090C464C45A4EBCC
:1045100005060BD0D8F8003014F8011B1B68404684
:1045200098470028F2D13046BDE8F8833E46FAE7C6
:104530007047203004F0ADBC203004F09CBC20302B
:1045400004F0ADBC38B5437F0D460BB9002038BD33
:1045500000F16804204604F0AAFC0028F6D12046A9
:10456000294604F079FC0120F1E700002DE9F04133
:104570001E4600254FF47A73C0E901530E4B0446E2
:1045800040F8203B1746884604F05DFC04F16800C3
:1045900004F059FCC4E90487084B9DF818202676DE
:1045A00053F8222062769DF81C2053F82230A3761F
:1045B00065772046BDE8F08144FC0000BCFF0000A8
:1045C000827E4FF0A04102F5E07210B5012340F267
:1045D0000C64C37641F82240427E02F5E07241F855
:1045E000224002694FF0CC71C2F8241502690621FD
:1045F000C2F800150269817EC2F808150269417E81
:10460000C2F80C1590F91820510902F01F029340CE
:1046100060310F4A42F8213090F91830002BBDBFAD
:1046200003F00F0302F6FC32D2189B18B5BF4023EB
:104630004022137683F8002390F91830012259099B
:1046400003F01F0302FA03F3014A42F8213010BDC0
:1046500000E100E02DE9F041044688461F4615467A
:10466000002A50D000F12006304604F000FC2369F7
:10467000C3F88885236901221A622369C3F8346567
:104680002369C3F8385523691A602269D2F84C317E
:104690001BB9D2F82431002BF8D00023C2F84C31DA
:1046A0002269D2F85C311BB9D2F82431002BF8D042
:1046B0000023C2F85C3122696FB9D2F8243153B9B2
:1046C0000123D3612369D3F84821002AFBD00022BB
:1046D000C3F8482109E0012353612369D3F8042179
:1046E000002AFBD00022C3F804212369D3F8242137
:1046F00012B10022C3F824212369D3F83C052066B7
:10470000C0B2BDE8F0811046FBE70123FFF7A2BF6E
:1047100010B5044680F8B010683004F0A8FB0123FF
:10472000637710BDF8B500234377036990F8B02094
:10473000C3F88825036901261E62036900F1680534
:104740000446C3F8445528460F4604F0A2FB2369EB
:10475000C3F8480523699E602369D3F850211AB92C
:10476000D3F82421002AF8D00022C3F8502128468B
:1047700004F08FFB236930B1D3F860211AB9D3F864
:104780002421002AF8D00022C3F8602123696FB9E0
:10479000D3F8242152B90122DA612369D3F84821E0
:1047A000002AFBD00022C3F8482109E001225A6107
:1047B0002369D3F80421002AFBD00022C3F8042186
:1047C0002369D3F8240168B10022C3F824212369A6
:1047D000D3F8C404C3F8C404022803D004280CBFCF
:1047E00003200420F8BD0121FFF79CBF70B5436989
:1047F000D3F86421044692B10022012500F120067D
:10480000C3F864210577304604F031FB6369C3F8CF
:10481000346563694022C3F8382563691D636369A1
:10482000D3F86821DAB10025C3F8685104F16806AD
:10483000012363772577304604F019FBD4F8B430B0
:1048400003B19847636965773046C3F8446504F05F
:1048500020FB6369C3F84805636901225A636369F1
:10486000D3F8042162B10022C3F80421237F3BB1B5
:104870006369D3F83C05D4F8B830206603B1984793
:104880006369D3F8242152B10022C3F8242163695B
:10489000D3F8D024C3F8D024636901225A6170BDD3
:1048A0000148FFF7A3BF00BF2004002007B516236F
:1048B0001722CDE900324FF040220423114603486D
:1048C000FFF754FE03B05DF804FB00BF2004002096
:1048D0000148FFF788BF00BF2004002010B54FF447
:1048E000C053038000230446837003610248FFF72E
:1048F00067FE204610BD00BF200400200161704704
:1049000041780148FFF704BF2004002008B5FFF7F5
:10491000F7FF0348FFF767FFB0FA80F0400908BDD2
:1049200020040020012303707047FF23C37200237B
:104930000373C370037143718371C3710372437254
:104940008372704710B5064A01440023884204D0A0
:1049500010F8014B6340D35CF8E7184610BD00BF68
:104960005CFC0000FFF7E1BF38B5084C0D46FFF7CF
:10497000C7FFE1212046FFF7E5FD29462046FFF766
:10498000E1FDBDE83840FFF7A3BF00BF20040020D1
:1049900010B5054C417801222046FFF7B6FE2046AF
:1049A000FFF7CAFDC0B210BD2004002010B5F021F1
:1049B0000446FFF7D9FF2046BDE81040FFF7E8BFE7
:1049C00070B5054604F0E4FD002400F57A7604F0A5
:1049D000DFFDB04246D22846FFF7E8FFC307044692
:1049E00046D52B6903B198471420013800BF00BF9A
:1049F00000BF00BF00BF00BF00BF00BF00BF00BFBF
:104A000000BF00BF00BF00BF00BF00BF00BF00BFAE
:104A100000BF00BF00BF00BF00BF00BF00BF00BF9E
:104A200000BF00BF00BF00BF00BF00BF00BF00BF8E
:104A300000BF00BF00BF00BF00BF00BF00BF00BF7E
:104A400000BF00BF00BF00BF00BF00BF00BF00BF6E
:104A500000BF00BF00BF00BF00BF00BF00BF00BF5E
:104A6000C3D1B4E70123AB700249034804F0BEF898
:104A7000204670BD5CFD0000A005002010B5E121BE
:104A80000446FFF771FF2046BDE81040FFF780BFE6
:104A900010B50446FFF794FF2046FFF731FF96213B
:104AA0000648FFF74FFDFFF713FF2046FFF788FF8B
:104AB0002046BDE81040FFF7E1BF00BF2004002002
:104AC000FFF7E6BF10B5C3210446FFF74DFF2046B0
:104AD000BDE81040FFF75CBF38B504460D46FFF750
:104AE0006FFF2046FFF70CFFD2210A48FFF72AFD8F
:104AF000E94345EA0111C9B20648FFF723FDFFF774
:104B0000E7FE2046FFF744FFA8421CBF0423A37022
:104B100038BD00BF2004002010B50446FFF7D2FFC7
:104B200040F00401C9B22046BDE81040FFF7D4BFF1
:104B300070B5164604460D46FFF742FF16B12046F3
:104B4000FFF7EAFF2046FFF7DBFEA5210548FFF748
:104B5000F9FC29460348FFF7F5FCBDE87040FFF774
:104B6000B7BE00BF2004002070B500220C465521BE
:104B70000646FFF7DDFF651E073415F8011F00220A
:104B80003046FFF7D5FFA542F7D170BDFFF7ECBF68
:104B9000FFF7CEBF10B50446FFF7B2FE2046002255
:104BA000F021FFF7C5FFBDE81040FFF791BE000000
:104BB00070B5164605460C46FFF702FF16B12846AB
:104BC000FFF7AAFF2846FFF79BFE87210648FFF75D
:104BD000B9FC002C0CBF214680210348FFF7B2FC32
:104BE000BDE87040FFF774BE2004002010B500221D
:104BF00004460121FFF7DCFF2046FFF7E1FEC0F38A
:104C0000401010BDFFF7F2BF10B50446FFF75AFF82
:104C100020460021BDE81040FFF75EBF38B50446CE
:104C2000FFF7CEFE2046FFF7EFFF2046FFF7C8FE56
:104C30002046FFF765FEB4210D48FFF783FCFFF720
:104C400047FE2046FFF7BCFE430744BF0223A37084
:104C50002378054643B12046FFF734FF40F00101B9
:104C6000C9B22046FFF738FFC5F3400038BD00BF8A
:104C7000200400202DE9F74F057B04460F46002D48
:104C80007AD1FFF7CBFF40B93C493D4803F0AEFF76
:104C90004FF0FF3003B0BDE8F08F2046FFF790FEE5
:104CA0002A46F0212046FFF743FFDFF8DC804FF073
:104CB000FF394FF0010A94F90B30EEB24FEAD60BF0
:104CC0009D4206F007060AFA06F62CDA04EB0B03FF
:104CD000DB78334020460193FFF772FE2046FFF752
:104CE0000FFE78214046FFF72DFC019B002B0CBFE7
:104CF000194680214046FFF725FCFFF7E9FD2046D5
:104D0000FFF75EFE8206014600F040030FD59BB11F
:104D100002221B4803F0CCFF1A49194803F066FF32
:104D20006FF00100B6E70CBF01230023D2E71BB9E7
:104D3000080658BF4FFA85F904EB0B03090693F9EF
:104D4000032076B205F101054CBF3243B243402D3A
:104D5000DA70B0D1B9F1FF3F04BF0123237384F8A7
:104D60000B90E31C013F0B3413F8012B07F8012FC4
:104D7000A342F9D101208DE700208BE767FD0000F9
:104D8000A005002073FD00002004002008B5FFF7F7
:104D900071FF20EAE070C0B208BDFFF73FBF704767
:104DA000054A8261002202710270092242700122CA
:104DB00081608270C27070479F4D000010B50C4634
:104DC00020460721FFF7BEFDE3791B1A58425841E0
:104DD00010BD70B5044680680E461546FFF7DDFF2E
:104DE000B8B13146A068FFF7D1FE0022BE21A0680D
:104DF000FFF7CEFE6E1E0835A068FFF761FE06F8CD
:104E0000010FAE42F8D1A068FFF7C7FF431E58421A
:104E1000584170BD10B51446FFF7DBFF38B10821CB
:104E20002046FFF78FFD237A1B1A5842584110BDC8
:104E300070B504460D4680681646FFF7AEFF29465A
:104E4000A068FFF7A3FE00224E21A068FFF7A0FE96
:104E50000022B178A068FFF79BFE0022F178A068DD
:104E6000FFF796FE2B78102B04D000223179A06832
:104E7000FFF78EFEA068FFF790FF2946A068FFF7B6
:104E800085FE2278A0684821FFF782FE142004F0F6
:104E900099FB237813B10A2004F094FBA068BDE8C5
:104EA0007040FFF77ABF38B504460D468068FFF7BB
:104EB00074FF2946A068FFF769FE0022B421A068AC
:104EC000FFF766FEA068FFF79DFE0546A068FFF7A6
:104ED00064FFB5FA85F0400938BDF0B585B01446D9
:104EE00001AA07460E46FFF795FF054690B13378B5
:104EF000102B0FD00B2C10D00C2C03D00A2C0ED161
:104F00003F2300E07F2301AA314638468DF8083060
:104F1000FFF78EFF284605B0F0BD5F23F3E71F23A0
:104F2000F1E71FB50B78102B10D001AAFFF772FF25
:104F300078B19DF808303F2B0ED003D81F2B0DD031
:104F4000002006E05F2B03D07F2BF9D10C2000E07E
:104F50000B2005B05DF804FB0A20FAE70920F8E70A
:104F60002DE9F04387B0044604F012FB00F51C5510
:104F7000A068224F224EDFF88C80FFF7F3FC00235D
:104F80001035237101A9A068FFF700FF90B304F06A
:104F9000FFFAA8422ED201A92046FFF70FFF20B347
:104FA0004146304603F00BFE237833B901A9204671
:104FB000FFF779FF08B10123237003AA01A9204656
:104FC000FFF707FF01A9204694F80190FFF7A9FF1A
:104FD000814505D960782379607001332371D1E769
:104FE00001A92046FFF79DFFF5E73946304603F05B
:104FF000E6FDC7E707B0BDE8F08300BF86FD00000F
:10500000A005002084FD0000817070471FB501AA33
:10501000FFF7DFFE9DF80400003018BF012005B047
:105020005DF804FB0939C9B20229F8B598BF104BE5
:105030000546164694BF33F9114040F2EE248AB17A
:10504000C3787BB103786BB904F0A2FA0746314606
:105050002846FFF7DBFF20B904F09AFA001BB8429C
:10506000F5D3F8BD2046BDE8F84004F0ABBA00BF68
:105070007EFD0000F8B504460F46FFF752FF0646D6
:1050800010B900252846F8BDA068FFF786FE002865
:10509000F7D03946A068FFF779FD2278A06844214F
:1050A000FFF776FDA5782DB13A4631462046FFF749
:1050B000B9FFE7E70125E5E710785378C00040EA3B
:1050C000C3200B78102B00B20BD1D1799379C0009B
:1050D000CB1ADB0120F07F0093FBF1F3103B184467
:1050E00000B2704730B585B001AA04460D46FFF7FF
:1050F00091FE30B101AA29462046FFF7DDFF05B039
:1051000030BD0148FBE700BF80E4FFFF10F5DC5F26
:10511000CABF07EE900ADFED037AFAEEEC7A17EEDB
:10512000900A70470000FEC208B5FFF7DBFFBDE83C
:105130000840FFF7EBBF042302461946012000F0A8
:105140002DBE042302461946052000F027BE024664
:1051500006230421092000F021BE0423024619463B
:105160000F2000F01BBE00002DE9FF41044600693E
:105170000E461746984608B104F060FA782004F00D
:1051800059FA78220546002106F0DDFC05F15400AD
:1051900000F002FC217D2561234800F055FE00252A
:1051A0003046FFF7D4FF2B462A462946009502A831
:1051B00003F0BCFC03A8FFF7D0FF29462E2000F027
:1051C0001BFE10F001052BD043463A4631462069BC
:1051D00001F051FA0128054622D1216902A800F008
:1051E00070FF03A8FFF7B9FF216902A800F077FF5D
:1051F00003A8FFF7A0FF216902A800F069FF03A838
:10520000FFF79FFF216902A800F070FF039B636016
:10521000206900F072FFA060206900F070FFE0607C
:10522000284604B0BDE8F0811F050020F8B504460B
:105230000F46017D0A4816461D4600F005FE384619
:10524000FFF785FF301DFFF788FF06980430FFF752
:1052500072FF07980430FFF774FF6B686360F8BD56
:105260001F050020F0B58DB01E46002317460093A1
:10527000FF2304460D461A46194602A803F056FCC1
:105280007A680C4B0493CDE905237268CDE90723B6
:10529000129A5268CDE90923039B0B930AAB019341
:1052A00008AB009304AA06AB29462046FFF7BEFFD1
:1052B0000DB0F0BD2C00010010B554685B680A4ABF
:1052C0008AB0CDE90732012303948DF80F30039B98
:1052D000099308ABCDE904240692009304AA06AB17
:1052E000FFF7C0FF0AB010BD2C0001007FB5094BCD
:1052F00052680493CDE90232012301928DF8073000
:10530000019B059302AA04ABFFF7D6FF07B05DF837
:1053100004FB00BF2C00010037B5044600212E20FD
:1053200000F06AFDC3072ED5206970B301F0BCF907
:105330000228054601D0042822D12169684600F0E0
:10534000C0FE01A8FFF709FF2169684600F0C7FE0B
:1053500001A8FFF7F0FE2169684600F0B9FE01A838
:10536000FFF7EFFE2169684600F0C0FE019B636015
:10537000206900F0C2FEA060206900F0C0FEE0607D
:10538000284603B030BD0525FAE70546F8E710B515
:10539000044603F0C3FB0423E21800210F2000F0B1
:1053A00003FE204610BD10B5044603F0B7FB0423EE
:1053B000E2180021052000F0F7FD204610BD10B5D1
:1053C000044603F0ABFB0423E2180021012000F0A7
:1053D000EBFD204610BD0000024A02604A684260B0
:1053E000704700BF2C00010037B500240A4D00941F
:1053F000234621462246094803F098FB284603F03D
:105400008DFB0A232B75064B2C611878012103B004
:10541000BDE8304004F068BADC040020F404002049
:105420001E05002008B503681B6B984780F001003B
:10543000C0B208BD13B502AB026803F8011D546881
:1054400019460122A04702B010BD007C083818BFE1
:1054500001207047037C087C984203D1083818BFAC
:10546000012070470020704770B590B0044604A832
:1054700015460E4603F052FB07A800F08DFA684669
:1054800003F04CFB0D4902A8FFF7A6FF02A904A8F0
:1054900001F055F96A46314604A801F001FB0128E4
:1054A00009D12368064A9B690292019A039202A9D4
:1054B0002A462046984710B070BD00BFDC0400208B
:1054C0002C00010038B50546007C0828144604D19C
:1054D00001236B600024204638BD92B200F052FBDD
:1054E0000028F5D0F7E7000008B5017C082903D0B3
:1054F000024800F015FD08BD0020FCE71F05002054
:1055000007B501220DF10701007C00F07DFB0028AA
:10551000CCBF9DF807004FF0FF3003B05DF804FBEF
:1055200008B512B2007C00F06FFB08BD036813B52C
:105530009B680446984740B10DF10701207C00F0BC
:1055400091FB9DF8070002B010BD4FF0FF30FAE765
:10555000007C00F095BB000000214FF47A72C0E996
:105560000112024A0260082202747047C8FD00005E
:10557000017C082906D04901083101F0F801032017
:1055800000F03ABC002070472DE9F84F0E46017C30
:1055900008290446174609D00A22594803F088FB17
:1055A0005849574803F022FB002099E05448DFF89F
:1055B0006CA1DFF84C9103F009FB00255FFA85FB35
:1055C0004FEA4B11083101F0F801032000F014FC00
:1055D00051468046484603F0F2FA102229464846D2
:1055E00003F04DFB4849484603F0E9FA10224146D2
:1055F000484603F05FFBB8F1000F04D008F0FB0849
:10560000B8F1180F43D1414984F810B03C4803F079
:10561000D6FA1022217C3A4803F04CFB237C082B5D
:10562000C2D03B4DDFF8D8802B88DFF8F4A00133DF
:105630002B8003F0ADFF2B8853FA80F080B2B0F5D9
:10564000806F36BF4FF4806328802B802A88207CAF
:105650000023012100F03AFAF51C06F1070915F8BC
:10566000011F0A22404603F023FB5146404603F047
:10567000A6FA4D45F3D1224803F0A8FA3A46311D67
:10568000207C00F04BFA30B9082323748CE70135F5
:10569000082D93D1C2E703F07BFF00F56A5506465B
:1056A00018352046FFF764FF17281BD0AE4219D2E9
:1056B00003F06EFF85421AD90A2003F083FFFDF73D
:1056C000DDFC2046FFF754FF0028DDD02046FFF721
:1056D0004FFF1728E5D10F49094803F087FA012049
:1056E000BDE8F88F03F054FF0028E5DBE0E70A4946
:1056F000034803F07BFA236820465B6A984753E728
:10570000A00500208FFD0000A2FD0000ABFD000001
:1057100000000020B4FD00005FFD00009EFD0000C1
:105720006CF9000038B50446007C082826D000F04B
:1057300021FA03F02DFF05462046FFF719FF48B177
:1057400003F026FF401BB0F57A7F03D2012003F05F
:1057500039FFF1E72046FFF70BFF10B1207C00F086
:10576000A7F9227C064B0748002123F812100823D2
:1057700023740549BDE8384003F038BA38BD00BF8E
:10578000FC040020A005002088FD000010B5037C6B
:10579000082B044616D0FFF7EBFE182806D80A4B54
:1057A00023FA00F0C04300F0010010BD1C2807D10F
:1057B000236820469B689847003018BF0120F4E713
:1057C0000120F2E70020F0E70100100107B50023F7
:1057D00000931A461946034803F0A8F903B05DF890
:1057E00004FB00BF0C05002003681B6B184700007A
:1057F000024A02608A694260704700BF2C000100C3
:10580000808B7047008C704713B502AB026803F8B9
:10581000011D546819460122A04702B010BD10B501
:105820000446238C23B123682046DB689847F8E7B9
:1058300010BD000010B50446007C082808D000F018
:1058400037F9227C034B002123F81210082323741C
:1058500010BD00BFFC0400200023C3830431007C82
:1058600000F02CBA007C00F041BA10B593B20446A7
:105870000A46C18B007C00F005FAE38B0344E38306
:1058800010BD13B5038C04461BB94FF0FF3002B0B6
:1058900010BD01220DF10701007C00F0B5F90028D0
:1058A000F3DD238C9DF80700013B2384EFE710B55F
:1058B000038C044613B94FF0FF3010BD934294BFE0
:1058C0001AB212B2007C00F09FF90028F3DD238C9D
:1058D0001B1A2384F1E707B5038C4BB10DF10701C7
:1058E000007C00F0BFF99DF8070003B05DF804FBF1
:1058F0004FF0FF30F9E7000013B5036804465B6919
:105900009847217C104800F00BFBD0B10822694673
:10591000207C00F079F9002813DD694604F11400B9
:1059200003F018F99DF804209DF805309DF8070054
:1059300003EB0223A3839DF8063000EB032080B223
:10594000208402B010BD00BF1F050020F8B5037C05
:10595000082B04460E4601D00020F8BD0025EFB20A
:105960007901083101F0F801032000F045FA60B92F
:105970002774207C0828EFD00023668223843246D7
:10598000022100F0A3F80120E7E71828F0D0013544
:10599000082DE4D1EDE7000010B500224FF47A7332
:1059A000C0E90123044B0360082304460374143048
:1059B00003F0B4F8204610BD08FE000070B590B0AA
:1059C000044604A815460E4603F0A8F807A8FFF7FA
:1059D000E3FF684603F0A2F80D4902A8FFF7FCFCBC
:1059E00002A904A800F0ABFE6A46314604A801F003
:1059F00057F8012809D12368064A1B6A0292019AC6
:105A0000039202A92A462046984710B070BD00BFF5
:105A1000DC0400202C00010007B5002300931A4687
:105A20001946034803F082F803B05DF804FB00BF99
:105A30001405002040010C300A46042300F0FC014C
:105A40000C2000F0ABB90B464101083101F0F80120
:105A5000184600F0D1B908B50221FFF7F4FF08BDE0
:105A60000B4641010C3101F0FC01184600F06EB903
:105A700038B50A0A05460C460421FFF7F1FFE2B2E9
:105A800005212846FFF7ECFF38BD08B50A4602217C
:105A9000FFF7E6FF08BD38B50A0A05460C46102197
:105AA000FFF7DEFFE2B211212846FFF7D9FF38BD2C
:105AB00010B5014604461022034800F0E4FAFF2125
:105AC0002046FFF7E2FF10BD1F050020F8B51F4676
:105AD0004B1E042B04460E46154619D8FFF7E8FF67
:105AE00046EA070200212046FFF7BAFF55B12946D2
:105AF0002046FFF7BDFF07480122214600F0C3FA08
:105B00000120F8BD044B1988013189B21980EFE7F3
:105B10000020F6E71F0500201C05002038B50B7893
:105B2000FF2B054614460AD14B78FF2B0ED18B78FC
:105B3000FF2B0BD1CB78FF2B08D1002014E02BB921
:105B40004B781BB98B780BB9C87868B16CB1284613
:105B5000FFF770FF21462846FFF79DFF0448042207
:105B6000294600F090FA012038BD2046FCE700BF2E
:105B70001F05002001460822014800F084BA00BF3A
:105B80001F050020B2F5006F2DE9F04128BF4FF44A
:105B90000062DFF8708004460E46154621464046F6
:105BA00000F0A0F9032107462046FFF74CFF172815
:105BB00001D01C281FD1AF42F0D3324621461148F4
:105BC0002B4600F0E8F9202221460E4800F05BFA4F
:105BD0002046FFF740FFC3060FD403212046FFF7FE
:105BE00032FF06460028F3D12046FFF761FF354615
:105BF0002846BDE8F0810025DFE710212046FFF7A9
:105C000044FFF5E71F050020F7B505460E4601469F
:105C10001348174600F084F904B274B903212846EA
:105C2000FFF711FF142805D020B1B0F11C0418BFF4
:105C30004FF0FF34204603B0F0BDBC42A8BF3C4645
:105C4000002CF7DD0023009332462946A3B2044816
:105C500000F0EEF940222946014800F014FAE9E785
:105C60001F05002013B501240A460094014623466F
:105C7000024800F0DDF9204602B010BD1F050020EB
:105C800070470000F7B505460E4601460A481C4617
:105C9000174600F027F9A04204D22946064800F032
:105CA00021F9044600943B4632462946024800F05A
:105CB00047F9204603B0F0BD1F05002038B50B782A
:105CC000054614462BB94B781BB98B780BB9C878AD
:105CD00040B144B12846FFF7ADFE28462146FFF704
:105CE000DAFE012038BD2046FCE7000038B5014649
:105CF000044620220C4800F0C6F92046FFF7ABFE10
:105D000010F010050AD12046FFF7A5FE0307F4D5D1
:105D100020461821FFF7B9FE284638BD204610213D
:105D2000FFF7B3FE0120F8E71F050020024B00211A
:105D3000187803F001BE00BF1E050020024B0121B0
:105D4000187803F0F9BD00BF1E050020F8B5114C0E
:105D5000114B05460F46204616460ECB03F076FE45
:105D6000FFF7E4FF290A204603F07DFEE9B2204652
:105D700003F079FE3946204603F075FE3146204691
:105D800003F071FEFFF7DAFF204603F06BFE0120FF
:105D9000F8BD00BF1406002020050020F8B51D4600
:105DA000134B06460F46134814460ECB03F04EFE27
:105DB000FFF7BCFF310A0F4803F055FEF1B20D4862
:105DC0000C4E03F050FE39460A4803F04CFE013CED
:105DD0006719BC4205D014F8011F304603F043FE9A
:105DE000F7E7FFF7ABFF034803F03CFE2846F8BD9A
:105DF000200500201406002070B5114B114C0546FB
:105E00000E4620460ECB03F021FEFFF78FFF290A36
:105E1000204603F028FEE9B2204603F024FE314676
:105E2000204603F020FE0021204603F01CFE05461C
:105E3000FFF784FF204603F015FE284670BD00BF23
:105E4000200500201406002038B51A4B1A4D1A7888
:105E5000297042B300244FF4FA601C7003F0B2FBC7
:105E60000121287803F040FD144803F0D9FD2146B4
:105E70002046FFF7C1FF60F07F02D2B20421204626
:105E8000FFF764FF65010C35EDB2022229461E20A2
:105E9000FFF75CFF0134022229461F20FFF756FF5F
:105EA000082CEFD138BD06490648BDE8384002F05D
:105EB0009DBE00BF020000201E0500201406002029
:105EC00048FE0000A005002038B520210546FFF758
:105ED000BAFD000284B221212846FFF7B4FD204418
:105EE00080B238BD70B50E4600243046FFF7ECFF97
:105EF000054618B13046FFF7E7FF0446AC42F4D13F
:105F0000204670BD38B526210546FFF79CFD0002EE
:105F100084B227212846FFF796FD204480B238BD81
:105F200070B50E4600243046FFF7ECFF054618B169
:105F30003046FFF7E7FF0446AC42F4D1204670BD7F
:105F40002DE9F0410E463046242115469846BDF80D
:105F50001870FFF778FD252104463046FFF773FDE2
:105F6000284400EB042084B27101204614313C44E3
:105F70003B464246A4B201F0FC01FFF70FFF220AA4
:105F800024213046FFF76CFDE2B225213046FFF7B1
:105F900067FDBDE8F08107B5009313460022FFF7C7
:105FA000CFFF03B05DF804FBF8B506460F461D466B
:105FB000144632B3144B15480ECB03F047FDFFF7E0
:105FC000B5FE310A114803F04EFDF1B20F4803F05F
:105FD0004AFD39460D480D4F03F045FD6B1E661E08
:105FE0001C44A64206D00021384603F03CFD06F8CA
:105FF000010FF6E7FFF7A2FE044803F033FD284641
:10600000F8BD1546FBE700BF200500201406002060
:1060100082B01046ADF8060049011A46BDF80600E8
:10602000BDF80830183101F0F80102B0FFF7BCBF2D
:106030002DE9F7430E4680462821304691461D46FD
:106040009DF82870FFF7FFFC000284B2292130463A
:10605000FFF7F9FC0444A4B200954B4622463146B2
:106060004046FFF7D5FF5FB92C44A4B2220A28218D
:106070003046FFF7F5FCE2B229213046FFF7F0FC8D
:1060800003B0BDE8F08310B50C4620460121FFF7B0
:10609000E7FC01212046FFF7D6FC0028F9D110BD0E
:1060A000044B4FF000421A6000229A6002221A71DB
:1060B000704700BF20050020142200210E3005F09B
:1060C00042BD10B50E31044602F03CFD204610BD25
:1060D00010B51C31044602F035FD204610BD10B548
:1060E0002031044602F02EFD204610BD10B52831A7
:1060F000044602F027FD204610BD406970478069C4
:10610000704730204B1C0870110902F00F02092A59
:1061100094BF3032373203F801290A460029F3D1FF
:106120007047000007B5002300931A46194603483C
:1061300002F0FCFC03B05DF804FB00BF2C0500205E
:106140002DE9F0418EB004468846164600212022F3
:1061500006A805F0F8FCFF231A461946009302A88A
:1061600002F0E4FC04F15405574B04934322039BD3
:10617000059304A92846FFF76FFB013000F0A180CA
:10618000524B069363688DF821601BBA0793330A5C
:106190008DF820301C22802306A926462846ADF81B
:1061A0002230FFF762FB1A2200210DF11E0005F0DC
:1061B000CAFC56F8080F0690B388ADF81C301022C0
:1061C00006A92846FFF751FB2022002106A805F06A
:1061D000BAFC0627202206A92846FFF746FB013F06
:1061E000F8D13B4B069340F23513ADF81C303D23FC
:1061F0008DF81F3007238DF8203001238DF82130D2
:106200003368CDF82230B388ADF8263031498DF8A7
:106210001E8040F60C430DF12A00ADF8283006F040
:1062200000FCE27A0CA92046FFF76BFF227B0DF100
:1062300032012046FFF765FF627B0DA92046FFF77C
:1062400060FF1E2206A92846FFF70FFBB8F1030FD7
:1062500028D140F23243ADF81830A37B8DF81A30C4
:10626000E37B8DF81B30237C8DF81C30637C8DF82C
:106270001D3040F23643ADF81E3094F824308DF8CE
:10628000203094F825308DF8213094F826308DF8A0
:1062900022300C2294F827308DF8233006A92846A6
:1062A000FFF7E3FA0C4A0D4B06A9CDE90623284671
:1062B000FF2309228DF82030FFF7D7FA2846FFF791
:1062C000D1FA0EB0BDE8F0812C00010001010600FA
:1062D0006382536355FE000037060103060F3A3B05
:1062E0002DE9F0478CB005468846174603F050F973
:1062F00005F1540406462046FFF7FEFA002809DCA3
:1063000003F046F9801B404500F21081322003F073
:1063100059F9F0E7242203A92046FFF7C8FA9DF8AF
:106320000C30022B40F0FD80B5F87030432B40F06C
:10633000F880049E36BA3E60062205F108010AA8DC
:1063400005F0CEFB28B92B689E4202D36B689E42B3
:1063500007D92046FFF763FA002630460CB0BDE8A7
:10636000F087079BC5F80E30CC262046FFF789FA48
:10637000013EFAD1B04605F124092046FFF742FA62
:10638000002840F3CF802046FFF77BFA0F2800F06B
:10639000818025DC032850D00FDC0028EDD00128B7
:1063A00041D02046FFF76DFAC7B2013FFFB2FF2F81
:1063B000E3D02046FFF765FAF7E7062853D00C280C
:1063C000EFD12046FFF75DFAC7B2781C05F066FBF7
:1063D0003A460146A8612046FFF769FAAB6967E0D3
:1063E000362868D00CDC332800F08D803528D8D1D1
:1063F0002046FFF746FA2046FFF743FAC6B2BCE74D
:106400003B2873D0FF28B8D03A28CAD12046FFF7DE
:1064100038FA042205F130012046FFF748FA2B6BC9
:106420001BBA2B63A9E72046FFF72BFA042205F1DC
:106430001C012046FFF73BFA9FE72046FFF721FAB1
:106440000422074605F120012046FFF730FAFFB28B
:106450004FF0000A043F57458FDD2046FFF711FA41
:106460000AF1010AF7E72046FFF70BFA0422074674
:1064700005F128012046FFF71AFAFFB24FF0000A93
:10648000043F57457FF779AF2046FFF7FAF90AF145
:10649000010AF6E72046FFF7F4F9C7B2781C05F0C9
:1064A000FDFA3A46014668612046FFF700FA6B693B
:1064B00003F8078061E72046FFF7E3F96B6A0746B8
:1064C0008BB1494601A802F03DFBEA6E029B9A425D
:1064D00009D0FFB2013FFFB2FF2F3FF44EAF20467D
:1064E000FFF7CFF9F6E704224946A2E72046FFF777
:1064F000C8F9042205F134012046FFF7D8F96B6B87
:106500001BBA6B6339E72046FFF7BBF9042205F19C
:106510002C012046FFF7CBF9EB6A1BBAEB62AB63A9
:106520002BE700262046FFF77AF916E7FF2614E747
:106530002DE9F34704464FF4FA61012002F04BFFC6
:106540002746606047F8540B3846FFF773F944213B
:106550003846FFF7FBF9002800F08B8003F018F8AD
:106560004FF00009804600254FF0030A94F85030A0
:10657000032B1CD02BBB63680133636003F008F866
:106580004FF47A72A0EB08000121B0FBF2F2204632
:1065900092B2FFF7D5FD012384F85030002DE5D1EC
:1065A00002F0F6FF636CA0EB08009842DBD9384696
:1065B000FFF740F9636801336360284602B0BDE825
:1065C000F087042B11D163680133636002F0E0FFB0
:1065D0004FF47A72A0EB08000321B0FBF2F22046E0
:1065E00092B2FFF7ADFD0223D6E7012B19D101AA24
:1065F000A16C2046FFF774FE0228064636D1019BA7
:10660000636002F0C5FF4FF47A72A0EB080003212B
:10661000B0FBF2F2204692B2FFF792FD84F8506090
:10662000BCE7022BBAD101AAA16C2046FFF758FEA5
:106630000528064615D1E36A84F850A013B94FF433
:106640006173E362236B13B9E36A5B082363D4E9E4
:106650000C320AB95A006263A363636BE3630125DA
:1066600084E7062802D184F8509097E7FF2EFAD0ED
:1066700094E70546A1E7F8B500250F460446C0E9B2
:106680000B554563C0E91052836485608581FFF72F
:1066900013FD3B68A360BB88A38184F8505020465B
:1066A000BDE8F840FFF744BF38B5044602F070FF7C
:1066B0000546206C00283ED0E26CA91A17D44FF48E
:1066C0007A7005F57A7291FBF0F300FB1311521A00
:1066D0000133E264A26B59008A42ACBFD21A002295
:1066E000A263E26B9142CCBF0023D31AE36394F818
:1066F0005030032B1DD1A36B002B1ADC042384F82C
:1067000050302046FFF714FF013094F85030032B2F
:1067100000D063B9E36B002B09DC002384F8503010
:106720002046FFF7C9FC2046FFF702FF033025642F
:1067300038BD0020E9E705F57A73E364F7E74B68B5
:10674000436000230381704730B50139084610F8D3
:10675000013F002BFBD11C460A2511F8010F70B137
:10676000032C14DC2E2806D1FF2B10DC1019013469
:1067700003710023F1E7303805FB0303EDE7FF2B3E
:1067800004DC032C02DC22440120137130BD002004
:10679000FCE7000007B5002300931A46194603489A
:1067A00002F0C4F903B05DF804FB00BF340500201B
:1067B0002DE9F74305460E4602F0EAFE05F10C040A
:1067C000288105F10801022202AD2046FFF74DF8AD
:1067D000012325F8023D022229462046FFF745F80D
:1067E0004FF48073022229462046ADF80630FFF7A9
:1067F0003CF80023022229462046ADF80630FFF778
:1068000034F8022229462046FFF72FF802222946B3
:106810002046FFF72AF837463378E3B13E46B046C4
:1068200018F8013B0BB12E2B13D1A6EB0709B9F1D8
:10683000000F0CDD01220DF1050120468DF80590B9
:10684000FFF713F84A4639462046FFF70EF8474649
:10685000E2E74646E3E702A9012201F8033D2046AC
:10686000FFF703F84FF48076294602222046ADF860
:106870000660FEF7FAFF022229462046ADF80660C0
:10688000FEF7F3FF012003B0BDE8F0832DE9F043EC
:1068900087B006460F46904602F07AFE06F10C04D9
:1068A00005462046FFF728F800280BDC02F070FEB2
:1068B000401BB84200F2EA80322002F083FEFCF76F
:1068C000DDFBEEE7726A73689A4240F0E280338D36
:1068D000352B40F0DE802046FEF794FF0B2840F376
:1068E000DB800C220DEB02012046FEF7E0FFBDF835
:1068F0000E203189130A43EA0223BDF80C201BB293
:106900009DB29142ADF8065001D1002B07DB204625
:10691000FEF785FF4FF6FC7007B0BDE8F08340F24C
:106920000F231D4005D02046FEF779FF4FF6FB7080
:10693000F2E7BDF812301F0A47EA0327BFB2AFB92A
:106940002046FEF76CFF4FF6FA70E5E79DF80A3037
:106950009BB92046FEF795FF2046FEF792FF2046A2
:10696000FEF78FFF2046FEF78CFF0135BDF8103093
:106970005BBAAAB29BB29A4214DA01220DF10A0163
:106980002046FEF794FF9DF80A30002BDED09DF8DC
:106990000A305A1E8DF80A20002BD7D02046FEF769
:1069A00070FFF4E70026B14601220DF105012046F3
:1069B000FEF77DFF9DF8053013F0C00F0AD193B1AB
:1069C0009DF805305A1E8DF8052043B12046FEF78C
:1069D00058FFF5E72046FEF754FF8DF805909DF827
:1069E0000530002BE0D1022202A92046FEF75FFF0E
:1069F00002220DF10A012046FEF759FF2046FEF75C
:106A000040FF2046FEF73DFF2046FEF73AFF2046B6
:106A1000FEF737FF02220DF106012046FEF747FF81
:106A2000BDF80830B3F5807F18D1BDF80A0040BA30
:106A300085B2012D12D1BDF8062052BA92B2042AB5
:106A400005D02046FEF7EBFE4FF6F77064E708F13D
:106A500004012046FEF72BFF28465DE70025BDF820
:106A600006305BBAAAB29BB29A4205F1010503DA7D
:106A70002046FEF706FFF2E70136B6B2B74293D1E1
:106A80002046FEF7CCFE4FF6F67045E74FF6FF7056
:106A900042E74FF6FE703FE74FF6FD703CE700001F
:106AA0002DE9F341054688461746FFF74DFE04469B
:106AB00000283BD1204B6A685B689A4238D002F0CC
:106AC00067FD05F10C0600F00F0101F5806130460D
:106AD000FEF73CFF01281CD1184B009335226B6850
:106AE000019369463046FEF7B7FE78B14146284625
:106AF000FFF75EFE50B13046FEF7B4FE30B13A46C5
:106B000041F288312846FFF7C1FE04463046FEF7C1
:106B100091FE0B490B4802F052F80A22214609481F
:106B200002F0AFF8204602B0BDE8F0810124F9E799
:106B30006FF00104F6E700BF340500202C000100CF
:106B40005CFE0000A0050020006903681B6918476F
:106B5000006903685B69184713B5006949680368F1
:106B6000034C01919B6900946946984702B010BD9F
:106B70002C00010000690368DB691847006903689D
:106B80009B6A18470069003018BF01207047006CED
:106B900070470164704710B590F83830044633B937
:106BA00020690368DB689847002808DA10BD03688D
:106BB0009B6898470028F3D14FF0FF30F6E794F830
:106BC0002220A2F10803022BF0D8A36A002BC2BF37
:106BD000E36A0133E3620A2AE8D1E36B013BE36332
:106BE000002BE3D1092384F82230DFE710B50446F7
:106BF000006903681B6A984794F82230083B022B0F
:106C000007D8A36A002B04DD0028A2BFE36A1B1883
:106C1000E36210BD73B590F82230092B04460ED103
:106C20000026206903689B68984740B12069036883
:106C3000DB689847C5B20A2D1CD184F8225094F81D
:106C400022300A2B04D1E36B13B9092384F82230D4
:106C500094F82230092B22D0206903689B6898475A
:106C600094F822300A2B03D1E36B9842A8BF184650
:106C700002B070BD0D2DD4D0284604F0F5FE0028DA
:106C8000CFD0E06BADF8046010228DF804500021E5
:106C9000050101A806F022F82844E063C1E70020BE
:106CA000E6E7000000234FF0FF32C0E90A23084A5C
:106CB00080F8223012680263064A4362126880F844
:106CC0003830C36347F2305342630364704700BFF8
:106CD000080000200C00002038B504461D460020A6
:106CE0004FF47A73C4E901030B4B2360C4E9041227
:106CF00004F1180001F012FF0123258484F84430C8
:106D000084F84530054904F1480002F0CCFB2046E8
:106D1000FFF7C8FF38BD00BFC0FE00009AFF0000AB
:106D200010B50446006903685B6A98472046BDE8D1
:106D30001040FFF7B7BF012380F8223070470000F2
:106D400038B504460069154601F039FF0449206949
:106D500001F035FF29462069BDE8384001F046BF03
:106D60009FFD000038B504460D460069114601F04C
:106D700026FF1D49206901F022FF2946206901F004
:106D80001EFF1A49206901F031FF94F84530F3B134
:106D90006369B3B11649206901F011FFD4E9040118
:106DA00001F00DFF238C502B08D01249206901F00F
:106DB00006FF0A22218C206901F061FF206901F0A1
:106DC00005FF0D4B0D491A682046FFF7B9FF94F8EF
:106DD000443023B10A4A0B492046FFF7B1FF012393
:106DE00084F82230002038BD85FE000087FE0000B8
:106DF00091FE0000F9F600000400002098FE00005B
:106E0000A3FE0000A9FE000038B50446006915463F
:106E100001F0D5FE0549206901F0D1FE294620691F
:106E20000A22BDE8384001F02CBF00BF9FFD0000E2
:106E300010B50446006901F0C9FE022384F822302F
:106E400010BD70B590F82230012B04460D46164651
:106E500001D8FFF7EDFF20690368324629465B68D9
:106E6000BDE87040184770B590F82230012B0446F9
:106E70000D4601D8FFF7DCFF2069036829461B682F
:106E8000BDE87040184710B50446206903689B6848
:106E9000984720B120690368DB689847F5E710BD83
:106EA0002DE9F347994690F82230083B022B04461F
:106EB0000E469246DDE90A7804D8FFF7E4FF204643
:106EC000FFF7F0FE94F82250012D44D894F8443096
:106ED00063B1D4E90401228C0368002934D121492B
:106EE0000091E16901919B6969462EE02069036880
:106EF0009B6A98470028ECD0314652462046FFF75F
:106F000031FF0646E0B9B9F1000F04D04A461649F0
:106F10002046FFF715FF002F20DD3A461349204693
:106F2000FFF772FFB8F1000F18D001252046FFF7D8
:106F30007FFF2DB123683A465B684146204698475B
:106F4000304602B0BDE8F087DB6998470028D3D10E
:106F50004FF0FF36F4E76FF00106F1E7002DEFD1B7
:106F6000E4E700BF2C00010061FE00006EFE00009F
:106F700090F82230012B01D8FFF75ABF7047FFF776
:106F8000F7BF000007B500234FF0FF32CDE9002323
:106F9000024AFFF785FF03B05DF804FBB4FE000072
:106FA0002DE9F04790F82230012B044651D9DFF843
:106FB000D8800025032700236362022384F822304F
:106FC00002F0E6FA464682464FF00A090A2D46D0FC
:106FD00002F0DEFA236CA0EB0A00984245D2236847
:106FE00020469B68984748B323682046DB6898474B
:106FF000431C0546ECD094F82230022B05D0032B1D
:107000000FD002F0C5FA8246E0E733782A2B01D090
:1070100083421AD17278731C0AB984F822701E4612
:10702000EFE7A0F13002092A95BF636A042309FB48
:10703000032384F8223098BF6362E2E74FF47A704A
:1070400002F0C0FAC2E70A2D06D16FF00300BDE8D6
:10705000F0876FF00100FAE76FF00200F7E7636A6C
:10706000C72B02DC652B18BF002594F82230042BB7
:10707000E9D1606AC72801DC65289CD10A2D18BFB8
:107080006FF00200E3E700BF7DFE000010B503686B
:107090000446DB68984794F82230A3F10802022ADC
:1070A000C0B232D9052B31D0072B39D0042B54D1A3
:1070B000226B137883420BD1531C2363537823B97B
:1070C000C4E90A33052284F822200A281DD136E0BB
:1070D000636B197881420BD15A1C62635B78002B79
:1070E000F3D1012384F83830062384F82230ECE70A
:1070F0001B4909688A42F7D11A4A12689342F3D1B0
:107100000D28F1D1072384F8223010BDA0F1300200
:10711000092AE9D8A36A0A2101FB0323A362D4E761
:107120000A28F2D194F838309BB1092384F8223030
:107130000023E36394F82230083B022BE5D90423B3
:1071400084F82230064B1B682363064B1B6863637D
:10715000DBE7082384F82230ECE70A28D5D1E9E7F9
:10716000080000200C00002038B5044602F010FA98
:10717000054694F82230083B022B13D902F008FA96
:10718000236C401B98420DD2236820469B68984789
:1071900018B12046FFF77AFFE8E74FF47A7002F063
:1071A00011FAE6E794F82230083B022B94BF002046
:1071B0006FF0020038BD10B590F82230083B022B6A
:1071C000044601D9FFF7D0FFA06A10BD7FB5054680
:1071D00008460E46FFF7EFFF1649044601A802F0E5
:1071E00062F9002C0EDD214601A802F035F948B9FC
:1071F0000021284602F057F901A802F00FF92846AD
:1072000004B070BDF36AA34209D0304601F066FFB6
:10721000431C04D0C1B201A802F0ACF9E7E7002C8E
:1072200002DD039B9C42E3D101A9284602F0E7F866
:10723000E2E700BF9AFF000038B590F82230083B23
:10724000022B054601D9002038BDFFF7B4FF0130FD
:10725000F9D02846EC6AFFF7AEFF8442B4BF0020A5
:107260000120F1E7FFF7E8BFFFF7E6BF07B500230E
:1072700000931A461946034801F058FC03B05DF824
:1072800004FB00BF3C05002000B55DF804FB0020B6
:10729000704700B501205DF804FB80687047C1604D
:1072A00070472DE9F84380460D46174601EB020969
:1072B0000C46A145A4EB050609D0D8F8003040469D
:1072C000DB689847431C03D004F8010BF1E73E4606
:1072D0003046BDE8F883C368013304D180690030CB
:1072E00018BF012070470120704743696BB1C26924
:1072F000012A0AD95A1C42611970C369013BC36152
:10730000436900221A700120704700207047000076
:1073100010B5D0E904435A1C42610A460248E118FC
:10732000FFF7B7FF012010BDD0020020C368013372
:1073300010B504460ED16369B3F5FA4F0EDA23682F
:107340002046DB689847202806DD2368C1B25B69C8
:1073500020469847012002E00130ECD1002010BD0A
:107360000346C068421C03D04FF0FF32DA6070471A
:10737000196931B19A6922B1481C1861013A08783B
:107380009A61704708B50346C068421C03D04FF0AD
:10739000FF32DA6008BDD3E90412501C5861114471
:1073A0000148FFF774FFF5E7D00200200368FF21D2
:1073B0001B68184710B5182004F070FB044618B17C
:1073C0001822002104F0BFFB204610BD70B5064610
:1073D0000C46CCB194F910306568002B04DBE168F1
:1073E00011B13046FFF7F2FF237C042B03D1606913
:1073F00008B104F05BFB206808B104F057FB20469D
:1074000004F054FB2C46E4E770BD00002DE9F04F7A
:10741000036885B0DB6805460E469847421C044663
:1074200004D14FF0FF3005B0BDE8F08F2D282FD1EB
:107430002B682846DB689847431C0446F1D04FF080
:10744000FF330093A4F13003092B4FF000070DD850
:107450004FF00A082B682846DB689847A0F13003F4
:10746000303C092B08FB07470446F3D92E2C11D0DA
:1074700024F02003452B0DD0009B7B437361022336
:1074800033742B6828465B69E1B298470020CAE74D
:107490000123D6E7384603F037FD2E2C8046894677
:1074A00039D12B68DFF814B1DB68284698470027EC
:1074B00004464FF0000A52465B464046494603F0F8
:1074C0008DFD80468946A4F1300003F01DFD424643
:1074D0004B4603F0CDFB2B688046DB682846894687
:1074E0009847A0F13003092B07F1FF370446E2D992
:1074F00024F02003452B2AD12B682846DB689847C7
:107500002B28044609D12B682846DB689847044697
:107510004FF0010A0AE00027EAE72D28F8D12B688E
:107520002846DB6898474FF0FF0A04464FF0000BEF
:107530000A22A4F13003092B0DD802FB0B3B2B6868
:107540000392DB6828469847039A0446F1E74FF018
:10755000010A4FF0000B009803F0D6FC42464B4660
:1075600003F03CFDCDE90001584603F0CDFC804618
:107570005046894603F0B8FC02460B464046494651
:1075800003F02CFD80463846894603F0BDFC0246D8
:107590000B464046494603F06BFB02460B46002073
:1075A000064902F089FA0B460246DDE9000103F0C4
:1075B00015FD04F00BF80323706161E7000024401F
:1075C00019B10A22496901F038BB0846704700002A
:1075D000F8B506462DED028BD1B391ED058A18EE74
:1075E000100A03F0A3FCB5EEC08AF1EE10FA0446CF
:1075F0000D4606D51A49304601F0E1FA05F100437F
:107600001D462946204603F0C1FF0A2201460746CF
:10761000304601F040FB1349304601F0D0FA3846BD
:1076200003F062FC02460B462046294603F01EFB8F
:1076300009A3D3E9002303F01BFB00220A4B03F04C
:10764000CDFC03F0A3FF0A220146304601F03CFBCB
:10765000BDEC028B0020F8BD9A9999999999A93FA0
:107660003B0401006CF9000000002440F8B50368F9
:10767000DB6806460F469847222803D04FF0FF34B8
:107680002046F8BD04233B7400F008FB05460028A3
:10769000F4D033683046DB689847431C044611D069
:1076A000222C36D01F2C34DD5C2C04D02946E0B2CD
:1076B00000F00AFBEDE733683046DB689847421C70
:1076C000044603D1284600F027FBD9E7622817D0EB
:1076D00007DC2F2803D05C2801D02228D9D12946E5
:1076E000E6E76E280FD004DC6628D2D129460C20AC
:1076F000DEE772280AD07428CBD129460920D7E7C3
:1077000029460820D4E729460A20D1E729460D203A
:10771000CEE7284600F0E4FA00247861B0E70000E4
:1077200038B50D461D49044601F049FA7DB3013DC7
:1077300015F8011F59B31F2907D9222905D05C2943
:1077400003D0204601F03FFAF2E75C21204601F029
:107750003AFA29780C2914D007D8092915D00A2912
:1077600011D00829E4D16221EBE72229E9D003D81E
:107770000D29DDD17221E4E72F29E2D05C29E0D088
:10778000D6E76621DDE76E21DBE77421D9E7222108
:10779000204601F018FA002038BD00BF4AFF000063
:1077A0004969FFF7BDBF0368DB6810B50446984719
:1077B000431C0AD02028236802DCDB682046F6E759
:1077C000C1B25B6920469847002010BD03682DE9CF
:1077D000F047DB6804468846914698477B2803D0EB
:1077E0004FF0FF30BDE8F087062388F810302046C0
:1077F000FFF7D9FF23682046DB6898477D2843D0F0
:107800002368C1B25B6920469847FF264FF0000A03
:10781000FFF7D0FD05460028E2D096B3C8F80C006B
:107820002046FFF7C0FF29462046FFF71FFF013023
:10783000D6D02046FFF7B7FF6B692B602368C5F8E9
:1078400014A0DB68204698473A28C9D12046FFF7A4
:10785000AAFF4A462946204600F018F80130BFD05A
:107860002046FFF7A0FF23682046DB6898472C28B6
:107870002F464FF00006CBD07D3818BF4FF0FF30B9
:10788000B0E778608760CBE70020ABE7F7B5044648
:107890000E461746FFF787FF013002D14FF0FF3049
:1078A00011E023682046DB689847431C0546F5D065
:1078B0002368C1B25B6920469847222D05D1314625
:1078C0002046FFF7D3FE03B0F0BD2D2D03D0A5F168
:1078D0003003092B04D831462046FFF797FDF2E725
:1078E0005B2D05D13A463146204600F095F8EAE78F
:1078F0007B2D05D13A4631462046FFF767FFE2E788
:107900006E2D15D102AD002345F8083D23680422F1
:107910001B6929462046984704280246BED11D49C6
:10792000284605F0BEF80028B8D100233374CAE712
:10793000662D16D1002300938DF8043023680522AC
:107940001B696946204698470528A7D10522124998
:10795000684605F0A6F80028A0D1012333743075DD
:10796000B1E7742D9AD102AD002345F8083D236894
:1079700004221B69294620469847042802468DD1D7
:107980000649284605F08DF8002887D10123337475
:10799000337598E73AFF00003FFF000045FF000005
:1079A000F8B5064617460D4611B900242046F8BD25
:1079B000FFF700FD04460028F7D02846FFF7F3FE46
:1079C0003A4621462846FFF761FF0130EED12146B5
:1079D0003046FFF7FBFCE8E70022FFF7E1BF0000BD
:1079E00010B588B04FF0FF3200230392094A00928D
:1079F0000446CDE901330846CDE90413079309B1E4
:107A000005F033F8069069462046FFF7E5FF08B019
:107A100010BD00BF78FF00002DE9F8430368DB6864
:107A200004468846914698475B2803D04FF0FF30C4
:107A3000BDE8F883052388F810302046FFF7B3FE31
:107A400023682046DB6898475D282AD02368C1B2A6
:107A50005B6920469847FF26FFF7ACFC05460028E7
:107A6000E4D0DEB1C8F80C002046FFF79CFE4A4681
:107A700029462046FFF70AFF06460028D6D12046B1
:107A8000FFF791FE23682046DB6898472C282F4695
:107A9000E2D05D3818BF4FF0FF30C9E778608760EB
:107AA000E2E70020C4E738B5054651B3CC687B2136
:107AB00001F089F8013002D14FF0FF3038BDB4B188
:107AC00021682846FFF72CFE0130F5D03A212846E0
:107AD00001F079F80130EFD02146284600F014F883
:107AE0000130E9D0646814B12C212846E0E77D21FB
:107AF000284601F068F801304FF0FF3018BF002031
:107B0000DCE70846DAE70000D9B10B7C062B18D871
:107B1000DFE803F004070D0F111315000A4901F007
:107B20004EB80B7D0BB10949F9E70949F7E7FFF7B3
:107B300047BDFFF74DBDFFF733BE00F00EB8FFF7AE
:107B4000B2BF0020704700BF3AFF000045FF0000B1
:107B50003FFF00001046FFF7D7BF38B50546F1B12B
:107B6000CC685B2101F02FF8013002D14FF0FF30DB
:107B700038BD54B121462846FFF7C6FF0130F5D085
:107B8000646814B12C212846ECE75D21284601F0F9
:107B90001AF801304FF0FF3018BF0020E8E7084620
:107BA000E6E7CB680022D0B201320BB15B68FAE79E
:107BB0007047C86820B11AB1013AD2B24068F9E7FB
:107BC000704738B5CC68154634B12946206804F0B2
:107BD000E4FE08B16468F7E7204638BD4AB1CB68D7
:107BE00013B9CA6070470B4659680029FBD15A6027
:107BF00093607047F8B505460E4617461C4673B1AC
:107C0000186808B103F052FF384604F013FF22460B
:107C1000206031462846BDE8F840FFF7DFBFF8BDD9
:107C200010B50C46FFF7C6FB10B102230374446184
:107C300010BDD0B516461F46FFF7BCFB044630B159
:107C4000032303743946304603F0C0FC60612046CC
:107C5000D0BD08B5FFF7AEFB08B10523037408BD1E
:107C600070B50D46194604461646FFF7D9FF324651
:107C7000034629462046BDE87040FFF7BBBF000021
:107C800007B5002300931A461946034800F04EFF3B
:107C900003B05DF804FB00BF4405002038B50C209C
:107CA00003F0FCFE044650B1064820604FF4807596
:107CB0002A46002103F047FF00236560A3602046A9
:107CC00038BD00BF40060020D1E90123934204D211
:107CD0000A68D0548B6801338B6000207047000025
:107CE000826838B5044622B10368134413F8013C96
:107CF0001BB121460020FFF7E7FFA06803F0CEFE8E
:107D0000054628B1034904F08CFE204603F0CEFE60
:107D1000284638BD4006002008B103F0C7BE7047B2
:107D200010B5054C204600F051FF20460349BDE840
:107D3000104000F03BBF00BFA005002094FF0000F2
:107D4000F0B503789FB0044643B3194B194F1B6835
:107D5000986803F077FD2046164904F0DDFE1EAD5D
:107D6000012445F8780D3946002004F0D5FE1E2C7C
:107D7000264645F8240002D001340028F3D10E4BEA
:107D8000009F1C6874B12168384604F040FE38B981
:107D90006368294630469847FFF7C2FF1FB0F0BD21
:107DA000A468EFE70549064800F016FFF4E700BFB6
:107DB0003000002085FE0000900500209BFF0000A1
:107DC000A0050020F8B505460C200F4603F066FE1E
:107DD0000C4B04461860284604F047FE013003F0BF
:107DE0005DFE2946064604F01CFE284604F03DFED2
:107DF00000233354044B1A68A260C4E900671C6076
:107E0000F8BD00BF900500205005002070B5164851
:107E1000164D01F0C1F9C4B20A2C0CD00D2C0AD0B9
:107E2000082C15D12146104800F0CDFE2B7873B1F7
:107E3000013B2B700BE02B780D4E0E490A480024B5
:107E4000F45400F0BCFE3046FFF77AFF2C7070BD92
:107E50002146054800F0B7FE2B783A2B9FBF5A1CED
:107E60002A70034AD454F2E7A005002094050020AC
:107E70005405002098FF000010B5044C204601F086
:107E800085F910B1FFF7C2FFF8E710BDA00500208B
:107E9000044A00231370044A01460448136001F0A9
:107EA00034B900BF9405002050050020A005002033
:107EB00070B504460D4601F06BFBC4F89000A06855
:107EC000036829461B68BDE87040184770B5044632
:107ED0000D46164601F05CFBC4F89000A0680368EC
:107EE000324629465B68BDE87040184770B5094BBB
:107EF00000250446456040F8A03B0E4600F00EFE0B
:107F00004FF0FF33C4F8B430A660C4F8B050204638
:107F100070BD00BFB4FF00002DE9F04105460E46DC
:107F200001F036FB43F697278046A86803689B68F4
:107F30009847044648B901F067FB01F029FBA0EB24
:107F40000800B842F1D9204605E0A8680368DB685C
:107F5000984730700120BDE8F08138B5148821447D
:107F60001546FFF7D9FF08B101342C8038BD2DE943
:107F7000F74F02AD002725F8027D00F10C068A4676
:107F80002A4631460446FFF7E8FF18B9002003B03F
:107F9000BDE8F08F0DF1080994F80C8009F8037D15
:107FA0004FF0010BBDF80630052B08D14FF0FF3321
:107FB000A068C4F8B43003685B6A9847E6E74946AE
:107FC0002046FFF7A9FF0028E0D0BDF806209DF865
:107FD0000510531C22449BB2117301F07F0212FB67
:107FE0000BF217440A06ADF80630BFB24FEACB1BBE
:107FF000D8D408F0F008013BB8F1300F8AF800300F
:108000001CD12A4631462046FFF7A7FF0028BDD0E5
:108010002A4631462046FFF7A0FF0028B6D09AF83E
:10802000003023445A7B9E7B237B06EB02269B0772
:10803000B6B201D50236B6B2022501E000252E46C1
:10804000ADB2BD4225D249462046FFF765FF002864
:108050009CD0D4F8B00078B1B8F1300F0CD1BDF895
:1080600006309AF800209B1A023BB34204DD0368F5
:108070009DF805101B689847BDF806307F2B9EBF02
:10808000E2189DF8051011730133ADF80630013583
:10809000D6E7D4F8B0302BB9BDF80620802A88BFC7
:1080A000ADF80630BDF8060071E737B500240DF1D4
:1080B000080C03F07F05601CDB09644418BF45F021
:1080C0008005C0B204F8045C0446002BEFD1C0F177
:1080D000040401AD1155984205DD191A11445C5D87
:1080E0004C710133F7E7013003B030BDF8B50646F7
:1080F00017461C46FFF7D9FFB368C0B21A6804449C
:10810000C0F105015568394422461846A84705467E
:1081100001F03EFAC6F89000A8B2031B584258413D
:10812000F8BD10B5E023044683818068036802220D
:1081300004F10C015B689847A0684FF0FF33C4F866
:10814000B43003685B699847A06803685B6A984726
:1081500001F01EFAC4E9240010BD023330B598B214
:108160000C46631A14F8015B9BB21DB1431C1554F5
:1081700098B2F6E7C11A0A44191202F8021C02F872
:10818000013C30BD38B50546806808B9002038BDCF
:1081900003689B6A984780B9D5F8B440002CF5D1A4
:1081A000A8686FF00203C5F8B43003685B699847AC
:1081B000A86803685B6A9847E8E70120E7E70000E2
:1081C0002DE9F04F85B00446894617461E460E9DA0
:1081D0009DF848A0FFF7D6FF8046002840F0CE80EB
:1081E000A068D4F8A8100368B4F8AC2000293FD0E8
:1081F000DB699847012840F0C880664B029345F23E
:108200005443ADF80C300423A4F88C008DF80E30E4
:1082100004F11102002302A8195C02F8011B0133CA
:10822000072BF9D165B39DF840309DF83C205B01E8
:1082300043F0040343EAC203DBB2BAF1000F01D0FA
:1082400043F0020317B1EEB943F0800323764FF0F9
:108250000F0B0023637684F81AB0484604F005FC3F
:108260001130802811D9A06803685B6A984785E0BF
:1082700049499B690291D4F8A410039102A9B8E777
:108280002B46DAE743F0C003E0E704F10C0A494665
:108290005B4652462046FFF760FF8146E5B128461F
:1082A00004F0E3FB09F1020318448028DBD82946D7
:1082B0004B4652462046FFF750FF0546119804F002
:1082C000D4FB023028448028CDD82B465246119941
:1082D0002046FFF742FF8146F7B1384604F0C5FB60
:1082E00009F1020318448028BDD84B46524639464E
:1082F0002046FFF732FF814676B1304604F0B5FBE9
:1083000009F1020318448028ADD84B465246314645
:108310002046FFF722FF8146A9F105039BB2524692
:1083200010212046FFF7E2FE01F032F9C4E92400F3
:1083300043F69725A06803689B68984758B901F0F1
:1083400027F9D4F89430C01AA842F3D96FF0030388
:10835000C4F8B43087E70DF107012046FFF707FEA8
:10836000042880D1E57B6DB901F012F94FF00108C6
:10837000C4F8940084F89850C4F8B450404605B04E
:10838000BDE8F08FC4F8B4506DE76FF00103C4F896
:10839000B430F3E700044D512C00010010B586B055
:1083A000012404940B9C03949DF8284002949DF8AA
:1083B00024400194089C0094FFF702FF06B010BD12
:1083C0002DE9F74F0446FFF7DDFE8146D8B101F0F5
:1083D000DFF8D4F8943043F69822C31A93428046CB
:1083E00004D8D4F89030C31A93421DD994F8983029
:1083F000A06863B16FF00303C4F8B43003685B6A2C
:1084000098474FF00009484603B0BDE8F08F214679
:10841000C02321F80C3F036802225B689847C4E937
:108420002488012384F89830A06803689B689847E3
:108430000028E8D00DF107012046FFF798FD05461A
:10844000002867D0237BC4F8948003F0F003302B1E
:108450004DD1D4F89C30002BD5D09DF80760B31CCB
:1084600004EB030BA2199BF80C70517B04F10C0A6E
:1084700007EB0127BFB25344F11C3A46514418465A
:10848000BB4403F047FB00228BF80C20217BAA1B86
:1084900001F00601033A022906F103010346A2EBAB
:1084A0000702D4F89C5039441ED12144023A087B7B
:1084B00091F80DB0711D39440BEB002B5144184657
:1084C000A8471FFA8BFB4FF41073A381A06884F8B0
:1084D0000FB04FEA2B23A373036804225B68514655
:1084E0009847C4F890808EE75144A8478BE7C02B8B
:1084F00009D1D023A068A381036802225B6804F13C
:108500000C0198477FE7D02B7FF47DAF002384F8E0
:10851000983078E72046FFF735FE002808BF4FF077
:10852000000970E72DE9F0470446894690461E464B
:108530009DF82070FFF726FE40B3484604F095FAF8
:10854000F31D1844802821D804F10C052A46052380
:1085500049462046FFF701FE002291B283188E4261
:108560009BB202F1010204D9234418F801101973D7
:10857000F3E7002FA3F105032A4620469BB20CBF68
:1085800030213121BDE8F047FFF7B0BD0020BDE844
:10859000F08773B5054610460E46144604F065FA9A
:1085A000002300932246034631462846FFF7BAFFD0
:1085B00002B070BDF7B5054610461F460E4614467C
:1085C00004F053FA00970346224631462846FFF747
:1085D000A9FF03B0F0BD012A2DE9F04104460F4682
:1085E00016462AD8084604F040FA0930802824D8D4
:1085F0002046FFF7C7FD00B3B4F88C3001339BB2BF
:10860000CBB1A4F88C30B4F88C30A3741A1204F1F6
:108610000C05627439462A4607232046FFF79DFD64
:1086200023182A461E73031F9BB220468221BDE8F1
:10863000F041FFF75BBD0123E3E70020BDE8F081D7
:108640000022FFF7C8BF70B5044608460E4604F086
:108650000CFA0930802822D82046FFF793FDF0B1AC
:10866000B4F88C3001339BB2BBB1A4F88C30B4F8B1
:108670008C30A3741A1204F10C05627431462A4638
:1086800007232046FFF769FD431F2A4620469BB279
:10869000A221BDE87040FFF729BD0123E5E70020D6
:1086A00070BDC0F8A810A0F8AC207047C0F89C10AE
:1086B0007047D0F8B400704707B5002300931A46FE
:1086C0001946034800F032FA03B05DF804FB00BF1E
:1086D000980500208271054A417112680449B2FB75
:1086E000F1F14FF47A724A43C260704710000020E3
:1086F00040420F0038B504460D464079022101F092
:10870000F3F800F045FFA0F5FA60A060657438BD8D
:1087100070B505460E460024687901F01FF9B04295
:10872000A3B206D1EA689A4204F10104F4D84FF0EA
:10873000FF33184670BD30B50D46D1B0044600F089
:1087400027FF3DB9A368C31AB3F5FA6F02D2207CA4
:1087500051B030BD00250221A060256060792571EF
:1087600001F0C2F8012000F02DFF0121607901F035
:10877000BBF82946607901F0DFF8A379153B012B9E
:1087800000F28C8040F24C40013800BF00BF00BFB7
:1087900000BF00BF00BF00BF00BF00BF00BF00BFE1
:1087A00000BF00BF00BF00BF00BF00BF00BF00BFD1
:1087B00000BF00BF00BF00BF00BF00BF00BF00BFC1
:1087C00000BF00BF00BF00BF00BF00BF00BF00BFB1
:1087D00000BF00BF00BF00BF00BF00BF00BF00BFA1
:1087E00000BF00BF00BF00BF00BF00BF00BF00BF91
:1087F00000BF00BF00BF00BF00BF00BF00BFC3D1AC
:108800006079022101F070F8607C00283BD00138CB
:1088100000BF00BF00BF00BF00BF00BF00BF00BF60
:1088200000BF00BF00BF00BF00BF00BF00BF00BF50
:1088300000BF00BF00BF00BF00BF00BF00BF00BF40
:1088400000BF00BF00BF00BF00BF00BF00BF00BF30
:1088500000BF00BF00BF00BF00BF00BF00BF00BF20
:1088600000BF00BF00BF00BF00BF00BF00BF00BF10
:1088700000BF00BF00BF00BF00BF00BF00BF00BF00
:1088800000BF00BFC3D172B600212046FFF740FFF2
:10889000013007D10020207462B659E7142000F09F
:1088A00091FEADE701212046FFF732FF0130F1D004
:1088B000002500212046FFF72BFF01214DF8050080
:1088C0002046FFF725FF0DEB05030835B5F5A07F22
:1088D0005860EED162B600225DF832500DEBC20353
:1088E000691C586801D0431C02D1002020742FE776
:1088F000D1108542635C4FEA4303DBB202F101020F
:1089000038BF43F00103282A6354E5D16178237806
:1089100022790B44A1780B44E1780B44DBB29A42F4
:10892000E3D10120E2E700002DE9F8430D462DEDEB
:10893000028B11460446FFF7FEFE00287ED0A37985
:108940000B3B0B2B7AD8DFE803F0063F7979797976
:10895000797979796565A378E07808EE103A0106AF
:10896000B8EE488A48BFFFEE007A00F00F0048BF1B
:1089700037EEC88A02F0C8FA31A3D3E9002302F027
:108980002DFB064618EE100A0F4602F0CFFA0B46F2
:1089900002463946304602F06BF902F017FE0346F4
:1089A0006DB102F0C3FA2AA3D3E9002302F016FB4B
:1089B000254B002202F05CF902F008FE0346BDECF4
:1089C000028B1846BDE8F883E078A67800F00F0027
:1089D00002F09AFA1AA3D3E9002302F0FFFA07EE95
:1089E000906AF8EE677A804617EE900A894602F0A0
:1089F0009DFA02460B464046494602F039F902F01C
:108A0000E5FD3206034648BF80F00043002DD6D076
:108A10001846C6E7A678E378300200F4FE40184313
:108A200007EE900AF8EEE77A17EE900A02F07EFA67
:108A300003A3D3E9002302F0D1FAE0E7034BBEE73A
:108A40009A9999999999B93F000040400000C07FD8
:108A5000CDCCCCCCCCCCFC3FD0B50446FFF76BFEE4
:108A600090B3A3790B3B0B2B2ED8DFE803F006065F
:108A70002D2D2D2D2D2D2D2D1C1C607802F044FA4E
:108A800014A3D3E9002302F0A9FA064620780F4682
:108A900002F03AFA02460B463046394602F0E8F850
:108AA00002F094FDD0BD208840BA80B207EE900A53
:108AB000F8EEE77A17EE900A02F038FA05A3D3E948
:108AC000002302F08BFAEBE70148EBE7AFF30080FD
:108AD0000000C07F9A9999999999B93F2DE9F84377
:108AE00006460D46071D00F10709002417F8011B73
:108AF0000A22284600F0DCF82E218046284600F0A5
:108B000062F84F4540440444F0D10A22F1792846E6
:108B100000F0CEF82044BDE8F8830000024A02606D
:108B200000224260704700BF2C00010030B5837105
:108B3000034D9DF80C30056001714271C37130BD69
:108B40002C000100024A02600A684260704700BFC0
:108B50002C0001000B68436070472DE9F041064688
:108B60000D4601EB02080C464445A4EB050707D06F
:108B7000336814F8011B1B68304698470028F3D16E
:108B80003846BDE8F08170B5044608460D4603F04E
:108B90006CFF23680246294620465B68BDE87040AA
:108BA000184709B1FFF7EFBF0846704708B5FFF750
:108BB000F8FF08BD03688A685B680968184708B54C
:108BC000FFF7EFFF08BD03681B6818470149FFF76F
:108BD000DABF00BF98FF000038B50546FFF7E1FF98
:108BE00004462846FFF7F2FF204438BD38B5054655
:108BF000FFF7D7FF04462846FFF7E8FF204438BDBB
:108C000070B58AB00D460AA9002301F8043D012A77
:108C100098BF0A22B5FBF2F402FB1456F3B2092EF8
:108C200094BF30333733DBB2254601F8013D002CC9
:108C3000F0D1FFF7B6FF0AB070BD2DE9F04107464D
:108C40000E4615462AB90368C9B21B68BDE8F04153
:108C500018470A2A05D1002905DBBDE8F041FFF7D6
:108C6000CFBFD2B2F9E72D21FFF7ADFF2A46044668
:108C700071423846FFF7C4FF2044BDE8F081FFF79A
:108C8000DCBF38B50546FFF7D8FF04462846FFF796
:108C90009DFF204438BD10B42AB903685DF8044B29
:108CA0001B68C9B21847D2B25DF8044BFFF7A8BFE2
:108CB000FFF7F1BF38B50546FFF7EDFF044628463C
:108CC000FFF784FF204438BDFFF7E5BF2DE9F84FDB
:108CD00019460646104614461D469DF8287002F0B7
:108CE00017FC28B14C493046BDE8F84FFFF74BBFA1
:108CF00025F000494FF0FF32484B2046494602F02C
:108D000007FC48B94FF0FF32444B2046494602F079
:108D1000E1FB08B94249E6E74FF06042414B20468B
:108D2000294602F0EBFB08B13F49DCE74FF0604217
:108D30003E4B2046294602F0C3FB0028F4D1002216
:108D400000232046294602F0BBFBD0B12D2130463E
:108D5000FFF739FF05F1004382461D463449DFF82D
:108D6000D8904FF0000B00204FF000085FFA8BF313
:108D70009F4208D942464B4602F05AFA0BF1010BCA
:108D8000F4E78246EAE722462B4601F071FF0D46E2
:108D9000044602F0FBFB0A22014680463046FFF7FC
:108DA0002FFF8244A7B3404602F09EF802460B46CE
:108DB0002046294601F05AFF04460D4630461D491B
:108DC000DFF87490FFF7DFFE4FF000088244013FA8
:108DD000FFB2FF2F1CD04B4642462046294602F0E8
:108DE000FDF80D46044602F0A9FB0A22014683461F
:108DF0003046FFF722FF8244584602F085F80246CB
:108E00000B462046294601F031FF04460D46DEE7B9
:108E10005046BDE8F88F00BF30000100FFFFEF7F34
:108E200034000100FFFFEF4138000100FFFFEFC1F8
:108E30000000E03F6CF90000000024409DF80010A5
:108E40000091FFF743BF08B54022002102F07BFEEE
:108E50000022C0E9102208BD026C10B5531C446CFE
:108E600003F03F039C421CBF8154036410BD0023E8
:108E7000C0E910337047D0E9102393421FBFC25C92
:108E8000013303F03F03436414BF10464FF0FF303B
:108E90007047D0E91030181A48BF40307047D0E909
:108EA0001023934214BFC05C4FF0FF307047036C37
:108EB000406C013303F03F031B1A5842584170477E
:108EC0000649074A074B9B1A03DD043BC858D0509C
:108ED000FBDC00F04DF8F7F7B3FA00004C0401009A
:108EE000000000205C020020FEE7FEE7FEE7FEE750
:108EF000FEE7FEE7FEE7FEE7FEE7FEE7094B1B782D
:108F0000062B0CD1084B1B681A0708D1074B1868B1
:108F100000F0F000A0F130035842584170470020A3
:108F2000704700BFE00F00F0E40F00F0E80F00F022
:108F30000C4B1B78062B10D10B4B1B681A070CD15E
:108F40000A4B186800F0F003302B08D000F0E00066
:108F5000A0F140035842584170470020704701205B
:108F6000704700BFE00F00F0E40F00F0E80F00F0E2
:108F700008B5FFF7C3FF10B14A4B4B4A1A60FFF721
:108F8000D7FF28B1494B4A4A1B68C3F342331360E9
:108F9000FFF7B4FF20B1474AD36823F08073D36052
:108FA000FFF7C6FF40B14FF080430022C3F80C2109
:108FB000C3F81021C3F83825FFF7A0FF10B13E4BCE
:108FC00003221A60FFF79AFF40B13C4B05221A605A
:108FD00001229A6700229A603F225A60384B1B7820
:108FE000062B50D1374B1B681B074CD1364B1B68E7
:108FF00003F0F003502B46D14FF08052334BD2F8A0
:109000000414C3F82015D2F80814C3F82415D2F8B4
:109010000C14C3F82815D2F81014C3F82C15D2F884
:109020001414C3F83015D2F81814C3F83415D2F854
:109030001C14C3F84015D2F82014C3F84415D2F814
:109040002414C3F84815D2F82814C3F84C15D2F8E4
:109050002C14C3F85015D2F83014C3F85415D2F8B4
:109060003414C3F86015D2F83814C3F86415D2F874
:109070003C14C3F86815D2F84014C3F86C15D2F844
:109080004424C3F87025124AD2F8883043F47003A0
:10909000C2F88830BFF34F8FBFF36F8F0D4B0E4A6E
:1090A0001A6008BD74C007400DF0ADBA440200104C
:1090B0003C050040F0ED00E0A005004010560040E7
:1090C000E00F00F0E40F00F0E80F00F000C00040F7
:1090D00000ED00E0100000200090D00310B5044621
:1090E00000F056FAE06023682046DB6898470028C5
:1090F00008DA00F04DFAE368C01AA3689842F2D388
:109100004FF0FF3010BD0120704703681322DB6968
:10911000184770470369C3F81C150369D3F81C216D
:10912000002AFBD00022C3F81C2101207047000058
:1091300010B490F95C30144C59090122203103F02D
:109140001F0302FA03F344F8213003695DF8044B6E
:109150000421C3F8081303695A600369DA600369DC
:109160000022C3F8002502694FF0FF33C2F80C3526
:109170000269C2F814350269C2F808350269143070
:10918000C2F81035FFF773BE00E100E01430FFF7BE
:1091900080BE1430FFF783BE1430FFF76CBE0000B2
:1091A000036990F85E2010B5C3F80C25036990F8A8
:1091B0005D20C3F8142590F861200369012A01BFDE
:1091C00090F85F40C3F81045036990F8604006BF0F
:1091D000C3F8084503690022B1F5966FC3F86C2502
:1091E00069D9B1F5166F69D9B1F5965F69D9B1F54D
:1091F000165F68D9B1F5615F67D9B1F5964F66D949
:10920000B1F5E14F65D9B1F5164F64D9B1F5614FAC
:1092100064D9B1F5963F64D9B1F5E13F63D9B1F5B1
:10922000613F63D9364B994263D9B1F5E12F63D9D8
:10923000B1F5612F94BF4FF070634FF08053026916
:10924000C2F8243503690422C3F80025016900230C
:10925000C1F808310169C1F81C31016901230B60B3
:1092600001698B600169C1F8042390F95C20510900
:1092700002F01F0293406031224A42F8213090F9F7
:109280005C30002BBDBF03F00F0302F6FC32D21896
:109290009B18B5BF60236022137683F8002390F9F2
:1092A0005C300122590903F01F0302FA03F3154A47
:1092B00042F8213010BD4FF49E23C0E74FF41D2328
:1092C000BDE7114BBBE7114BB9E7114BB7E7114BAA
:1092D000B5E7114BB3E74FF41D03B0E74FF46B0351
:1092E000ADE70E4BABE74FF0EB73A8E74FF06C73B5
:1092F000A5E74FF08063A2E74FF0E8639FE700BF68
:1093000090D0030000E100E000B0130000502700FF
:1093100000F03A0000A04E0000C0750000903A0135
:109320002DE9F0411E4600254FF47A73C0E9015340
:109330000D4B044640F8143B17468846FFF783FD63
:109340000A4AC4F8108084F85C7052F8263084F819
:109350005D309DF8183052F8233084F85E3084F880
:1093600061502046BDE8F08144000100BCFF0000D0
:1093700010B50369D3F8082104464AB1D3F818158B
:109380001430C9B2FFF768FD23690022C3F8082131
:1093900010BD00000148FFF7EBBF00BFA005002093
:1093A00007B5192300930222182303490348FFF746
:1093B000B7FF03B05DF804FB00200040A0050020CB
:1093C00010B5044628B103F0F9F990FBF4F303FB60
:1093D0001404204610BD884210B5044603DA081A6A
:1093E000FFF7EEFF0444204610BD10B5029C401A62
:1093F000E41A6043521A90FBF2F0184410BD0023A7
:10940000C0E9003310B50C68836004604C684460A8
:109410008C688460C1E900338B6010BD10B50446D0
:10942000006802F043FB204610BD10B504460068FA
:1094300008B102F03BFB00232360C4E9013310BDF7
:1094400038B504460D460068013103F0EBF910B160
:10945000C4E90005012038BD036810B5044623B1F6
:1094600043688B4201D3012010BD2046FFF7E8FF7F
:109470000028F9D0A368002BF5D122681370F2E719
:1094800070B50E46114604461546FFF7E5FF20B9B4
:109490002046FFF7CAFF204670BDA5603146206810
:1094A00003F0BFFAF7E738B500230446C0E90033FC
:1094B00083600D4639B1084603F0D7FA29460246C3
:1094C0002046FFF7DDFF204638BD38B50546006869
:1094D0000C4668B16A688B689A4207D3096803F042
:1094E000A0FAA368AB600023A36038BD02F0DEFAE7
:1094F00023682B6063686B60A368AB600023C4E9DA
:109500000033F1E7884210B50B46044604D00968E1
:1095100021B19A68FFF7B4FF204610BDFFF785FF21
:10952000FAE710B500230446C0E900338360FFF773
:10953000E9FF204610BD884210B5044601D0FFF770
:10954000C4FF204610BD70B505460E4609B900207F
:1095500070BD6AB1846814442146FFF77DFF00287E
:10956000F5D02868AB683146184403F05AFAAC606D
:109570000120EDE707B500238DF80410012201A9B1
:109580008DF80530FFF7DFFF03B05DF804FB000046
:109590000A4B19680A4B30B5D3F804050C060D0ABE
:1095A00044EA00024FF47A712B46A2FB014501FB0D
:1095B0000355E00B40EA454030BD00BF04060020E3
:1095C0000010014038B5044648B1FFF7E1FF0546F9
:1095D00000F01AF8FFF7DCFF401BA042F8D338BDBB
:1095E000074B0022C3F8042182B0D3F80431054AA6
:1095F0000193019B13680133DBB2136002B0704723
:1096000000100140040600207047704708B500F0C4
:1096100017F8FFF7FAFF0120FFF7D4FFF8F7B8FCBF
:10962000034CF8F7B7FC002CFBD0AFF30080F8E751
:109630000000000002F032BA02F030BA02F036BA8E
:109640002A4BE02283F811234FF40032C3F8802123
:109650001A604FF080430122C3F818259A6003F581
:1096600088330021C3F808150221C3F80413C3F896
:1096700044131A604FF01023D3F80022002A03DBB2
:10968000D3F80432002B2FDA194B0122C3F804253A
:10969000D3F80024002AFBD04FF010221521C2F885
:1096A0000012D3F80024002AFBD04FF0102315221B
:1096B000C3F804220E4B1A46D3F800140029FBD03D
:1096C0000021C3F80415D2F80034002BFBD0BFF3FF
:1096D0004F8F0849084BCA6802F4E0621343CB601D
:1096E000BFF34F8F00BFFDE7704700BF00E100E010
:1096F00000E0014000ED00E00400FA05192837B54C
:109700000CD84B4B53F82030052B00F0828007D843
:10971000032B12D07BD8022B00F08180002074E054
:109720001D2B78D003D81C2BF8D1052206E01E2B68
:1097300073D01F2BF2D1082200E002223D4B1968A2
:1097400008296EDD0A296FDD0D29B5BF0C240E2412
:10975000022303233848C0F8F0350123C0F8003550
:1097600000200546030103F1804303F5E043013087
:109770000828C3F81455C3F81055F3D12F4B1868B7
:109780002F4B1B6800021B0303F4805300F4E060BE
:109790001843294BC3F81805C3F81425C3F810253E
:1097A0000DF10602C3F82C260122C3F830261A60F8
:1097B000D3F80021002AFBD00022C3F800210122A7
:1097C0005A601D4B1A46D3F804010028FBD0002034
:1097D000C3F8040101209860D2F81431002BFBD0AB
:1097E0000023C2F81431BDF906209A42124AB8BFCC
:1097F000ADF80630A142C2F80035BDF9060004D02C
:1098000035BF611A091BC840884003B030BD032230
:1098100094E7042292E7062290E707228EE70122CE
:109820008CE70824002395E70A24012392E700BF70
:10983000BCFF000020000020007000402400002039
:1098400010060020192830B53CD8224B53F82000D0
:10985000214B00221D4653F82240B4F1FF3F32D184
:109860001E4C45F822006FEA41411D4D1D4B2468F6
:1098700053F822306FEA514125F81210012101FA04
:1098800004F4C3F86005013CC3F8640505EB42022B
:10989000C3F86805C3F86C050020C3F80015C3F8C9
:1098A0000C05C3F80405C3F80845C3F81405C3F84C
:1098B0001005C3F82025C3F82415C3F82815C3F8EC
:1098C0002C05996030BD8442CAD00132032AC2D12E
:1098D000F8E700BFBCFF00001400002028000020B3
:1098E000080600206C00010019280FD8114B53F80E
:1098F000203003290AD8DFE801F002160A1003F528
:10990000E0734FF0A042002142F82310704703F5A6
:10991000E0734FF0A0420C21F6E703F5E0734FF03F
:10992000A0420421F0E703F5E0734FF0A0420321C9
:10993000EAE700BFBCFF000019280CD8064B53F81B
:109940002020012393404FF0A04211B9C2F80C35FA
:109950007047C2F808357047BCFF000019289FBF48
:109960004FF0A043054AD3F8103552F820009ABFB3
:1099700023FA00F000F0010000207047BCFF000057
:1099800038B50025057329B90B4B0C4A0C48232127
:1099900001F06CFE01600B4951F82220027151F870
:1099A000233083719DF8103051F823304371022326
:1099B000C371856038BD00BF78000100DB00010085
:1099C00086000100BCFF0000037B23B9437383734F
:1099D000036101230373704784B00DF1100C0CE98F
:1099E0000E009DF80810026800230129C2F8003516
:1099F000039B12D00BD303290CD0C2F85435019B22
:109A0000C2F824350123C2F8003504B0704743F092
:109A10000203F2E743F00403EFE743F00603ECE749
:109A200010B5FFF7D1FF03688279C3F808254279A2
:109A3000C3F80C250279C3F81025034BBDE810408C
:109A40000ECBFFF7C9BF00BF2806002010B485B0B9
:109A500001AC84E80E0094E80E0005B05DF8044BFC
:109A6000FFF7BABF70470368C3F81C15D3F8082185
:109A7000002AFBD0D3F818050022C3F80821C0B291
:109A80007047000007B5094B09490A484FF080426A
:109A90001A6000229A6002221A710B2300930C2292
:109AA0000D23FFF76DFF03B05DF804FB28060020CF
:109AB00000300040140600202DE9F04FDFF8089335
:109AC0008DB006460F4614461D4600F081F999F9FF
:109AD0000080B8F1FF3FCDE9000136D022462B4689
:109AE0002046294601F014FD834670BB32463B46B2
:109AF0003046394601F00CFD002282460023002842
:109B000040F0A0803046394601F0D0FC10B300226E
:109B100000232046294601F0C9FC8346002867D06F
:109B20000122A24B029200210022CDF828A0CDE90B
:109B30000467CDE90645CDE908120393B8F1000F9B
:109B400041D09B4C0023CDE90034DDE900010DB08C
:109B5000BDE8F08FDDE9000100F062FF80460028DB
:109B600000F08B804FF0000A4FF0000B52465B462E
:109B7000DDE9000101F09AFC0028E6D030463946C4
:109B800000F04EFF0028E0D02046294600F048FFB4
:109B90000028DAD099F90030844A03920421002287
:109BA000022BCDE90467CDE90645CDE908AB02916A
:109BB0000A9203D002A800F039FF50B901F078FDF5
:109BC0002223036005E002A800F030FF002800F027
:109BD00098800A9B1BB101F06BFD0A9B0360DDE9D5
:109BE0000834CDE90034DDE900010DB0BDE8F08FA7
:109BF0002046294600F014FF0028A6D000220023AA
:109C00002046294601F05CFC00289ED0674A99F95D
:109C10000030CDF828B00121CDE90467CDE9064533
:109C2000CDE90212002B71D062490020022BCDE950
:109C300008016FD101F03CFD212303600A9B002B3A
:109C4000CDD0C8E72046294601F030FC00283FF47B
:109C50007CAF01230293564B5449CDF828B0002223
:109C6000B8F1020FCDE90467CDE906450391CDE9CE
:109C70000823A8D1CDE9002367E73046394600F034
:109C8000CFFE00283FF46EAF2046294600F0C8FE04
:109C900000283FF467AFDDE900231046194601F0C4
:109CA00037FC99F900A0002866D10323DFF8FCC037
:109CB0000A9029462046029300223F4BCDF80CC063
:109CC000CDE90645CDE9046701F088F90022044694
:109CD0000D46002330463946BAF1000F20D1374FE8
:109CE0004FF06046CDE9086701F0EAFB18BB02A817
:109CF00000F09CFE0028A1D101F0DAFC22230360D1
:109D00009CE701F0D5FC2123036062E700230024D7
:109D1000CDE9083402A800F089FE00288ED189E739
:109D2000274F0026CDE9086701F0CAFBA0B9BAF1B8
:109D3000020FE1D0DBE72046294600F07FFE2246F5
:109D40002B4601F0B3FBA0B91E4B99F900A04FF0D0
:109D50006042CDE90823EAE72046294600F06EFE7E
:109D600022462B4601F0A2FB18B9124B0022CDE986
:109D7000082399F900A0DAE701220C4BCDF82880DE
:109D80000292CDE90467CDE906450393BAF1000FCD
:109D9000BCD0002200231046194601F049FABAF15E
:109DA000020FCDE908013FF445AFB3E71801010008
:109DB0000000F03F0000F0FF0000E03FFFFFEF4732
:109DC0000000F07FFFFFEFC72C0000200000000024
:109DD0002DE9F04F23F0004555EA020493B00DD071
:109DE000794E21F00044B4420F4682460FDD04F163
:109DF000404404F5801454EA0A035BD1734C0023F9
:109E0000CDE90034DDE9000113B0BDE8F08F9846DC
:109E100094464ED0B542EADC6B4EB54266D0002F78
:109E20008B468146CDE9022364DB0026BCF1000F9E
:109E30000ED1654B9D4246D0644B9D4200F0978009
:109E4000B8F1804F00F0B280614B984500F0CC83B0
:109E50004846594600F0E0FDCDE90001BAF1000F97
:109E600006D1002C60D0594B27F040429A425BD07B
:109E7000FF0F013F56EA070300F08280554B9D42D9
:109E800040F3B08003F104739D4240F34184524B90
:109E90009C4240F38280B8F1000F40F3828048A3D7
:109EA000D3E900231046194601F098F8CDE90001E6
:109EB000A8E728B1494813B0BDE8F04F00F0B8BD9D
:109EC000A542F7DCA8E704F1404303F5801353EA09
:109ED0000A0393D0404B9C4240F39083B8F1000FAB
:109EE0005FDBDDE90234CDE900348BE7BCF1000F24
:109EF00095D07CE73A4B9D4237DCA3F154739D42E9
:109F000093DD2B15A3F2FF33142B40F3E983C3F148
:109F100034032CFA03F202FA03F3634585D102F00D
:109F20000102C2F1020681E7B8F1000F07DADDE9AC
:109F300000230020254901F07BF9CDE90001002F25
:109F4000BFF660AF04F1404404F5801454EA060300
:109F500000F03C84012E7FF455AFDDE90045224638
:109F600005F10043CDE900234CE702265EE7B8F196
:109F7000000FC0F24F8348465946CDE9000141E742
:109F80004A4648465B46594600F070FE02460B467C
:109F900001F04EF9CDE9000134E7B8F1000FFFF60A
:109FA0007EAF00230024CDE900342BE74A46484623
:109FB0005B46594601F012F8CDE9000122E700BFE7
:109FC0009C7500883CE4377E0000F07F0000F03F85
:109FD0000000E03F0000E041FFFFEF3F1C010100F7
:109FE000FFFF3F43B4F5801F80F28F83DDE900015E
:109FF0000022CF4B00F0F2FFCDE900010C466FF0DC
:10A00000340C2315CB4DC4F31302A3F2FF3342F0FB
:10A010007F5403EB0C01AA420B9144F4401440F32B
:10A020006F83C54B9A4240F3F38300220023CDE9AE
:10A03000082301310B91A4F58014CDE91023BF4B07
:10A040000022CDE906230025DDE90001DDE9062334
:10A050002146824600F00AFEA346DDE9062380463B
:10A06000894650462146CDE90CAB00F001FE024680
:10A070000B460020B14901F0DBF80A460146CDE964
:10A080000E12134649460246404600F0A7FF6310F1
:10A0900043F0005382468B4603F500238C46CDE9FE
:10A0A00004AB5919D3460023CDE900BC0093DDE988
:10A0B00000AB002004460D4602460B46504659466A
:10A0C00000F08CFF02460B464046494600F0CEFDAC
:10A0D000DDE90623804689462046294600F0C6FD74
:10A0E00002460B46DDE90C0100F0C0FD52465B461E
:10A0F00000F074FF02460B464046494600F0B6FDAC
:10A10000DDE90E2300F06AFFDDE90445CDE9060133
:10A1100022462B462046294600F060FF72A3D3E971
:10A12000002304460D4600F059FF71A3D3E9002334
:10A1300000F09EFD22462B4600F050FF6EA3D3E9AF
:10A14000002300F095FD22462B4600F047FF6CA34C
:10A15000D3E9002300F08CFD22462B4600F03EFFA1
:10A1600069A3D3E9002300F083FD22462B4600F0CB
:10A1700035FF67A3D3E9002300F07AFD224680462D
:10A1800089462B462046294600F028FF02460B460A
:10A190004046494600F022FF524604460D465B46C3
:10A1A000DDE9040100F064FDDDE9062300F016FF9F
:10A1B00022462B4600F05CFD5246804689465B46AF
:10A1C0005046594600F00AFF00225D4BCDE90C01D4
:10A1D00000F04EFD42464B4600F04AFD00980D4609
:10A1E000044622462B465046594600F0F7FE002210
:10A1F00082468B46524B2046294600F037FDDDE96A
:10A200000C2300F033FD02460B464046494600F061
:10A210002DFDDDE9042300F0E1FE2246804689465B
:10A220002B46DDE9060100F0D9FE02460B4640460A
:10A23000494600F01DFD8046894602460B465046C1
:10A24000594600F015FD009833A3D3E900230446D6
:10A250000D4600F0C3FE5246CDE904015B462046A0
:10A26000294600F003FD02460B464046494600F0F1
:10A27000FDFC2BA3D3E9002300F0B0FE2AA3D3E911
:10A280000023804689462046294600F0A7FE024664
:10A290000B464046494600F0EBFCDDE9102300F098
:10A2A000E7FC80460B98894600F02EFE4246824627
:10A2B0008B464B46DDE9040100F0DAFCDDE90823BA
:10A2C00000F0D6FC52465B4600F0D2FC00985246A5
:10A2D0005B4604460D4600F0C9FCDDE9082300F0AA
:10A2E000C5FCDDE904232DE0EF4E454A287ECA3F38
:10A2F00065DBC9934A86CD3F01411DA96074D13FFA
:10A300004D268F515555D53FFFAB6FDBB66DDB3F0B
:10A31000033333333333E33F000000E009C7EE3F3C
:10A32000FD033ADC09C7EE3FF5015B14E02F3EBEAA
:10A33000000040438E98030079B60B000000F03F08
:10A340000000084000F092FC0B4602464946404699
:10A3500000F08CFC013E56EA070382468B46DDE99D
:10A36000020114BFD84BD94B0022CDE90423024689
:10A370000B46CDE9002300230093DDE90067324658
:10A380003B4600F073FC22462B4600F027FEDDE939
:10A390000223804689465046594600F01FFE024679
:10A3A0000B464046494600F063FC324680468946EB
:10A3B0003B4620462946CDE9028900F00FFE0B46B8
:10A3C000024606460F464046494600F051FCC04B47
:10A3D000994204460D468A4640F3268101F13F43E7
:10A3E00003F5E003034340F0F781A3A3D3E900237F
:10A3F000DDE9020100F03CFC3246804689463B46DE
:10A400002046294600F032FC02460B4640464946AB
:10A4100001F074F8002840F0DF81A8464FEA285385
:10A42000A3F2FE324FF4801313415344C3F30A5294
:10A43000A84DA2F2FF321541C3F3130423EA05012C
:10A440000020C2F1140B44F48014BAF1000F02464C
:10A450000B4644FA0BFB30463946B8BFCBF1000B34
:10A4600000F004FC02460B4606460F46DDE90201F9
:10A4700000F0FEFB4FEA0B5A0D46002480A3D3E9FF
:10A4800000232046294600F0A9FD32468046894631
:10A490003B462046294600F0E9FB02460B46DDE933
:10A4A000020100F0E3FB78A3D3E9002300F096FD5E
:10A4B00077A3D3E9002306460F462046294600F03D
:10A4C0008DFD02460B463046394600F0D1FB06466C
:10A4D0000F4602460B464046494600F0C9FB42463D
:10A4E0004B4604460D4600F0C1FB02460B46304683
:10A4F000394600F0BBFB2246804689462B46204663
:10A50000294600F06BFD64A3D3E9002306460F46FD
:10A5100000F064FD62A3D3E9002300F0A7FB3246FC
:10A520003B4600F05BFD60A3D3E9002300F0A0FBF5
:10A5300032463B4600F052FD5DA3D3E9002300F014
:10A5400095FB32463B4600F049FD5BA3D3E900236F
:10A5500000F08EFB32463B4600F040FD02460B46C3
:10A560002046294600F082FB06460F4602460B466F
:10A570002046294600F032FD0022CDE900014FF0CF
:10A5800080433046394600F071FB02460B46DDE958
:10A59000000100F04DFE424606460F464B4620465F
:10A5A000294600F01BFD42464B4600F061FB024687
:10A5B0000B463046394600F059FB22462B4600F048
:10A5C00055FB02460B4600203F4900F04FFB8A44F2
:10A5D000BAF5801FC0F22D815146DDE9042300F059
:10A5E000FDFCCDE900010DE4002FFFF631AC48463B
:10A5F000594613B0BDE8F04F00F04CB9B8F1000F68
:10A60000BFF6CFACDDE90234009304F100430193BF
:10A61000FFF7F8BB4A465B4600202B4900F008FED6
:10A62000CDE90001FFF7EEBB2B4B21F00048984528
:10A6300040F3E280294B0B4403430AD132463B46A8
:10A6400000F014FBDDE9022300F04EFF00283FF488
:10A65000E5AE1BA3D3E90023DDE9040100F0BEFC55
:10A6600017A3D3E9002300F0B9FCCDE90001FFF7FF
:10A67000C9BB00BFAFF30080FE822B654715973C36
:10A6800000000000432EE63FEF39FAFE422EE63F7F
:10A69000396CA80C615C20BED0A4BE726937663EDE
:10A6A000F16BD2C541BDBB3E2CDE25AF6A56113FD2
:10A6B00093BDBE166CC1663F3E5555555555C53FB9
:10A6C00059F3F8C21F6EA5010000F03F0000F0BF73
:10A6D000FFFF8F40FFFF0F00FFCB904000346F3F24
:10A6E000BCF1000F40F09180C3F1140345FA03F26E
:10A6F00002FA03F3AB4200F0A0806646FFF79CBB72
:10A7000000220023CDE9082397E44FF0000C78E401
:10A710005B4B9C427FF741AC5A4B9C423FF7BBAB33
:10A72000DDE900010022574B00F0A0FA46A3D3E96F
:10A73000002304460D4600F051FC45A3D3E9002355
:10A7400082468B462046294600F048FC0022CDE98F
:10A7500000014D4B2046294600F040FC02460B46C6
:10A760003DA1D1E9000100F081FA22462B4600F01C
:10A7700035FC02460B460020444900F077FA224699
:10A78000804689462B462046294600F027FC024693
:10A790000B464046494600F021FC31A3D3E9002393
:10A7A00000F01CFC02460B46DDE9000100F05EFAF9
:10A7B00002460B46804689465046594600F058FAF4
:10A7C000002004460D4652465B46BBE5DDE900230A
:10A7D00010461946FFF7D8BB23A3D3E90023DDE9D0
:10A7E000040100F0FBFB20A3D3E9002300F0F6FBFB
:10A7F000CDE90001FFF706BB244B98453FF70EAEAD
:10A80000DDE900239246934637E60026FFF720BB9A
:10A8100017A3D3E90023CDE9082317A3D3E9002325
:10A82000CDE910231A4B00224FF48025CDE90623F1
:10A830000AE45A4600F090F9CFE602F00102C2F1B4
:10A840000206FFF7F9BA00BF000000604715F73FA6
:10A8500044DF5DF80BAE543E555555555555D53F23
:10A86000FE822B654715F73F9C7500883CE4377ED8
:10A870000000004003B8E23F06D0CF43EBFD4C3E62
:10A88000FEFFEF3F0000F03F0000D03F0000E03F40
:10A890000000F83F5F4A8A432DE9F0410D46074624
:10A8A00000F0948000290B460446064654DD0F153F
:10A8B00000F0A780C3F31303A7F2FF3743F480131C
:10A8C000F20FF80702EB43034FEA460503D5ED0FFD
:10A8D00005EB4303B50000267F10B44616224FF463
:10A8E00000110CEB010098424FEAD5744FEA450580
:10A8F00003DC1B1A00EB010C0E44013A04EB43038A
:10A900004FEA5101EDD11046964620244FF0004207
:10A9100009E052D05B00013C03EBD5734FEA5202D1
:10A920004FEA450537D0634502EB0E01F1DD002902
:10A9300001EB020E0ADBE046A3EB0C03A94288BF41
:10A9400003F1FF336D1A1044C446E3E7BEF1000F74
:10A95000F1DB0CF10108EFE721F00042024329D0BE
:10A96000002945D10146CA0A153B4905002AFAD0FB
:10A9700012F4801001D048E030465200D40200F1B9
:10A980000106F9D5C6F1200401FA06F6E1401F1AC6
:10A9900041EA02038EE72B4324D14408731003F1EC
:10A9A0007F53F20703F5001348BF44F0004403EB64
:10A9B000075127463846BDE8F081A942AAD80029A8
:10A9C00001EB020EC2DB98460023BBE702460B46B2
:10A9D00000F004FB3A462B4600F04AF90746384699
:10A9E000BDE8F081411C16BF421C01365408D5E772
:10A9F000024600F03BF902460B4600F019FC074600
:10AA0000D8E71A4621463B46B2E70E4620244FF0CF
:10AA1000FF30BBE70000F07F21F00043194670478C
:10AA200041F0004101F58010C00F704700207047D1
:10AA300000200149704700BF0000F87F2DE9F04178
:10AA4000C1F30A57A7F2FF35132D82B002460B4619
:10AA50000C464FEAD178064633DC002D4EDB3B49ED
:10AA6000294103EA0100104326D049080B4052EA6D
:10AA700003060CD04FF48023132D24EA010143FA7E
:10AA800005F444EA01040CBF4FF0004600263049AB
:10AA900001EBC8082346D8E900453246204629463E
:10AAA00000F0E6F8CDE9000122462B46DDE9000181
:10AAB00000F0DCF802460B461046194602B0BDE82D
:10AAC000F081332D07DDB5F5806FF5D100F0D0F8BA
:10AAD00002460B46F0E7A7F213474FF0FF31F9406B
:10AAE0000842E9D049080842D1D04FF0804320EA1B
:10AAF000010143FA07F741EA0706C8E721F00041E0
:10AB00000143D9D0C3F3130101434E42104D0E430C
:10AB1000360B05EBC8055C0C06F40023D5E900678D
:10AB2000640443EA04010B463046394600F0A0F8BD
:10AB3000CDE9000132463B46DDE9000100F096F820
:10AB400021F00041024641EAC873B5E7FFFF0F005C
:10AB50002001010000000000F8B5C1F30A530446CB
:10AB60000D460E4617460BBB21F000460346334305
:10AB70001BD0354B002200F031FA344B9F42044683
:10AB80000D4635DBC1F30A530E46363B3B4440F2DB
:10AB9000FE72934232DC002B11DD26F0FF4626F4D4
:10ABA000E00646EA035520462946F8BD40F2FF720A
:10ABB0009342EBD102460B4600F05AF8F8BD13F170
:10ABC000350F28DA4CF250339F4222462B460ADDDD
:10ABD00019A1D1E9000100F03DF817A3D3E9002342
:10ABE00000F0FCF9F8BD16A1D1E9000100F032F83F
:10ABF00013A3D3E9002300F0F1F9F8BD22462B4658
:10AC00000DA1D1E9000100F025F80BA3D3E9002341
:10AC100000F0E4F9F8BD26F0FF4626F4E0063633EE
:10AC200046EA0355204629460022094B00F0D6F992
:10AC3000F8BD00BFAFF300809C7500883CE4377E10
:10AC400059F3F8C21F6EA50100005043B03CFFFF4E
:10AC50000000903C03F0004321F0004242EA03016F
:10AC6000704700BF81F0004102E000BF83F0004365
:10AC700030B54FEA41044FEA430594EA050F08BF97
:10AC800090EA020F1FBF54EA000C55EA020C7FEA5B
:10AC9000645C7FEA655C00F0E2804FEA5454D4EBD8
:10ACA0005555B8BF6D420CDD2C4480EA020281EAA2
:10ACB000030382EA000083EA010180EA020281EADA
:10ACC0000303362D88BF30BD11F0004F4FEA01312C
:10ACD0004FF4801C4CEA113102D0404261EB41013B
:10ACE00013F0004F4FEA03334CEA133302D05242C1
:10ACF00063EB430394EA050F00F0A780A4F101047D
:10AD0000D5F1200E0DDB02FA0EFC22FA05F28018B6
:10AD100041F1000103FA0EF2801843FA05F359419C
:10AD20000EE0A5F120050EF1200E012A03FA0EFC1B
:10AD300028BF4CF0020C43FA05F3C01851EBE37145
:10AD400001F0004507D54FF0000EDCF1000C7EEB62
:10AD500000006EEB0101B1F5801F1BD3B1F5001FA0
:10AD60000CD349085FEA30004FEA3C0C04F10104BF
:10AD70004FEA445212F5800F80F09A80BCF1004FE8
:10AD800008BF5FEA500C50F1000041EB045141EA6A
:10AD9000050130BD5FEA4C0C404141EB010111F46B
:10ADA000801FA4F10104E9D191F0000F04BF014616
:10ADB0000020B1FA81F308BF2033A3F10B03B3F1F4
:10ADC00020020CDA0C3208DD02F1140CC2F10C0284
:10ADD00001FA0CF021FA02F10CE002F11402D8BFE2
:10ADE000C2F1200C01FA02F120FA0CFCDCBF41EAAE
:10ADF0000C019040E41AA2BF01EB0451294330BD7D
:10AE00006FEA04041F3C1CDA0C340EDC04F1140459
:10AE1000C4F1200220FA04F001FA02F340EA030030
:10AE200021FA04F345EA030130BDC4F10C04C4F176
:10AE3000200220FA02F001FA04F340EA0300294656
:10AE400030BD21FA04F0294630BD94F0000F83F4A0
:10AE5000801306BF81F480110134013D4EE77FEA83
:10AE6000645C18BF7FEA655C29D094EA050F08BFCF
:10AE700090EA020F05D054EA000C04BF19461046B0
:10AE800030BD91EA030F1EBF0021002030BD5FEAF4
:10AE9000545C05D14000494128BF41F0004130BD1C
:10AEA00014F580043CBF01F5801130BD01F0004570
:10AEB00045F0FE4141F470014FF0000030BD7FEAE3
:10AEC000645C1ABF194610467FEA655C1CBF0B46DE
:10AED000024650EA013406BF52EA033591EA030FF5
:10AEE00041F4002130BD00BF90F0000F04BF0021ED
:10AEF000704730B54FF4806404F132044FF0000520
:10AF00004FF0000150E700BF90F0000F04BF002198
:10AF1000704730B54FF4806404F1320410F00045FE
:10AF200048BF40424FF000013EE700BF42004FEAF9
:10AF3000E2014FEA31014FEA02701FBF12F07F4376
:10AF400093F07F4F81F06051704732F07F4208BF2D
:10AF5000704793F07F4F04BF41F40021704730B534
:10AF60004FF4607401F0004521F000411CE700BF80
:10AF700050EA010208BF704730B54FF000050AE003
:10AF800050EA010208BF704730B511F0004502D504
:10AF9000404261EB41014FF4806404F132045FEA06
:10AFA000915C3FF4D8AE4FF003025FEADC0C18BFAF
:10AFB00003325FEADC0C18BF033202EBDC02C2F1A1
:10AFC000200300FA03FC20FA02F001FA03FE40EA33
:10AFD0000E0021FA02F11444BDE600BF70B54FF037
:10AFE000FF0C4CF4E06C1CEA11541DBF1CEA135515
:10AFF00094EA0C0F95EA0C0F00F0DEF82C4481EA7D
:10B00000030621EA4C5123EA4C5350EA013518BF9C
:10B0100052EA033541F4801143F4801338D0A0FB89
:10B0200002CE4FF00005E1FB02E506F00042E0FB36
:10B0300003E54FF00006E1FB03569CF0000F18BF3C
:10B040004EF0010EA4F1FF04B6F5007F64F54074E4
:10B0500004D25FEA4E0E6D4146EB060642EAC62177
:10B0600041EA55514FEAC52040EA5E504FEACE2EE4
:10B07000B4F1FD0C88BFBCF5E06F1ED8BEF1004FE7
:10B0800008BF5FEA500E50F1000041EB045170BD63
:10B0900006F0004646EA010140EA020081EA0301A7
:10B0A000B4EB5C04C2BFD4EB0C0541EA045170BDA3
:10B0B00041F480114FF0000E013C00F3AB8014F11D
:10B0C000360FDEBF002001F0004170BDC4F1000466
:10B0D000203C35DA0C341BDC04F11404C4F12005E7
:10B0E00000FA05F320FA04F001FA05F240EA020042
:10B0F00001F0004221F0004110EBD37021FA04F678
:10B1000042EB06015EEA430E08BF20EAD37070BD31
:10B11000C4F10C04C4F1200500FA04F320FA05F090
:10B1200001FA04F240EA020001F0004110EBD37092
:10B1300041F100015EEA430E08BF20EAD37070BD02
:10B14000C4F1200500FA05F24EEA020E20FA04F3DB
:10B1500001FA05F243EA020321FA04F001F000418A
:10B1600021FA04F220EA020000EBD3705EEA430EFB
:10B1700008BF20EAD37070BD94F0000F0FD101F02A
:10B180000046400041EB010111F4801F08BF013C63
:10B19000F7D041EA060195F0000F18BF704703F0A1
:10B1A0000046520043EB030313F4801F08BF013D28
:10B1B000F7D043EA0603704794EA0C0F0CEA1355E4
:10B1C00018BF95EA0C0F0CD050EA410618BF52EA9E
:10B1D0004306D1D181EA030101F000414FF00000A4
:10B1E00070BD50EA410606BF1046194652EA4306B2
:10B1F00019D094EA0C0F02D150EA013613D195EA26
:10B200000C0F05D152EA03361CBF104619460AD16D
:10B2100081EA030101F0004141F0FE4141F4700177
:10B220004FF0000070BD41F0FE4141F4780170BD67
:10B2300070B54FF0FF0C4CF4E06C1CEA11541DBFCC
:10B240001CEA135594EA0C0F95EA0C0F00F0A7F8CE
:10B25000A4EB050481EA030E52EA03354FEA0131FB
:10B2600000F088804FEA03334FF0805545EA13130E
:10B2700043EA12634FEA022245EA111545EA1065D6
:10B280004FEA00260EF000419D4208BF964244F16D
:10B29000FD0404F5407402D25B084FEA3202B61A8C
:10B2A00065EB03055B084FEA32024FF480104FF460
:10B2B000002CB6EB020E75EB030E22BFB61A7546D4
:10B2C00040EA0C005B084FEA3202B6EB020E75EB67
:10B2D000030E22BFB61A754640EA5C005B084FEACF
:10B2E0003202B6EB020E75EB030E22BFB61A75469C
:10B2F00040EA9C005B084FEA3202B6EB020E75EBA7
:10B30000030E22BFB61A754640EADC0055EA060E67
:10B3100018D04FEA051545EA16754FEA06164FEAAA
:10B32000C30343EA52734FEAC2025FEA1C1CC0D156
:10B3300011F4801F0BD141EA00014FF000004FF0E3
:10B34000004CB6E711F4801F04BF01430020B4F1A4
:10B35000FD0C88BFBCF5E06F3FF6AFAEB5EB030C5C
:10B3600004BFB6EB020C5FEA500C50F1000041EB59
:10B37000045170BD0EF0004E4EEA113114EB5C0426
:10B38000C2BFD4EB0C0541EA045170BD41F48011F9
:10B390004FF0000E013C90E645EA060E8DE60CEA01
:10B3A000135594EA0C0F08BF95EA0C0F3FF43BAF1E
:10B3B00094EA0C0F0AD150EA01347FF434AF95EAD5
:10B3C0000C0F7FF425AF104619462CE795EA0C0FB9
:10B3D00006D152EA03353FF4FDAE1046194622E786
:10B3E00050EA410618BF52EA43067FF4C5AE50EA60
:10B3F00041047FF40DAF52EA43057FF4EBAE12E750
:10B400004FF0FF3C06E000BF4FF0010C02E000BF30
:10B410004FF0010C4DF804CD4FEA410C7FEA6C5C13
:10B420004FEA430C18BF7FEA6C5C1BD001B050EAB6
:10B43000410C0CBF52EA430C91EA030F02BF90EAA1
:10B44000020F0020704710F1000F91EA030F58BF60
:10B45000994208BF90422CBFD8176FEAE37040F0C2
:10B46000010070474FEA410C7FEA6C5C02D150EA60
:10B47000013C07D14FEA430C7FEA6C5CD6D152EA1B
:10B48000033CD3D05DF8040B704700BF84461046E0
:10B4900062468C461946634600E000BF01B5FFF7DF
:10B4A000B7FF002848BF10F1000F01BD4DF808EDAF
:10B4B000FFF7F4FF0CBF012000205DF808FB00BF80
:10B4C0004DF808EDFFF7EAFF34BF012000205DF8DA
:10B4D00008FB00BF4DF808EDFFF7E0FF94BF012027
:10B4E00000205DF808FB00BF4DF808EDFFF7CEFF28
:10B4F00094BF012000205DF808FB00BF4DF808ED67
:10B50000FFF7C4FF34BF012000205DF808FB00BF37
:10B510004FEA410C7FEA6C5C02D150EA013C0AD14F
:10B520004FEA430C7FEA6C5C02D152EA033C02D141
:10B530004FF0000070474FF0010070474FEA4102A2
:10B5400012F5001215D211D56FF47873B3EB625275
:10B5500012D94FEAC12343F0004343EA505311F09C
:10B56000004F23FA02F018BF404270474FF000002E
:10B57000704750EA013005D111F0004008BF6FF06C
:10B58000004070474FF00000704700BF4A0011D2E2
:10B5900012F5001211D20DD56FF47873B3EB62522D
:10B5A0000ED44FEAC12343F0004343EA505323FA39
:10B5B00002F070474FF00000704750EA013002D1AE
:10B5C0004FF0FF3070474FF0000070474FEA4102E4
:10B5D000B2F1E04324BFB3F5001CDCF1FE5C0DD9F1
:10B5E00001F0004C4FEAC0024CEA5070B2F1004F3B
:10B5F00040EB830008BF20F00100704711F0804F3E
:10B6000021D113F13872BCBF01F00040704741F402
:10B6100080114FEA5252C2F11802C2F1200C10FA06
:10B620000CF320FA02F018BF40F001004FEAC123EA
:10B630004FEAD32303FA0CFC40EA0C0023FA02F38E
:10B640004FEA4303CCE77FEA625307D150EA013364
:10B650001EBF4FF0FE4040F44000704701F0004034
:10B6600040F0FE4040F40000704700BF1FB51C468C
:10B67000094B1B680546D86852B1084B0091CDE9CB
:10B68000013207492B46224600F09AF901F0BEFC30
:10B69000044B1A46F2E700BF3000002030010100E1
:10B6A0003D0101009AFF00000A22002101F016BBB3
:10B6B000014B1868704700BF3000002008B5074BE9
:10B6C000044613B10021AFF30080054B1868836A6C
:10B6D00003B19847204603F071FC00BF0000000052
:10B6E000CC0101008A892DE9F041054610070C467E
:10B6F00058D44B68002B05DC0B6C002B02DC0020BF
:10B70000BDE8F081E66A002EF9D0002312F48052E1
:10B710002F68216A2B6032D0606DA3895A0705D546
:10B720006368C01A636B0BB1236CC01A0023024616
:10B73000E66A216A2846B047431CA38906D12968D6
:10B740001D2948D8294ACA40D60744D5002262603C
:10B75000D9042269226004D5421C01D12B6803B9A7
:10B760006065616B2F600029C9D004F144039942E0
:10B7700002D0284600F0F0F900206063C0E7012302
:10B780002846B047411CC8D12B68002BC5D01D2BC3
:10B7900001D0162B01D12F60B1E7A38943F04003FC
:10B7A000A381ADE70F69002FA9D093070E6808BFEA
:10B7B0004B690F6018BF0023A6EB07088B60B8F138
:10B7C000000F9CDD43463A46216AA66A2846B047E8
:10B7D000002806DCA38943F04003A3814FF0FF302B
:10B7E0008EE70744A8EB0008E9E700BF010040200E
:10B7F00038B50B6905460C46DBB118B183690BB946
:10B8000000F072F80C4B9C4209D16C68B4F90C3012
:10B810007BB121462846BDE83840FFF763BF074BA0
:10B820009C4201D1AC68F1E7054B9C4208BFEC6833
:10B83000ECE7002038BD00BF8C010100AC01010025
:10B840006C010100014620B9044B0549186800F05D
:10B85000C9B8044B1868FFF7CBBF00BFCC0101008B
:10B86000F1B7000030000020002310B50446C0E905
:10B870000033836081814366C281C0E90433836100
:10B88000194608225C3000F05EF9054B6362054BF7
:10B89000A362054BE362054B2462236310BD00BF26
:10B8A00011C9000037C900006FC9000093C900002A
:10B8B000014900F097B800BFF1B7000070B54A1E0B
:10B8C000682555430E4605F1740100F093F90446CE
:10B8D00040B10021C0E900160C30A06005F16802FB
:10B8E00000F031F9204670BD836910B5044633BBC2
:10B8F000C0E912330365124B124A1B6882629842F8
:10B9000004BF0123836100F01FF86060204600F04F
:10B910001BF8A060204600F017F80022E060042128
:10B920006068FFF7A1FF01220921A068FFF79CFFD3
:10B9300002221221E068FFF797FF0123A36110BDE7
:10B94000CC010100B1B80000F8B51B4B1E68B3690B
:10B95000074613B93046FFF7C7FF4836D6E901342A
:10B96000013B03D5336833B13668F7E7B4F90C50BF
:10B970006DB16834F4E704213846FFF79FFF30606B
:10B980000028F1D10C233B6004462046F8BD0B4B48
:10B990006566C4E90055A560C4E90335C4E90555E9
:10B9A0000822294604F15C0000F0CDF8C4E90D55E9
:10B9B000C4E91255E9E700BFCC0101000100FFFF17
:10B9C0000EB403B5014603AB054853F8042B0068D9
:10B9D000019300F091F902B05DF804EB03B07047F9
:10B9E000300000202DE9F8438046894600F14804E4
:10B9F000002614B93046BDE8F883D4E90175013F4B
:10BA000001D52468F5E7AB89012B07D9B5F90E30CC
:10BA1000013303D029464046C84706436835EEE760
:10BA200070B50D4E0D4CA41BA4100025A54209D1E4
:10BA30000B4E0C4C03F0C4FAA41BA4100025A54225
:10BA400005D170BD56F8253098470135EEE756F818
:10BA5000253098470135F2E700020020000200205F
:10BA6000000200205802002010B5044600F008F83B
:10BA70002044407800F0440010BDD0F8EC0070473E
:10BA8000044B054A1B681B6A002B08BF1346D3F8FA
:10BA9000EC0070473000002094000020024B01466B
:10BAA000186800F0A7B800BF30000020024B014624
:10BAB000186800F051B800BF3000002082B001B912
:10BAC00001A942B14BB113780B601278101C18BF5A
:10BAD000012002B070471046FBE76FF00100F8E765
:10BAE00030B50024A24201D1002007E0035D0134FB
:10BAF0000D1915F8015CAB42F4D0581B30BD10B5E0
:10BB0000431E0A44914200D110BD11F8014B03F8C5
:10BB1000014FF7E7884210B501EB020307D8421E38
:10BB200099420AD011F8014B02F8014FF8E783421D
:10BB3000F5D98118D21AD34200D110BD13F8014DA6
:10BB400001F8014DF7E702440346934200D17047E4
:10BB500003F8011BF9E7000038B50546002945D078
:10BB600051F8043C0C1F002BB8BFE41802F088F910
:10BB70001F4A1368104633B9636014602846BDE855
:10BB8000384002F07EB9A3420CD921686218934272
:10BB900004BF1A685B68636004BF521822600460C7
:10BBA000ECE713465A680AB1A242FAD91968581844
:10BBB000A0420BD120680144581882421960DDD19F
:10BBC000106852685A6001441960D7E702D90C2303
:10BBD0002B60D3E7206821188A4204BF116852689D
:10BBE000626004BF091821605C60C7E738BD00BF10
:10BBF0003406002070B5CD1C25F0030508350C2D4A
:10BC000038BF0C25002D064601DBA94203D90C23C1
:10BC10003360002070BD02F033F9214A14682146D8
:10BC200091B9204C23681BB9304600F003FE206018
:10BC30002946304600F0FEFD431C24D10C2333601E
:10BC4000304602F01EF9E4E70B685B1B18D40B2B9F
:10BC50000FD90B60CD50CC18304602F012F904F128
:10BC60000B00231D20F00700C31AD3D05A42E25024
:10BC7000D0E78C424B6816BF636013600C46EBE75D
:10BC80000C464968CCE7C41C24F00304A04205D04C
:10BC9000211A304600F0CEFD0130CFD02560DBE721
:10BCA00034060020380600209368013B002B10B4B6
:10BCB000936007DA9469A34201DB0A2902D110BC20
:10BCC00001F0C4B81368581C10601970084610BC05
:10BCD0007047F8B506460F461446D518AC4201D158
:10BCE000002007E03A4614F8011B3046FFF7DCFF5E
:10BCF000431CF3D1F8BD00002DE9F04F9DB00C4678
:10BD000017460393064618B183690BB9FFF7ECFD9C
:10BD10007B4B9C4257D17468A38918075DD5236972
:10BD2000002B5AD00023099320238DF8293030238B
:10BD30008DF82A304FF0010BB846454615F8013B07
:10BD40000BB1252B54D1B8EB070A0BD053463A461A
:10BD500021463046FFF7BDFF013000F0C280099B4D
:10BD60005344099398F80030002B00F0BA80002368
:10BD70004FF0FF32CDE90523049307938DF853303C
:10BD80001A93A846052218F8011B5E4802F028F80D
:10BD9000049B78BBD90644BF20228DF853201A0794
:10BDA00044BF2B228DF853202A782A2A2AD0079ABA
:10BDB000A84600200A25414611F8013B303B092BDB
:10BDC00069D960B324E0504B9C4201D1B468A3E729
:10BDD0004E4B9C4208BFF4689EE72146304601F076
:10BDE000A7F800289ED04FF0FF301DB0BDE8F08FBF
:10BDF000A846A2E7434A801A0BFA00F018430490C1
:10BE00004546BEE7039A111D12680391002A01DB23
:10BE1000079204E0524243F002030792049398F819
:10BE200000302E2B0ED198F801302A2B38D1039BED
:10BE30001A1D1B680392002BB8BF4FF0FF3308F1A7
:10BE400002080593324D98F800100322284601F0AD
:10BE5000C7FF40B14023401B03FA00F0049B03439B
:10BE600008F10108049398F800102A488DF828106A
:10BE7000062208F1010701F0B3FF002837D0264B56
:10BE80001BBB039B073323F0070308330393099B72
:10BE90004B44099350E705FB0232012088468AE7AC
:10BEA000002308F10108059319460A25404610F8B9
:10BEB000012B303A092A03D9002BC3D00591C1E7E1
:10BEC00005FB012101238046F0E703AB00932246E6
:10BED000124B04A9304600F0B3F8B0F1FF3F8146A1
:10BEE000D5D1A3895B063FF57EAF09987DE703AB0B
:10BEF00000932246094B04A9304600F04DFBECE7C5
:10BF00008C010100D6010100AC0101006C010100AF
:10BF1000DC010100E001010041C00000D3BC0000D1
:10BF20002DE9F04788B0002B149F109DDDE9121A0F
:10BF30001E4627F02007BBBF03F100431E46002327
:10BF40002D23462F14460B7004D0452F00D1013508
:10BF5000022300E0032307AA049206AACDE902A265
:10BF6000CDE900352246334601F0F6F8472F8046EA
:10BF700002D1119BDB0726D5462F08EB050911D10D
:10BF800098F80030302B0AD1002200232046314699
:10BF9000FFF78CFA18B9C5F10105CAF80050DAF8B4
:10BFA000003099440022002320463146FFF77EFAF4
:10BFB00038B93022079B4B4505D2591C07911A709E
:10BFC000F8E7CDF81C90079B159AA3EB08034046B1
:10BFD000136008B0BDE8F087F7B500290446BABF82
:10BFE00049422D232B23092904F8022B437020DD1D
:10BFF0000DF107031F460A2691FBF6F506FB151106
:10C000003031092D03F8011C03F1FF32294609DC08
:10C010003031023B02F8011CBB42224604D3101A05
:10C0200003B0F0BD1346E7E713F8012B04F8012B2A
:10C03000F2E7302319448370021DC170EFE700005E
:10C040002DE9F04F91B00C461A9F93461E460546C7
:10C0500001F03CFE03680993184600F006FD00233A
:10C060000E933B680A90073323F0070303F108029D
:10C0700094F81880D4F800A03A60D3E90023C4E90A
:10C080001223D4E9127929F000430B934FF0FF32C9
:10C09000A64B0B993846FFF73BFA68BB4FF0FF32CF
:10C0A000A24B0B993846FFF715FA28BB0022002354
:10C0B00038464946FFF704FA10B12D2384F843307F
:10C0C0009B4F9C4BB8F1470F98BF1F46032323613A
:10C0D0002AF0040323604FF0000900965B460FAA84
:10C0E0002146284600F0E2F9013040F090804FF000
:10C0F000FF3011B0BDE8F08F3A464B46384649460E
:10C10000FFF706FA10B18C4F8C4BDBE76368591CC4
:10C110004AF480620EA90DA840D1062363600DF198
:10C120003303CDE901234FF0000C63682260CDE9B1
:10C13000030800933A464B46CDE9051C2846FFF715
:10C14000EFFE08F0DF03472B074609D10D9BD81CF3
:10C1500002DB6268934247DDA8F102085FFA88F8C3
:10C16000B8F1650F0D9924D80139424604F1500009
:10C170000D91FFF731FF0E9A1318012A81462361B2
:10C1800002DC2268D10701D5013323619DF83330E9
:10C19000002BA2D02D2384F843309EE7B8F1670F1F
:10C1A00000F06E81B8F1470FB9D1002BB7D1012350
:10C1B000B4E7B8F1660F19D1002963680CDD21617D
:10C1C00013B92268D20702D501330B4423610D9BBA
:10C1D000A3654FF00009D9E713B92268D00701D54C
:10C1E0000233F3E70123F1E74FF06708DDE90D3291
:10C1F000934205DB22682361D107E8D50133E5E7E7
:10C20000002BD4BFC3F1020301231344DEE72368EC
:10C210005A0507D423693A4659462846B0470130A3
:10C2200029D164E7B8F1650F40F2D78000220023DE
:10C23000D4E91201FFF73AF988B30123404A59467D
:10C240002846B04701303FF452AFDDE90D239A4252
:10C2500002DB2368D8070ED5DDE9092359462846B5
:10C26000B04701303FF443AF002704F11A080E9B9A
:10C27000013BBB4209DC23689F0700F1FD80E068B9
:10C280000F9B9842B8BF184633E7012342465946F0
:10C290002846B04701303FF42AAF0137E7E70D9B4E
:10C2A000002B2BDC0123264A59462846B047013093
:10C2B0003FF41DAF0D9B23B90E9B13B92368D9071B
:10C2C000D9D5DDE9092359462846B04701303FF466
:10C2D0000EAF4FF0000804F11A090D9B5B42434575
:10C2E00001DC0E9B97E701234A4659462846B04792
:10C2F00001303FF4FCAE08F10108EEE70E9AA36DA1
:10C300009A42A8BF1A46002A904607DD13465946AE
:10C310003A462846B04701303FF4E9AE04F11A032B
:10C320004FF0000A28EAE8780B9315E0FFFFEF7F53
:10C3300034000100E701010030000100EB010100C1
:10C3400038FF000001230B9A59462846B0470130B8
:10C350003FF4CDAE0AF1010AD4F85890A9EB0803D6
:10C360005345EFDCDDE90D239A424F4414DB23688B
:10C37000DA0711D40E9B0D99A3EB0902A3EB010977
:10C380009145A8BF9146B9F1000F0DDC002729EABD
:10C39000E97904F11A0818E0DDE90923594628462D
:10C3A000B0470130E6D1A2E64B463A465946284608
:10C3B000B0470130EAD19AE6012342465946284661
:10C3C000B04701303FF493AE0137DDE90D239B1AEE
:10C3D000A3EB0903BB42EFDC4DE70E9A012A01DC17
:10C3E000DB0738D501233A4659462846B047013085
:10C3F0003FF47DAEDDE9092359462846B0470130B8
:10C4000007F101073FF473AE0E9B002203F1FF38E2
:10C41000D4E912010023FFF749F8C0B943463A4670
:10C4200059462846B04701300DD160E60123424607
:10C4300059462846B04701303FF459AE01370E9BAC
:10C44000013BBB42F2DC4B4604F15002E4E600271C
:10C4500004F11A08F3E70123E1E7012342465946B4
:10C460002846B04701303FF442AE0137E3680F9AE7
:10C470009B1ABB42F1DC02E7002704F11908F5E73B
:10C48000002B3FF494AE4FF0000CCDE9051C0DF1EC
:10C4900033012260CDE90308CDE9012100933A463A
:10C4A0004B462846FFF73CFD07464FE62DE9F0478F
:10C4B00091461F468A680B69DDF820809342B8BF19
:10C4C0001346C9F8003091F8432006460C4612B1D5
:10C4D0000133C9F800302368990642BFD9F800300B
:10C4E0000233C9F80030256815F0060507D104F1BC
:10C4F000190AE368D9F800209B1AAB4228DC94F8AB
:10C5000043302268003318BF012392062DD404F172
:10C51000430239463046C047013020D02368E568E1
:10C52000D9F8002003F00603042B08BFAD1AA36856
:10C5300022690CBF25EAE57500259342C4BF9B1A0A
:10C54000ED184FF000091A344D451AD1002008E0CB
:10C550000123524639463046C047013003D14FF0DF
:10C56000FF30BDE8F0870135C3E7E1185A1C3020E1
:10C5700081F84300224494F8451082F843100233B6
:10C58000C5E70123224639463046C0470130E6D090
:10C5900009F10109D8E700002DE9F04301F1430C4E
:10C5A0000C46097E85B06E291746064698460C9AB9
:10C5B00000F0B38022D8632936D00AD8002900F0D1
:10C5C000B980582900F0838004F1420584F84210B4
:10C5D00032E0642901D06929F6D120681368050684
:10C5E00003F104012AD51B681160002B03DA2D2208
:10C5F0005B4284F843206F480A2239E0732900F037
:10C600009D8008D86F2920D07029DDD1236843F0A0
:10C610002003236003E0752917D07829D4D178232B
:10C6200084F84530644855E01368191D1B68116093
:10C6300004F1420584F8423001238CE01B6811604C
:10C6400010F0400F18BF1BB2CFE713682568181D04
:10C650001060280601D51B6802E06806FBD51B8820
:10C6600054486F2914BF0A220822002184F843107D
:10C670006568A560002DC0F29580216821F0040155
:10C680002160002B3DD1002D40F08E806546082AA8
:10C690000BD12368DB0708D5236962689A42DEBFA5
:10C6A000302305F8013C05F1FF35ACEB05032361B0
:10C6B000CDF800803B4603AA21463046FFF7F6FE40
:10C6C00001304DD14FF0FF3005B0BDE8F08339485F
:10C6D00084F84510136821681D1D1B6815600A0643
:10C6E0000BD5CA0744BF41F0200121601BB9226865
:10C6F00022F0200222601022B7E74D0648BF9BB20D
:10C70000EFE76546B3FBF2F102FB1133C35C05F8BA
:10C71000013D0B460029F5D1B9E713682568616929
:10C72000181D106028061B6801D5196002E06A0612
:10C73000FBD51980002323616546B9E71368191DED
:10C7400011601D6862680021284601F049FB08B1AC
:10C75000401B606063682361002384F84330A7E7CF
:10C7600023692A4639463046C0470130AAD023689B
:10C770009B0713D4E068039B9842B8BF1846A3E711
:10C7800001234A4639463046C04701309AD0013528
:10C79000E368039A9B1AAB42F2DCEBE7002504F155
:10C7A0001909F5E7002BACD1037884F8423004F185
:10C7B00042056CE7EF0101000002010038B5134BA0
:10C7C0001C68A36B7BB91820FFF768F9104A114B5E
:10C7D000A063C0E90023104B83600B2383810122F7
:10C7E0000023C0E90423A16B0C480A694B690C4C77
:10C7F000504304FB0300A2FB04230344541C43F1F5
:10C800000005C1E9044525F0004038BD3000002096
:10C810000E33CDAB34126DE6ECDE05002DF451582D
:10C820002D7F954C024B0A460146186801F014BE54
:10C830003000002038B5064C00230546084623602A
:10C8400002F0A6FB431C02D1236803B12B6038BD64
:10C85000400700200CB430B5174B0C1E9DB01D686E
:10C8600008DA8B232B604FF0FF301DB0BDE830405D
:10C8700002B070474FF40273ADF8143014BF04F1E6
:10C88000FF332346049307934FF6FF7302900690FD
:10C89000ADF81630209A21AB02A92846019301F089
:10C8A0005BFE431CBCBF8B232B60002CDDD0029BA6
:10C8B00000221A70D9E700BF300000200EB430B556
:10C8C0009CB01FAC4FF4017254F8045BADF8142017
:10C8D0000290069000F0C9F80B4B039007900B9361
:10C8E0000A48019400230F9314934FF6FF73ADF899
:10C8F00016302A46234602A9006801F07DFF1CB0CD
:10C90000BDE8304003B0704733C90000300000205C
:10C9100010B50C46B1F90E1002F016FA0028ABBFA4
:10C92000636DA3891B1823F48053ACBF6365A38197
:10C9300010BD002070472DE9F0411F468B89DB05B3
:10C9400005460C46164605D502230022B1F90E1005
:10C9500001F0CAF9A389B4F90E1023F48053A3811E
:10C9600032463B462846BDE8F04100F0CFBA10B54C
:10C970000C46B1F90E1001F0B7F9431CA38915BF9D
:10C98000606523F4805343F48053A38118BFA381CF
:10C9900010BDB1F90E1000F041BBF8B506460F46C8
:10C9A00016F8014BFFF76CF8204417F8015B437849
:10C9B00003F00303012B08BF2034FFF761F828447C
:10C9C000427802F00302012A08BF2035601B01D122
:10C9D000002DE5D1F8BD10B503461A785C1C3AB9B4
:10C9E000013B11F8012B03F8012F002AF9D110BDEA
:10C9F0002346F2E7C9B2034610F8012B1AB18A4266
:10CA0000F9D118467047002918BF0023F9E710F83C
:10CA1000012B11F8013B012A28BF9A42F7D0D01A06
:10CA20007047034611F8012B03F8012B002AF9D1B6
:10CA300070470000024B0146186800F003B800BFC1
:10CA40003000002070B5064608460C4600F00DF890
:10CA5000451C29463046FFF7CDF8064618B12A4650
:10CA60002146FFF74CF8304670BD034613F8012B02
:10CA7000002AFBD1181A0138704730B503461C78DC
:10CA80005D1C44B912F1FF3204D311F8014B03F8D5
:10CA9000014B14B930BD2B46F1E7002AF2D11A70D0
:10CAA000F0E710B56AB10139841810F8013B11F8AC
:10CAB000012F934203D1A04201D0002BF5D1981A47
:10CAC00010BD1046FCE770B50139044602B970BDCF
:10CAD000234611F8015F03F8015B561E2DB914447B
:10CAE000A342F4D003F8015BFAE71C463246EDE7B7
:10CAF00038B503460D4669B9BDE83840FFF77ABF3F
:10CB0000431C044629461846FFF774FF0028F7D156
:10CB1000204638BD0024F5E7134B2DE9F0411D6890
:10CB2000AC6D06460F46B4B95020FEF7B7FFA865B6
:10CB3000C0E90044C0E90244C0E90444C0E90A4431
:10CB4000C0E90C44C0E90E44C0E91044C0E91244F5
:10CB5000846104774462AA6D394630460123BDE8FA
:10CB6000F04100F003B800BF30000020F0B518B964
:10CB7000106808B9F0BD204604460F4614F8015B62
:10CB800017F8016B1EB96DB915602846F2E7B5427A
:10CB9000F6D1002BEFD114600370EBE72B460DE0CC
:10CBA00026B91C4623460F4613F8015B17F8016BA4
:10CBB000B542F5D1002DF1D0002121701360D9E7E5
:10CBC0002DE9F0478046894692461E460F463D466F
:10CBD000089815F8014BFEF750FF2044437813F0F6
:10CBE000080332D12D2C32D17C78BD1C0122002EBD
:10CBF0005DD0102E09D1302C07D12B7803F0DF0344
:10CC0000582B4FD16C7810260235002A14BF4FF0F4
:10CC100000416FF000410027B1FBF6FC384606FBEF
:10CC20001C1EA4F13003092B17D81C46A64223DD95
:10CC30007B1C07D084451CD301D1A64519DB00FB22
:10CC40000640012715F8014BEBE72F46BFE72B2CD9
:10CC500004BFBD1C7C781A46C9E7A4F14103192B17
:10CC600001D8373CE2E7A4F16103192B04D8573C03
:10CC7000DCE74FF0FF37E5E77B1C08D12223C8F83B
:10CC800000300846BAF1000F07D1BDE8F08702B1C5
:10CC90004042BAF1000FF8D00FB105F1FF39CAF8E0
:10CCA0000090F2E73024002EAFD10826ADE7302CFB
:10CCB000A3D00A26A9E7000037B5064C064D246824
:10CCC000246A002C08BF2C460094FFF779FF03B0BC
:10CCD00030BD00BF3000002094000020084B37B565
:10CCE0001C68084D236A002B08BF2B46009313468F
:10CCF0000A4601462046FFF763FF03B030BD00BF80
:10CD000030000020940000202DE9F047804689463D
:10CD100092461E460F463D46089815F8014BFEF711
:10CD2000ACFE2044437813F0080330D12D2C30D1D1
:10CD30007C78BD1C0121002E5CD0102E09D1302C36
:10CD400007D12B7803F0DF03582B4ED16C781026D7
:10CD500002354FF0FF320023B2FBF6F206FB02FC75
:10CD60006FEA0C0C1846A4F13007092F17D83C467F
:10CD7000A64223DD002B1EDB82421CD301D1A44539
:10CD800019DB00FB0640012315F8014BEBE72F46AA
:10CD9000C1E72B2C04BFBD1C7C781946CBE7A4F15E
:10CDA0004107192F01D8373CE2E7A4F16107192F99
:10CDB00004D8573CDCE74FF0FF33E5E7002B09DAF6
:10CDC0002223C8F800304FF0FF30BAF1000F07D12E
:10CDD000BDE8F08701B14042BAF1000FF8D00BB1C5
:10CDE00005F1FF39CAF80090F2E73024002EB0D1E7
:10CDF0000826AEE7302CA4D00A26AAE737B5064CA1
:10CE0000064D2468246A002C08BF2C460094FFF7C6
:10CE10007BFF03B030BD00BF300000209400002035
:10CE2000024B01461868FFF705BD00BF3000002027
:10CE300010B50446FEF724FE2044437803F00303B4
:10CE4000022B08BF203C204610BD0000F8B50E465E
:10CE50001446054618B183690BB9FEF745FD214B11
:10CE60009C422AD16C68A369A360A3891A072ED5B6
:10CE7000236963B323692068C01A6369F6B28342E9
:10CE8000374604DC21462846FEF7B2FC28BBA368DF
:10CE9000013BA36023685A1C22601E706369013045
:10CEA000834204D0A389DB0719D50A2E17D1214666
:10CEB0002846FEF79DFC90B10FE00B4B9C4201D140
:10CEC000AC68D0E7094B9C4208BFEC68CBE7214631
:10CED000284600F02DF80028CCD04FF0FF37384618
:10CEE000F8BD00BF8C010100AC0101006C01010024
:10CEF00049B1FF2A85BF8A2303600A704FF0FF30D3
:10CF000098BF0120704708467047000038B5074CAD
:10CF1000054608461146002222601A4602F046F8ED
:10CF2000431C02D1236803B12B6038BD40070020A9
:10CF3000324B70B51D6806460C4625B1AB6913B976
:10CF40002846FEF7D1FC2E4B9C420FD16C68B4F9F9
:10CF50000C309AB215072CD4D00611D409223260B5
:10CF600043F04003A3814FF0FF303EE0254B9C424D
:10CF700001D1AC68EBE7244B9C4208BFEC68E6E7C4
:10CF8000510712D5616B41B104F14403994202D0BB
:10CF90003046FEF7E1FD00236363A38923F02403F9
:10CFA000A3810023636023692360A38943F00803FE
:10CFB000A38123694BB9A38903F42073B3F5007FE0
:10CFC00003D02146304600F0C5FEA28912F00103CD
:10CFD0000CD00023A36063695B42A361236953B94A
:10CFE000B4F90C3013F08000BAD170BD920758BF6D
:10CFF0006369A360F2E70020F7E700BF300000207C
:10D000008C010100AC0101006C01010008B5062093
:10D0100001F006FF012001F0D1FF000038B5064CF9
:10D02000002305460846236001F07AFF431C02D125
:10D03000236803B12B6038BD400700202DE9F74F6E
:10D0400003690C69A3428046C0F28280013C01F171
:10D0500014074FEA840C00F1140657F8245056F8D0
:10D06000240006EB0C03013507EB0C090193B0FB20
:10D07000F5F595B34FF0000A3846B646D34650F85A
:10D08000042B93B205FB03A34FEA134A9BB2ABEB0D
:10D090000303120CDEF800B005FB02A213FA8BF3B7
:10D0A0004FEA124A1FFA82FBDEF80020CBEB124255
:10D0B00002EB23429BB243EA024381454FEA224BF3
:10D0C0004EF8043BDBD256F80C3033B9019B043BDD
:10D0D0009E421A4630D3C8F81040404601F0E8F8A6
:10D0E000002825DB013530464FF0000C57F8042BA3
:10D0F000D0F800E093B2ACEB0303120C13FA8EF3FA
:10D10000C2EB1E4202EB23429BB243EA0243B94503
:10D110004FEA224C40F8043BE8D256F8242006EBB4
:10D1200084032AB9043B9E421A460BD3C8F8104028
:10D13000284603B0BDE8F08F1268043B002ACAD12C
:10D14000013CC5E71268043B002AEFD1013CEAE745
:10D150000020EEE7000000002DE9F04F456A95B091
:10D1600016461F460446DDF88480CDE902673DB9C6
:10D170001020FEF793FC6062C0E901550560C560B0
:10D18000636A196851B15A684A60012393408B6001
:10D19000204600F0ABFE636A00221A603B1EBBBF54
:10D1A00023F00043039300230122ACBFC8F80030F2
:10D1B000C8F80020AE4BDDF80C8033EA08031BD121
:10D1C000209A42F20F731360029B23B9C8F3130035
:10D1D000002800F04B85229B53B9A64B21E0A64BBB
:10D1E00006930833229A1360069815B0BDE8F08FB5
:10D1F000A04B06930333F5E7DDE902670022002325
:10D2000030463946FEF752F9824660B1209A012332
:10D210001360229B002B00F02685984B229A136006
:10D22000013B0693E0E712AB019313AB0093324648
:10D230003B46204601F0B3F8C8F30A558346002D5B
:10D240007CD0C7F3130343F07F59B04649F440192B
:10D25000A5F2FF35CDF840A00022894B4046494653
:10D26000FDF704FD7CA3D3E90023FDF7B7FE7CA303
:10D27000D3E90023FDF7FCFC064628460F46FDF7E0
:10D2800043FE79A3D3E90023FDF7A8FE02460B462F
:10D2900030463946FDF7ECFC06460F46FEF74EF9E0
:10D2A00000228246002330463946FEF709F948B18C
:10D2B0005046FDF729FE32463B46FEF7F7F808B91F
:10D2C0000AF1FF3ABAF1160F59D86E4901EBCA01BB
:10D2D000DDE90223D1E90001FEF710F9002850D062
:10D2E0000AF1FF3A00230D93129B5D1B6B1E0793FF
:10D2F00043BF0023C5F1010907934FF00009BAF1BC
:10D30000000F40DB079BCDF830A053440793002368
:10D3100008931E9B092B00F28E80052BC4BF043B93
:10D320001E931E9BA3F10203CCBF00250125032BF6
:10D3300000F28D80DFE803F07B7D2F6FDDE9125373
:10D340001D4405F23240202813DDC0F14000029B4D
:10D3500008FA00F805F2124023FA00F048EA00004B
:10D36000FDF7C2FD01238046A1F1F879013D10933C
:10D3700072E7029BC0F1200003FA00F0F0E70123FE
:10D38000B1E70D90B0E7CAF1000308930023A9EBC1
:10D390000A090C93BDE7012309931F9B002B75DD40
:10D3A00004939846666A00227260042202F1140017
:10D3B000984271686FD9204600F064FD636A30605E
:10D3C0001B680693B8F10E0F00F2EE80002D00F0FE
:10D3D000EB80DDE90223BAF1000FCDE90E2378DD01
:10D3E000284A0AF00F0302EBC303D3E900234FEAF4
:10D3F0002A16F006CDE90A2369D5234BDDE90E0193
:10D40000D3E90823FDF714FFCDE9020106F00F066A
:10D4100003251D4F50E0012309931F9B534403F143
:10D42000010804934346012BB8BF0123BAE7002348
:10D43000B2E70023F0E7012500231E9309954FF082
:10D44000FF3304939846002212231F92AAE7012378
:10D450000993F4E7AFF3008061436F63A787D23F7E
:10D46000B3C8608B288AC63FFB799F501344D33FD3
:10D470000000F07F1B0301001203010039FF0000D0
:10D480000000F83F4803010020030100012304933A
:10D4900098461A46D9E701317160520086E7F107D4
:10D4A00008D5DDE90A01D7E90023FDF797FDCDE9AD
:10D4B0000A01013576100837002EF0D1DDE90A2384
:10D4C000DDE90201FDF7B4FECDE902011BE0022512
:10D4D0009FE700F0A480CAF10006A24BA24F06F01D
:10D4E0000F0203EBC203D3E90023DDE90E01FDF7D0
:10D4F00075FDCDE90201361100230225002E40F012
:10D500008380002BE0D10D9B002B00F08A80DDE9A9
:10D510000223CDE90A23DDE90A010022934BFDF73E
:10D52000CFFF00287DD0B8F1000F7AD0049B002BEC
:10D5300036DD00228E4BDDE90A01FDF74FFDCDE916
:10D540000201049E0AF1FF3701352846FDF7DCFC95
:10D55000DDE90223FDF742FD0022864BFDF788FB43
:10D56000A1F15075CDE90A010B95002E5CD1002286
:10D57000814BDDE90201FDF779FB0A9A2B46CDE9E3
:10D580000201FDF7BBFF002840F084820A9A05F1F2
:10D590000043DDE90201FDF793FF002840F07882A7
:10D5A000DDE90E23CDE90223139B002BC0F24E814F
:10D5B000BAF10E0F00F34A816A4B03EBCA03D3E9B9
:10D5C0000023CDE904231F9B002B80F2D980B8F102
:10D5D000000F00F3D58040F05A820022664BDDE94F
:10D5E0000401FDF7FBFCDDE90223FDF77DFF464664
:10D5F0004746002840F03082069B069A5D1C312386
:10D6000013700AF1010A2BE2F20705D5D7E90023CE
:10D61000FDF7E4FC01350123761008376EE702259B
:10D6200071E75746464690E74E4B03EBC60353E976
:10D630000201099B002B48D002460B4600204F49AF
:10D64000FDF7F6FDDDE90A23FDF710FBCDE90A0140
:10D65000069DDDE90201FDF771FF1190FDF754FC15
:10D6600002460B46DDE90201FDF700FB119B30335A
:10D6700005F8013BDDE90A23CDE90201FDF720FFB2
:10D68000002864D1DDE9022300203849FDF7EEFAD5
:10D69000DDE90A23FDF714FF002840F0B780069B60
:10D6A000EB1A9E427FF77CAF0022314BDDE90A0185
:10D6B000FDF794FC0022CDE90A012D4BDDE90201C2
:10D6C000FDF78CFCCDE90201C3E7DDE90A23FDF794
:10D6D00085FC069BCDE90A019D191E46DDE9020184
:10D6E000FDF72CFF1190FDF70FFC02460B46DDE91C
:10D6F0000201FDF7BBFA119B303306F8013BAE4245
:10D70000CDE902014FF0000225D11C4BDDE90A01F1
:10D71000FDF7AEFA02460B46DDE90201FDF7EEFE2B
:10D72000002873D1DDE90A2300201449FDF79EFA91
:10D7300002460B46DDE90201FDF7C2FE00283FF478
:10D740002FAF15F8013C302B05F1FF3201D0BA465E
:10D750004BE01546F5E7064BFDF740FCCDE902012D
:10D76000BCE700BF48030100200301000000F03FB8
:10D770000000244000001C40000014400000E03F76
:10D78000DDE90267069DDDE9042330463946FDF7F1
:10D790004FFDFDF7D3FE8146FDF7B6FBDDE904231F
:10D7A000FDF71CFC02460B463046394609F13006AF
:10D7B000FDF75CFA05F8016B069EAE1BB04502460C
:10D7C0000B4636D1FDF754FADDE9042306460F4631
:10D7D000FDF794FEC8B9DDE9042330463946FDF76C
:10D7E00065FE10B119F0010F0FD15946204600F027
:10D7F0007DFB0023209A2B700AF101031360229B0A
:10D80000002B3FF4F1AC1D60EEE4574615F8012CF7
:10D81000392A05F1FF3306D1069A9A4207D13023FF
:10D820001370013713461A7801321A708FE71D46BC
:10D83000ECE70022994BFDF7D1FB002200230646BE
:10D840000F46FDF733FE00289DD0CEE7099A002A47
:10D8500000F088801E9A012A6DDC109A002A66D09A
:10D8600003F23343089E4D46079A01211A4420468D
:10D870009944079200F0DAFB0746002D0BDD079B69
:10D88000002B08DDAB42079AA8BF2B46A9EB030982
:10D89000ED1AD31A0793089BEBB1099B002B65D0B7
:10D8A0008EB139463246204600F060FC5A460146A9
:10D8B0000746204600F0C3FB59460A90204600F078
:10D8C00015FB0A9B9B46089B9A1B04D05946204691
:10D8D00000F04CFC83460121204600F0A7FB0C9B86
:10D8E0000646002B00F0C9811A460146204600F08A
:10D8F0003DFC1E9B012B06463EDC029B002B37D1D4
:10D90000039BC3F31303002B34D1039B23F0004389
:10D910001B0D1B052BB1079B0133079309F101096F
:10D92000012308930C9B002B28D101202EE0129B91
:10D93000C3F1360396E7089B08F1FF36B342BFBF39
:10D94000089B0896F21A0C9BB7BF9B189E1B0C9362
:10D950000026B8F1000FB9BFA9EB080500234D461A
:10D96000434681E7089E099F4D4686E7089AADE742
:10D970000023D6E7029BD4E700230893336906EB24
:10D980008303186900F004FBC0F12000079B1844D2
:10D9900010F01F0047D0C0F12003042B3BDD079B94
:10D9A000C0F11C008144054403440793B9F1000F02
:10D9B00005DD59464A46204600F026FC8346079B73
:10D9C000002B05DD31461A46204600F01DFC0646B8
:10D9D0000D9B53B33146584600F06AFC002824DA08
:10D9E000002359460A22204600F097FA099B0AF1C3
:10D9F000FF3A8346002B00F04781002339460A2274
:10DA0000204600F08AFA049B002B07464EDC1E9B42
:10DA1000022B4BDD11E0C9D0079A1C331A449944FC
:10DA20001D441346C1E70346F6E7B8F1000F37DCA3
:10DA30001E9B022B34DDCDF81080049B63B9314668
:10DA40000522204600F069FA01460646584600F0D5
:10DA50002FFC00283FF7D0AD1F9B069D6FEA030AFD
:10DA60004FF000093146204600F040FA002F3FF405
:10DA7000BCAEB9F1000F05D0B94503D049462046E8
:10DA800000F034FA3946204600F030FAADE60026C0
:10DA90003746E1E7BA463746AEE500BF000024400E
:10DAA000099BCDF81080002B00F0F580002D05DDDE
:10DAB00039462A46204600F0A7FB0746089B002B64
:10DAC0004CD07968204600F0DDF93A69023205460B
:10DAD000920007F10C010C30FEF711F801222946E3
:10DAE000204600F091FB069B0793029B03F0010385
:10DAF000B9460893074631465846FFF79FFA49460C
:10DB0000054600F13008584600F0D2FB3A46029034
:10DB10003146204600F0E6FBC368024603BB0146DF
:10DB20000990584600F0C4FB099A03461146204666
:10DB3000099300F0DBF9099BA3B91E9A92B9089AE0
:10DB400082B9B8F1390F29D0029B002B01DD05F114
:10DB50003108079B5D1C83F8008083E73846C2E7E5
:10DB60000123E3E7029A002A04DB24D11E9A12BBA8
:10DB7000089A02BB002BECDD59460122204600F03A
:10DB800043FB3146834600F093FB002803DCE0D1E1
:10DB900018F0010FDDD0B8F1390FD8D1079B079AE3
:10DBA0005D1C3923137015F8013C392B05F1FF3248
:10DBB0004ED0013353E0079A002B02F1010506DD38
:10DBC000B8F1390FEAD008F10108079BC3E7069BBB
:10DBD000049A05F8018CEB1A934221D05946002390
:10DBE0000A22204600F099F9B94583464FF0000318
:10DBF0004FF00A024946204605D100F08EF98146D1
:10DC00000746079577E700F088F9394681460023F3
:10DC10000A22204600F081F90746F2E74FF000099A
:10DC200059460122204600F0EFFA3146834600F0C3
:10DC30003FFB0028B7DC02D118F0010FB3D115F873
:10DC4000013C302B05F1FF327FF40CAF1546F6E7AF
:10DC5000069B934205D1069A0AF1010A31231370FB
:10DC600000E715469FE7174BFFF7DBBA229B002B17
:10DC70007FF4B5AA144BFFF7D4BA1E9B012B7FF794
:10DC80003CAE0C9B089350E6049B002B03DC1E9BD0
:10DC9000022B3FF7D2AE069D31465846FFF7CEF92C
:10DCA00000F1300805F8018B069B049AEB1A9A42A2
:10DCB000B4DD594600230A22204600F02EF983469F
:10DCC000EAE700BF38FF000012030100044B1B68A5
:10DCD000186A044B002808BF1846F030704700BF90
:10DCE000300000209400002038B5074C0546084657
:10DCF0001146002222601A4601F03AF9431C02D173
:10DD0000236803B12B6038BD4007002070B50E4674
:10DD1000B1F90E10002996B014461D4607DA00230B
:10DD20002B60B3891A0610D44FF480630EE06A4664
:10DD300001F0CCF80028F2DB019A02F47042A2F55F
:10DD400000535A425A412A60EEE7402300202360E4
:10DD500016B070BD8B8973B59D0706460C4607D576
:10DD600004F14703236023610123636102B070BDA6
:10DD700001AB6A46FFF7CAFF009905463046FDF73A
:10DD800039FF48B9B4F90C309A05EFD423F00303F6
:10DD900043F00203A381E3E70D4BB362A389206044
:10DDA00043F08003A381009B6361019B20615BB111
:10DDB000B4F90E10304601F09BF828B1A38923F086
:10DDC000030343F00103A381A3891D43A581CDE78C
:10DDD000B1B80000000000000000000000000000DA
:10DDE00001F0FF01102A2BDB10F0070F08D010F80C
:10DDF000013B013A8B422DD010F0070F42B3F6D110
:10DE0000F0B441EA012141EA014122F007047FF028
:10DE100000070023F0E80256083C85EA010586EA7F
:10DE2000010685FA47F5A3FA87F586FA47F6A5FABB
:10DE300087F68EB9EED1F0BC01F0FF0102F00702C7
:10DE400032B110F8013B013A83EA010313B1F8D172
:10DE50000020704701387047002D06BF3546033853
:10DE6000073815F0010F07D1013015F4807F02BF8C
:10DE7000013015F4C03F0130F0BC0138704700BFDD
:10DE80007047704770B5456A04460E463DB910208C
:10DE9000FDF704FE6062C0E901550560C560656A72
:10DEA000EB6883B1636ADB6853F82600B8B90121D7
:10DEB00001FA06F56A1D9200204600F0BFFA60B133
:10DEC000C0E901650EE021220421204600F0B6FAE7
:10DED000636AE860DB68002BE4D1002070BD026853
:10DEE00043F826200023C0E90333F7E770B5446AFE
:10DEF00006460D463CB91020FDF7D0FD7062C0E922
:10DF000001440460C4603DB1736A6A68DB6853F819
:10DF10002210296043F8225070BD2DE9F0410D69AF
:10DF20001F4606460C4601F1140C0023DCF80000E5
:10DF300081B202FB01710F0C000C02FB007089B270
:10DF4000013301EB00419D424FEA10474CF8041B9E
:10DF5000ECDCD7B1A368AB4212DC6168304601311A
:10DF6000FFF790FF2269023204F10C018046920013
:10DF70000C30FDF7C4FD21463046FFF7B7FF44469D
:10DF800004EB850301355F6125612046BDE8F08122
:10DF9000020C12040346B2B90304102013F07F4FA1
:10DFA00004BF1B02083013F0704F04BF1B01043084
:10DFB00013F0404F04BF9B000230002B06DB5B00D8
:10DFC00003D5013070470020E8E720207047036840
:10DFD00013F0070201460BD0DA0723D4980749BF94
:10DFE0005B089B0801200B605CBF0B600220704740
:10DFF00098B2A8B91B0C102013F0FF0F04BF1B0A26
:10E0000008301A0704BF1B0904309A0704BF9B0895
:10E010000230DA0702D45B0806D001300B6070478B
:10E020001046E9E7002070472020704710B50C46E5
:10E030000121FFF727FF01224461026110BD2DE994
:10E04000F74F14460A6923699A42B8BF0B468846BF
:10E05000BCBFA0461C46D8F81070D4F81090D8F871
:10E060000830D8F8041007EB0906B342B8BF0131F5
:10E07000FFF708FF00F1140505EB860E2B46002282
:10E08000734516D304F1140208F1140102EB89035D
:10E0900001EB87070093009B019293420CD8002E5E
:10E0A00003DD5EF8043D002B5DD0066103B0BDE8E2
:10E0B000F08F43F8042BE3E7B2F800B0BBF1000F98
:10E0C00023D08946AC464FF0000859F8044BDCF8E1
:10E0D00000A0A3B21FFA8AFA0BFB03A34FEA144A6B
:10E0E000DCF8004043444FEA14480BFB0A8404EB7D
:10E0F0001344E2469BB243EA04434F454FEA1448B7
:10E100004AF8043B2BD8CCF80480019BB3F802A05A
:10E110000432BAF1000F20D02B688946A8464FF090
:10E12000000BB9F800C0B8F802400AFB0C445C448C
:10E13000C4469BB243EA04434CF8043B59F8043B01
:10E14000B8F804B01B0C0AFB03B303EB14434F45B0
:10E150004FEA134B05D8C8F8043004359BE7D44682
:10E16000B3E7E046DDE7013E99E700002DE9F8431B
:10E17000154612F0030206460F4607D0013A214C1D
:10E18000002354F82220FFF7C8FE0746AD1035D013
:10E19000746A3CB91020FDF781FC7062C0E901444B
:10E1A0000460C460D6F82480D8F808404CB940F226
:10E1B00071213046FFF73AFF0023C8F808000446F3
:10E1C00003604FF00008EB070AD539462246304677
:10E1D000FFF735FF394681463046FFF787FE4F4649
:10E1E0006D100BD0206838B9224621463046FFF723
:10E1F00026FF2060C0F800800446E4E73846BDE80A
:10E20000F88300BF100401002DE9F0470C464FEAE7
:10E21000621A236949680AEB0309A3680746164690
:10E2200009F10105AB4232DB3846FFF72BFE002334
:10E23000804600F114011A4653452BDB20692AEA77
:10E24000EA7A04F1140316F01F0201EB8A0103EBD2
:10E25000800C25D0C2F1200E00201E688A46964010
:10E2600030434AF8040B53F8040B9C4520FA0EF097
:10E2700014D8486008B109F10205013D3846C8F8D4
:10E2800010502146FFF732FE4046BDE8F0870131CD
:10E290005B00C7E741F823200133CDE75146DCE7B7
:10E2A000043953F8042B41F8042F9C45F9D8E4E7CE
:10E2B00003690A699B1A30B50CD1920014301431ED
:10E2C0008418114454F8045D51F8042D954203D08C
:10E2D00005D30123184630BDA042F3D3FAE74FF02F
:10E2E000FF33F7E72DE9F0470D460746114628466C
:10E2F0001446FFF7DDFF061E08D131463846FFF70A
:10E30000C1FD0123C0E90436BDE8F087A4BF234660
:10E310002C4638466168A6BF1D4600260126FFF739
:10E32000B1FD2B69C660266905F1140904F11402D8
:10E3300002EB860709EB830800F114054FF0000E8D
:10E3400052F804AB59F8044B1EFA8AF1A3B2C91A69
:10E35000230CC3EB1A4303EB214389B24FEA234E4C
:10E36000C84541EA0343944645F8043BE8D8BC4518
:10E3700004D355F8043D83B10661C5E75CF8041B7E
:10E380001EFA81F31A1402EB11429BB243EA0243D4
:10E390004FEA224E45F8043BE9E7013EE9E72DE963
:10E3A000F34101211C469046DDE90865FFF76AFD4F
:10E3B000C4F31302C4F30A54074634BB0192B8F104
:10E3C000000227D002A840F8082DFFF700FE0099B0
:10E3D000F0B1019AC0F1200302FA03F30B43C240EB
:10E3E0007B610192019BBB61002B14BF02210121C3
:10E3F0003961C4B1A4F2334404443460C0F135003F
:10E400002860384602B0BDE8F08142F48012D5E7BA
:10E410007961E7E701A8FFF7DAFD019B7B61012144
:10E4200039612030E5E707EB8103A0F2324030602C
:10E430001869FFF7ADFDC0EB4110E1E738B502FB0D
:10E4400001F42146FDF7D6FB054618B1224600210E
:10E45000FDF779FB284638BDF8B5074614460E4649
:10E4600021B91146BDE8F840FDF7C4BB22B9FDF75C
:10E4700073FB25462846F8BD00F04AFDA0420FD2A6
:10E4800021463846FDF7B6FB05460028F2D0314656
:10E490002246FDF734FB31463846FDF75DFBE9E7E0
:10E4A0003546E7E72DE9F0478E689E4282460C46E6
:10E4B0009046994637D88A8912F4906F31D02568F2
:10E4C00009696F1A6569022305EB450595FBF3F5AC
:10E4D00009F101033B449D4238BF1D46530530D529
:10E4E0002946FDF787FB064650B90C23CAF80030D1
:10E4F000A38943F04003A3814FF0FF30BDE8F087CC
:10E500003A462169FDF7FBFAA38923F4906343F0AF
:10E510008003A381266165613E44ED1B2660A560F2
:10E520004E464E4500D94E46324641462068FDF7DC
:10E53000F1FAA3689B1BA36023681E442660002099
:10E54000DCE72A46FFF788FF06460028E2D121696A
:10E550005046FDF701FBC8E72DE9F04F9DB080461E
:10E5600003938B891D060C4616460FD50B696BB9B4
:10E570004021FDF73FFB2060206128B90C23C8F83B
:10E5800000304FF0FF30C7E0402363610023099360
:10E5900020238DF8293030238DF82A304FF0010BDD
:10E5A00037463D4615F8013B0BB1252B3ED1B7EB65
:10E5B000060A0BD05346324621464046FFF772FF0B
:10E5C000013000F0A480099B534409933B78002B51
:10E5D00000F09D8000234FF0FF32CDE90523049326
:10E5E00007938DF853301A932F46052217F8011B15
:10E5F0004F48FFF7F5FB049BD0B9D90644BF202252
:10E600008DF853201A0744BF2B228DF853202A7807
:10E610002A2A15D0079A2F4600200A25394611F8D4
:10E62000013B303B092B4DD9B8B10FE02F46B8E77D
:10E630003F4A801A0BFA00F0184304903D46D3E796
:10E64000039A111D12680391002A01DB079204E06E
:10E65000524243F00203079204933B782E2B0CD1D5
:10E660007B782A2B33D1039B1A1D1B680392002B46
:10E67000B8BF4FF0FF33023705932E4D3978032290
:10E680002846FFF7ADFB38B14023401B03FA00F0EA
:10E69000049B034301370493397827488DF82810E9
:10E6A00006227E1CFFF79CFB002838D0234B13BBAF
:10E6B000039B073323F0070308330393099B4B4461
:10E6C00009936DE705FB023201200F46A6E7002300
:10E6D0000137059319460A25384610F8012B303AC0
:10E6E000092A03D9002BC8D00591C6E705FB0121F3
:10E6F00001230746F0E703AB00932246104B04A921
:10E700004046FDF79DFCB0F1FF3F8146D6D1A3897D
:10E710005B063FF536AF09981DB0BDE8F08F03AB3F
:10E7200000932246064B04A94046FDF735FFEAE771
:10E73000D6010100DC010100E001010041C0000040
:10E74000A5E4000038B54B1C144603D14FF0FF354B
:10E75000284638BD938923F020039381636B526868
:10E76000CDB28BB1A36B934208DD23685A1E2260A1
:10E7700003F8015C636801336360E9E7214600F058
:10E780006BFB0028F1D0E1E72169236851B1994280
:10E7900008D213F8011CA94204D1013B01322360C5
:10E7A0006260D5E7C4E90F3204F1440363630323D5
:10E7B000A363234603F8465F23600123DCE710B51B
:10E7C0000C46496B69B104F14403994201D0FDF74D
:10E7D000C3F9236C63600020606313B1E36B2360B3
:10E7E00010BD2369236000236360A38943F02003E5
:10E7F000A3814FF0FF30F3E72DE9F04FADF5257D14
:10E800000DF10C0801930023469347939E4BA2936E
:10E81000DFF87C929D4BCDF8208106460C4692464F
:10E82000A3930A279AF80030002B00F02A8155465E
:10E83000FDF726F915F801BB5844437813F0080397
:10E840001CD06368002B12DDFDF71AF923681A78D3
:10E8500010444278120701D4AA46E3E7479A0132EE
:10E86000479262680133013A62602360E9E7A39B43
:10E870002146304698470028E6D0EDE7BBF1250F4A
:10E8800040F08280459343939AF801302A2B03D1BC
:10E89000102343930AF10205AA4615F8011BA1F1C2
:10E8A0003002092A22D903227948FFF799FA38B1B0
:10E8B000A0EB090301209840439B18434390AA46CC
:10E8C0009AF80030672B0AF101052BD8652B80F0F0
:10E8D0009F80472B10D8452B80F09A80002B6CD05E
:10E8E000252B51D003234993449727E0459B07FBF1
:10E8F0000313303B4593CFE75B2B6AD00CD8582BE2
:10E90000F0D1439A42F400724392102244926E2B4B
:10E910008CBF0423032310E0632B65D0642BE1D16B
:10E920004497F4E7702B4BD026D86E2B62D04CD88E
:10E93000692BD7D100234493032349936368002BA9
:10E9400068DD439B590607D4FDF79AF823681A78C7
:10E9500010444278120764D4499B022B73DC01AB4C
:10E96000224643A9304600F097F8012800F089803C
:10E9700002287FF471AF1DE0752BD1D0782BC0D069
:10E98000732BAFD10223D8E76368002B0CDD23681B
:10E990001A785A4575D1013362682360479B013A62
:10E9A00001336260479357E7A39B2146304698475F
:10E9B0000028ECD04698002859D14FF0FF305CE099
:10E9C000439A42F0200243929BE708234493042396
:10E9D000B3E72946404600F0C9F9439B43F04003A2
:10E9E000439305460123A8E7439B43F04003439329
:10E9F0000023A2E74398C3063FF52EAF019B479A39
:10EA0000191D01911B68C0074CBF1A801A6023E7CB
:10EA1000052392E7A39B214630469847002890D0D3
:10EA2000C8E7479A013247926268013A002A626059
:10EA300002DD0133236087E7A39B214630469847D8
:10EA4000002881D0B6E7042B06DC01AB224643A99F
:10EA5000304600F085F888E70E4B002B3FF4FCAE03
:10EA600001AB224643A93046AFF300807DE7A3897E
:10EA700013F0400F18BF4FF0FF300DF5257DBDE8B6
:10EA8000F08F4698F9E700BF45E70000BFE70000B8
:10EA9000DC010100000000002DE9F04115468A6804
:10EAA00080460C4632B98A69002A14BF4FF0FF3203
:10EAB00001228A602268D1065FBF1A68111D1960A1
:10EAC00017680026A369DBB1012B07D12B686269A7
:10EAD0001B78D35CA3B9002E32D106E0022B07D0FD
:10EAE000002E2DD1A369012B2AD10120BDE8F08190
:10EAF000FCF7C6FF2B681B78184443781B07EFD43C
:10EB00002368DA065EBF2B681B783B702A686B6847
:10EB100002F101022A60A26803F1FF3302F1FF3221
:10EB20006B6006F1010658BF0137A26042B1002BAD
:10EB3000C8DCD4F880312946404698470028C1D027
:10EB4000236813F0100305D1E2680132E260A26984
:10EB500002B13B7023691E4426610020C6E7000015
:10EB60002DE9F04F9A46744B0C468346164693E8BF
:10EB7000070087B003ABA76883E807006F4BA16964
:10EB80006F4A032908BF1A467B1EB3F5AE7F84BFC8
:10EB900040F25D13A3602368009243F4506388BF82
:10EBA0006FF4AE7504F11C0923608CBF7F19002738
:10EBB0004B464FF000080193316803AB022253F833
:10EBC00028000978FFF70CF9019B30B3B8F1010F69
:10EBD0005AD162682AB92268082142F40072616041
:10EBE0002260226822F4A0622260A268511EA16005
:10EBF0009AB13268511C316012781A705D1C7368CA
:10EC0000013B002B736007DCD4F880313146584655
:10EC10009847002840F086802B4608F10108B8F19B
:10EC2000030FC8D162680AB90A2262606268454966
:10EC300060690193891A00F099F8019B4FF0000870
:10EC40001D46A3682268002B3AD03168606991F8AC
:10EC500000C010F80C00002832D0BCF1300F21D1D8
:10EC600010051FD508F1010817B10133013FA3605A
:10EC70007368013B002B73601BDD33680133336025
:10EC8000A368013BA360DCE7B8F1020FADD12268B5
:10EC900002F4C061B1F5007FBFD11021616042F480
:10ECA0008072A1E722F4106222600B782B7001358C
:10ECB000DEE7D4F880313146584698470028DFD047
:10ECC0002368D9050CD54D4508D915F8011CD4F891
:10ECD0007C313246584698476F1E3D464D4529D0F7
:10ECE000226812F0100213D12A706368009E494610
:10ECF0005846B047DAF8003021681A1DCAF80020DB
:10ED000011F0200F1B6810D01860E3680133E36036
:10ED1000A5EB0905A844256945442561002007B0F5
:10ED2000BDE8F08F4FF00008CAE7CA074CBF188053
:10ED30001860EAE70120F2E71C040100B9CC0000EA
:10ED4000FDCD00003804010038B5074C05460846E3
:10ED50001146002222601A4600F012F9431C02D12B
:10ED6000236803B12B6038BD4007002070B50B78D5
:10ED70005E2B13BF4A1C8A1C4B78002108BF01215F
:10ED8000441E00F1FF0504F8011FAC42FBD113B98A
:10ED9000013A104670BD81F00104C454511C11F8B1
:10EDA000015C2D2D01F1FF360A4606D05D2DF0D015
:10EDB0000DB93246EDE72B46EFE70E785D2EFAD01F
:10EDC000B342F8DC01339E42C454FBDC0231E6E777
:10EDD0001F2938B504460D4604D9162303604FF0A9
:10EDE000FF3038BD426C12B152F821304BB9204689
:10EDF00000F030F82A4601462046BDE8384000F0D1
:10EE000017B8012B0AD0591C03D116230360012027
:10EE1000E7E7002442F82540284698470020E0E72D
:10EE2000024B01461868FFF7D3BF00BF3000002037
:10EE300038B5074C0023054608461146236000F00C
:10EE40008FF8431C02D1236803B12B6038BD00BF8B
:10EE50004007002000F074B82DE9F0410C46496BE2
:10EE600004F1440399421DD14FF48061FCF7C2FEC6
:10EE700018B94FF0FF30BDE8F0814FF48063A36311
:10EE800094F84630606380F8FF3394F8453080F89A
:10EE9000FE3394F8443080F8FD3300F2FD302060FA
:10EEA0000020E8E7A66B77003A46FFF7D5FA05465B
:10EEB0000028DED000EB0608014632464046FCF74B
:10EEC0001EFEC4F80080C4E90D57E9E738B5074CC9
:10EED0000023054608461146236000F029F8431C2C
:10EEE00002D1236803B12B6038BD00BF400700206A
:10EEF00038B5064C002305460846236000F028F884
:10EF0000431C02D1236803B12B6038BD40070020A9
:10EF100051F8043C181F002BBCBF0B58C018704799
:10EF2000024B58221A604FF0FF3070474007002014
:10EF3000024B58221A604FF0FF3070474007002004
:10EF4000024B58221A604FF0FF30704740070020F4
:10EF5000024B58221A600020704700BF4007002073
:10EF6000024B58221A604FF0FF30704740070020D4
:10EF7000024B58221A604FF0FF30704740070020C4
:10EF8000024B58221A604FF0FF30704740070020B4
:10EF9000044A05491368002B08BF0B46184410604B
:10EFA000184670473C06002048070020024B5822B4
:10EFB0001A604FF0FF30704740070020FEE700BFA7
:10EFC000F8B500BFF8BC08BC9E467047F8B500BF56
:10EFD000F8BC08BC9E4670476D61700073636D6439
:10EFE0000072636D6400496E3A2000656D697400BB
:10EFF0006974656D00494E3A00204448543232200D
:10F00000747970652E20543D00C2B04320483D0005
:10F01000250044454352454153450044495341422C
:10F020004C45440046414E5F4F4E4C5900494E43BB
:10F030005245415345004F4E00636D6400445259A0
:10F040000066616E00485356004C4F57004D4544D2
:10F0500049554D004F4646005247420073657400C3
:10F06000584F4E004155544F00434F4F4C004841BC
:10F070004C5400484541540048494748006D6F646E
:10F08000650052455354005452554500584F46466A
:10F090000000000000000000000046414C53450005
:10F0A000544F47474C4500454E41424C4544005360
:10F0B00074617475732064656666657265640A00C0
:10F0C00025642C25642C256400556E6B6E6F776E5D
:10F0D00020636D64200A005075623A20002D3E00C6
:10F0E00054787432436D643A0052414D3D002049DA
:10F0F00074656D3D00205375623D00205375666652
:10F100003D0020436D643D00205061723D28003C6D
:10F11000002900536B697020477270005265737448
:10F120006F7265642066726F6D3A005475726E6519
:10F1300064206F66662066726F6D3A00584F4646CF
:10F1400020736B69707065642E2050726576206341
:10F150006D643A005475726E696E6720584F4E0A9E
:10F1600000416C7265616479204163746976650A57
:10F1700000416C726561647920496E6163746976DF
:10F18000650A00416C72656164792048616C746540
:10F19000640A00466F7263652057686974650A00E7
:10F1A0003A204E6F2073746F7265642076616C75BF
:10F1B0006573202D2064656661756C740A00526564
:10F1C00073746F7265643A200050696E3A0053653B
:10F1D00074436D643A002053746F726520002056AA
:10F1E000616C3D00536574466C61673A0020696E3E
:10F1F00076616C696400206163746976650A002039
:10F20000696E6163746976650A00204772703A001E
:10F2100020756E6B6E6F776E0A002076616C756577
:10F220002069732000436C72466C61673A000000ED
:10F23000000000000000000065170000750F0000CE
:10F2400000000000000000000000000000000000BE
:10F2500000000000000000000000000000000000AE
:10F2600020457870697265640A002F616C61726D67
:10F270002F736E7372002F616C61726D2F6F7672D7
:10F28000687400205365743A00204375723A002078
:10F290004F464600204F4E00202D74617267657402
:10F2A000207A6F6E652D006F77004F6E652077694D
:10F2B00072652052656164790A006974656D730036
:10F2C000546865726D6F3A003D4C4F57002C0069D1
:10F2D0006E006D717474000A5B005D20004F4F4D2D
:10F2E0002100536B697070696E672E2E0024636F66
:10F2F0006D6D616E64005365742064796E616D6933
:10F30000632049500A0053617665640A00506173B6
:10F3100073776F726420757064617465640A000AA3
:10F3200055736520746865736520636F6D6D616EDC
:10F3300064733A202768656C7027202D20746869F3
:10F340007320746578740A276D61632064653A617F
:10F35000643A62653A65663A66653A3030272073EA
:10F36000657420616E642073746F7265204D414333
:10F370002D6164647265737320696E204545505237
:10F380004F4D0A276970205B69705B2C646E735B5C
:10F390002C67775B2C7375626E65745D5D5D5D27B0
:10F3A000202D207365742073746174696320495043
:10F3B0000A277361766527202D20736176652063A7
:10F3C0006F6E66696720696E204E5652414D0A275E
:10F3D00067657427205B636F6E666967206164648C
:10F3E000725D27202D2067657420636F6E666967E4
:10F3F0002066726F6D207072652D636F6E6669672F
:10F40000757265642055524C20616E642073746F70
:10F41000726520616464720A276C6F616427202D15
:10F42000206C6F616420636F6E6669672066726F1F
:10F430006D204E5652414D0A2770776427202D20AB
:10F44000646566696E65204D515454207061737314
:10F45000776F72640A276B696C6C27202D207465A6
:10F460007374207761746368646F670A27636C65DF
:10F47000617227202D20636C6561722045455052D2
:10F480004F4D0A277265626F6F7427202D207265B9
:10F49000626F6F7420636F6E74726F6C6C65720054
:10F4A000536176696E6720636F6E66696720746F5B
:10F4B00020454550524F4D2E2E00536176656420F5
:10F4C000746F20454550524F4D004D41433A003E28
:10F4D0003E3E0068656C700073617665006C6F611C
:10F4E0006400676574006D6163006B696C6C007229
:10F4F00065710069700070776400636C656172000B
:10F500007265626F6F74004E6F204D414320636FD0
:10F510006E666967757265643A2073657420666902
:10F52000726D776172652773204D41430A002F6128
:10F530006C61726D6F66662F736E737200536F66C7
:10F5400074207265626F6F74696E672E2E2E0025AF
:10F55000783A25783A25783A25783A25783A257800
:10F56000256300636F756C64206E6F742070617228
:10F5700073653A2000557064617465640A000A720C
:10F58000657175657374204D51545420436F6E66D8
:10F590006967002F726573702F23002F7265712FBA
:10F5A000636F6E6600205361766564002044656673
:10F5B00061756C7420636F6E66696720736572761F
:10F5C000657220757365643A20002F636E662F257F
:10F5D0003032782D253032782D253032782D253077
:10F5E00032782D253032782D253032782E636F6EAB
:10F5F0006669672E6A736F6E00436F6E6669672077
:10F600005552493A20687474703A2F2F0048545468
:10F61000502053746174757320636F64653A2000E1
:10F62000436F6E6669672070617273696E672066EA
:10F6300061696C65640A00446F6E652E0A00436F51
:10F640006E6669672072657472696576696E672097
:10F650006661696C65640A00436F6E6E6563742051
:10F660006661696C65640A000A436F6E6669677556
:10F670007265643A000A6974656D7320000A696EE8
:10F680007075747320000A6D71747420000A312D36
:10F690007769726520004C6F6164696E6720436F03
:10F6A0006E6669672066726F6D20454550524F4DFA
:10F6B000006C6F6164206661696C6564004C6F6109
:10F6C000646564004E6F2073746F72656420636FAD
:10F6D0006E6669670043757272656E74204C414EA8
:10F6E00020636F6E6669672869702C646E732C677F
:10F6F000772C7375626E6574293A00537461727465
:10F70000696E67206C616E004C6F61646564206691
:10F71000726F6D20666C6173682049503A00204416
:10F720004E533A002047573A00204D41534B3A0080
:10F730000A4E6F204950206461746120666F756EB7
:10F740006420696E20666C6173680A004661696CAA
:10F75000656420746F20636F6E66696775726520DB
:10F7600045746865726E6574207573696E672044B0
:10F770004843502E20596F752063616E2073657465
:10F78000206970206D616E75616C6C79210027694C
:10F7900070205B69705B2C646E735B2C67775B2CED
:10F7A0007375626E65745D5D5D5D27202D207365E8
:10F7B00074207374617469632049500A00476F7440
:10F7C00020495020616464726573733A0045455066
:10F7D000524F4D20636C65617265640A000A4C618A
:10F7E0007A79686F6D652E7275204C696768744808
:10F7F000756220636F6E74726F6C6C657220003975
:10F800003335366661375F323031392D31302D3145
:10F81000360020432B2B2076657273696F6E3A0099
:10F820003230313130334C000A282D2957415443AE
:10F8300048444F47000A436F6E66696720736572DC
:10F840007665723A006C617A79686F6D652E7275B3
:10F85000000A4669726D77617265204D414320410F
:10F860006464726573732000435553544F4D5F4673
:10F8700049524D574152455F4D4143000A282D29B9
:10F880004672656552616D207072696E74696E674B
:10F89000000A282B294453323438322D31303000BD
:10F8A0000A282B2957697A4E657435353030000A9D
:10F8B000282D29444D58000A282D294D4F444255E2
:10F8C00053000A282B294F57495245000A282B2953
:10F8D000444854000A282D29434F554E54455200A0
:10F8E0000A282B29484152445245534554206F6EF3
:10F8F0002070696E3D000A282D295245535441520B
:10F90000545F4C414E5F4F4E5F4D5154545F4552D2
:10F91000524F525300446576696365204E616D65B0
:10F920003A005573696E67204D51545420706173CD
:10F9300073776F72642066726F6D20636F6E666995
:10F9400067000A417474656D7074696E67204D516B
:10F95000545420636F6E6E656374696F6E20746FAC
:10F96000200020757365723A00202E2E2E00636FE2
:10F970006E6E656374656420617320002B2F2B2FDE
:10F9800023004177616974696E6720666F72207227
:10F99000657461696E656420746F70696373006675
:10F9A00061696C65642C2072633D0020747279205B
:10F9B000616761696E20696E2035207365636F6EC3
:10F9C000647300543A00416363657074696E672024
:10F9D000636F6D6D616E64732E2E2E0A004E6F2064
:10F9E0006C696E6B004572726F723A2072656E655B
:10F9F000776564206661696C0052656E6577656441
:10FA000020737563636573732E20495020616464AD
:10FA1000726573733A004572726F723A2072656252
:10FA2000696E64206661696C00526562696E64206B
:10FA3000737563636573732E20495020616464722B
:10FA40006573733A0044656C6574696E6720636F13
:10FA50006E662E2052414D207761733A002B005282
:10FA6000657365742041726475696E6F207769747F
:10FA700068206469676974616C2070696E20003267
:10FA80003100246461746174797065006672656523
:10FA90006865617000322E312E3000757074696DAA
:10FAA000652C667265656865617000302D31303097
:10FAB000006C617A79686F6D652E7275004F4E2CFF
:10FAC0004F46462C48414C542C524553542C584FC9
:10FAD0004E2C584F46462C544F47474C45006469BE
:10FAE00073636F6E6E656374656400687376006936
:10FAF0006E746567657200656E756D00246E616D6C
:10FB00006500636F6C6F7200666C6F6174002468CF
:10FB10006F6D696500246E6F646573007265616462
:10FB200079002473746174650024737461747300C4
:10FB300024666F726D617400757074696D6500394B
:10FB40003335366661375F323031392D31302D3102
:10FB500036004C696768744875622000445332343B
:10FB600038325F3130305F4932435F544F5F315735
:10FB70005F42524944474520696E697400445332DC
:10FB80003438322D3130302070726573656E7400F8
:10FB900009436865636B696E6720666F7220312D5B
:10FBA0005769726520646576696365732E2E2E0031
:10FBB00009526573657420646F6E650009445332A1
:10FBC000343832206572726F7200536561726368F7
:10FBD000696E6700312D7769726520636F756E7489
:10FBE0003A2000204E6F64653A0020616C697665AA
:10FBF00000646576230020416464723A002C200082
:10FC00004E6F7420696D706C656D656E746564000F
:10FC1000726F6F7400626373740030313233343545
:10FC20003637383941424344454600696E00735FB8
:10FC30006F7574006D79686F6D65000000000000DD
:10FC40000000000045450000FD4400003345000071
:10FC5000394500003F45000031450000005EBCE230
:10FC6000613FDD83C29C7E20A3FD1F419DC3217F98
:10FC7000FCA2401E5F01E3BD3E6082DC237D9FC18C
:10FC8000421CFEA0E1BF5D0380DE3C62BEE0025C80
:10FC9000DF81633D7C22C09E1D43A1FF4618FAA46C
:10FCA00027799BC584DA3866E5BB5907DB85673958
:10FCB000BAE406581947A5FB7826C49A653BD9874C
:10FCC000045AB8E6A7F91B45C6987A24F8A6441A40
:10FCD00099C7257B3A6486D85B05E7B98CD2306E2C
:10FCE000EDB3510F4E10F2AC2F7193CD114FADF318
:10FCF000702ECC92D38D6F31B2EC0E50AFF1134D0C
:10FD0000CE90722C6D33D18F0C52B0EE326C8ED0FF
:10FD1000530DEFB1F0AE4C1291CF2D73CA947628EB
:10FD2000ABF517490856B4EA6937D58B5709EBB5D7
:10FD300036688AD495CB2977F4AA4816E9B7550BCB
:10FD400088D6346A2B7597C94A14F6A8742AC896BF
:10FD5000154BA9F7B6E80A54D7896B35317720548B
:10FD6000696D656F75740052657365742065727294
:10FD70006F720020636F6D705F69642100005E0028
:10FD8000BC00770156004900436C6F736564002026
:10FD90002D20436C69656E74206275737900533A47
:10FDA000200020536E5352743A2000536F636B65EA
:10FDB000743A200045737461626C6973686564000D
:10FDC000000000000000000035540000C554000091
:10FDD000E9540000015500002D5500005155000068
:10FDE0008955000069540000215500002557000086
:10FDF0008D5700004B54000055540000255400005E
:10FE00000000000000000000095800006B580000CE
:10FE10000558000083580000D75800001F58000004
:10FE20004D5900003558000059580000BD590000D8
:10FE300065580000F9580000AF580000E95700006D
:10FE4000F157000001580000496E697420736B6916
:10FE5000707065640057495A6E6574005265733D51
:10FE600000436F6E74656E742D5479706500436F36
:10FE70006E74656E742D4C656E67746800485454DA
:10FE8000502F2A2E2A200020485454502F312E3132
:10FE900000486F73743A2000557365722D41676591
:10FEA0006E7400636C6F736500436F6E6E65637490
:10FEB000696F6E004745540000000000000000001C
:10FEC000676E0000436E0000156C0000976B000029
:10FED000496B0000516B0000596B0000756B00000E
:10FEE000ED6B0000216D00007D6B0000856B000054
:10FEF00069720000657200008F6B0000936B000058
:10FF00005472616E736665722D456E636F64696EBF
:10FF1000673A206368756E6B656400436F6E746545
:10FF20006E742D4C656E6774683A2000417264757A
:10FF3000696E6F2F322E322E30006E756C6C00663B
:10FF4000616C73650074727565002200000000002A
:10FF500000000000117300005B8B00002D73000097
:10FF600085730000A37200009F7200009B72000066
:10FF70000000000000000000EB7200005B8B00003E
:10FF8000D772000061730000A37200009F7200002E
:10FF90009B7200003E3E20000D0A00496E76616CA7
:10FFA000696420636F6D6D616E6400000000000085
:10FFB00000000000B17E0000CD7E00000B000000BC
:10FFC0000C0000000D0000000E0000000F000000FB
:10FFD00010000000110000001200000013000000DB
:10FFE00014000000160000001700000018000000B8
:10FFF0001900000003000000040000001C000000C5
:020000021000EC
:100000001D0000001E0000001F0000000500000091
:10001000020000001A0000001B00000008000000A1
:10002000060000000000000000000000DD8A000063
:100030006E616E00696E66006F76660000000000FB
:1000400000000000159100005B8B00008D91000006
:100050009991000093910000139100000B91000012
:10006000A1910000319100000791000000C0014003
:100070000010024000200240705F73706920213D33
:10008000204E554C4C002F55736572732F616E6472
:100090007265792F2E706C6174666F726D696F2F47
:1000A0007061636B616765732F6672616D65776FF1
:1000B000726B2D61726475696E6F6E6F72646963C5
:1000C0006E7266352F6C69627261726965732F5347
:1000D00050492F5350492E63707000535049436C60
:1000E0006173733A3A535049436C617373284E52AB
:1000F000465F5350495F547970652A2C2075696EAC
:1001000074385F742C2075696E74385F742C207598
:10011000696E74385F742900706F7700000000000A
:10012000000000000000304300000000000030C369
:100130002C2066756E6374696F6E3A20006173736C
:10014000657274696F6E2022257322206661696C66
:1001500065643A2066696C6520222573222C206C28
:10016000696E65202564257325730A000000000070
:10017000000000000000000000000000000000007F
:10018000000000000000000000000000000000006F
:10019000000000000000000000000000000000005F
:1001A000000000000000000000000000000000004F
:1001B000000000000000000000000000000000003F
:1001C00000000000000000000000000034000020DB
:1001D000504F53495800232D302B2000686C4C00A1
:1001E00065666745464700494E46004E414E003021
:1001F000313233343536373839414243444546008D
:10020000303132333435363738396162636465668C
:1002100000002020202020202020202828282828F6
:1002200020202020202020202020202020202020CE
:100230002020881010101010101010101010101026
:100240001010040404040404040404041010101026
:1002500010101041414141414101010101010101E1
:100260000101010101010101010101010110101051
:1002700010101042424242424202020202020202B4
:100280000202020202020202020202020210101024
:10029000102000000000000000000000000000002E
:1002A000000000000000000000000000000000004E
:1002B000000000000000000000000000000000003E
:1002C000000000000000000000000000000000002E
:1002D000000000000000000000000000000000001E
:1002E000000000000000000000000000000000000E
:1002F00000000000000000000000000000000000FE
:1003000000000000000000000000000000000000ED
:100310000000496E66696E697479004E614E000096
:100320000080E03779C34143176E05B5B5B89346F1
:10033000F5F93FE9034F384D321D30F94877825ABD
:100340003CBF737FDD4F1575000000000000F03FDB
:1003500000000000000024400000000000005940A0
:100360000000000000408F40000000000088C340F3
:1003700000000000006AF8400000000080842E4168
:1003800000000000D01263410000000084D79741B4
:100390000000000065CDCD41000000205FA00242BA
:1003A000000000E876483742000000A2941A6D422F
:1003B000000040E59C30A2420000901EC4BCD64222
:1003C00000003426F56B0C430080E03779C34143CD
:1003D00000A0D8855734764300C84E676DC1AB4343
:1003E000003D9160E458E143408CB5781DAF154461
:1003F00050EFE2D6E41A4B4492D54D06CFF080443C
:10040000F64AE1C7022DB544B49DD9794378EA4450
:1004100005000000190000007D0000003A04010002
:100420009DF800003D040100412D46612D663839DC
:1004300030313233343536375D002B2D007858009B
:0404400000000000B8
:08044400FCFFFE7F0100000037
:10044C00000401002CFF00001BFF000000FF000057
:10045C000090D003FFFFFFFFFFFFFFFFFFFFFFFF39
:10046C000A0000000100000008000000010000006C
:10047C0034000020000000008C010100AC010100E0
:10048C006C010100000000000000000000000000F2
:10049C000000000000000000000000000000000050
:1004AC000000000000000000000000000000000040
:1004BC000000000000000000000000000000000030
:1004CC000000000000000000000000000000000020
:1004DC0000000000430000000000000000000000CD
:1004EC000000000000000000000000000000000000
:1004FC0000000000430000000000000000000000AD
:10050C0000000000000000000000000000000000DF
:10051C00000000004300000000000000000000008C
:10052C0000000000000000000000000000000000BF
:10053C00000000004300000000000000000000006C
:10054C00000000000000000000000000000000009F
:10055C00000000004300000000000000000000004C
:10056C00000000000000000000000000000000007F
:10057C00000000004300000000000000000000002C
:10058C00000000000000000000000000000000005F
:10059C00000000004300000000000000000000000C
:1005AC00000000000000000000000000000000003F
:1005BC0000000000F1CE0000BDBA000000000000F9
:1005CC00110201006CF900009AFF00009AFF000074
:1005DC009AFF00009AFF00009AFF00009AFF0000AB
:1005EC009AFF00009AFF00009AFF0000FFFFFFFF38
:1005FC00FFFFFFFFFFFFFFFFFFFF00000100415364
:10060C004349490000000000000000000000000009
:10061C00000000000000000000000000000041533A
:10062C0043494900000000000000000000000000E9
:10063C0000000000000000000000000000000000AE
:10064C0025040000B5040000D1040000ED040000F6
:10065C0015080000751F0000991F00008939000063
:10066C00D5410000E1440000AD480000E953000012
:10067C00CD570000195A0000A16000002561000050
:10068C00956700006D720000817C0000B986000047
:0C069C00A1930000859A000001040000FA
:0400000300008EC1AA
:00000001FF
